:020000040000FA
:04000000ADEF00F070
:100008005582D9CF05F0DACF06F00F0112A91BD01F
:100018008EBC02D0839483928EA802D083A20ED085
:10002800899425EE04F0010EDBBE07D0000EDE5CDD
:10003800020EDE5802E3899201D089828EB883B21B
:1000480001D08984129912A17CD08EB883B289928A
:10005800901C076E8E1C086E04C509F005C50AF0D1
:100068000ABE03D0020E0A5C2FE28EA802D083A239
:100078002BD0094A0A2A09C004F50AC005F502C5A9
:1000880009F003C50AF0060E0924D96E050E0A20E8
:10009800DA6E07C0DFFF060E0924D96E070E0A20A4
:1000A800DA6E08C0DFFF094A0A2A0168010E026EEB
:1000B80009C003F00AC004F00150031602500416E8
:1000C80003C002F504C003F58EB883B2898489841D
:1000D8008EA0FED78EA802D083A202D0899401D028
:1000E800898425EE04F0010EDBBE07D0FB0EDE5C32
:1000F800010EDE5802E3899201D0898208A81FD038
:100108000BD0838202D0838405D0839418D083A235
:1001180016D08394839213D007507F0B016E026A26
:1001280002500DE10150040AF2E0100AF0E0340A2E
:10013800E8E01F0AEFE07F0AE6E01F0AE6E00F01A9
:1001480012910E01CA9906C0DAFF05C0D9FF55926F
:1001580011000FEF51F07DC0D9FF7EC0DAFFDE6AD3
:10016800DD6A7CC00BF0B4EC46F00BC098F00CC014
:1001780099F0000199BF0B0CD8909835D96E993534
:10018800DA6E860ED926010EDA22DECFAFF0DDCF89
:10019800B0F0AF51B01101E10C0C7DC0D9FF7EC0A9
:1001A800DAFFAFC0DEFFB0C0DDFF7F91AFC0D9FF7F
:1001B800B0C0DAFFDF5012E020EE01F0AF51D926CF
:1001C800B051DA22DF50EDEC60F00001A46FA4B169
:1001D80005D07F51D8A4A4A5000C0A0CAFC0D9FF44
:1001E800B0C0DAFFDF6A20EE01F0AF51D926B05176
:1001F800DA2298C0DFFF20EE01F0AF51D926B051C6
:10020800DA22DF5056EC43F00001A46FA4B1030CCE
:100218007F5102E0A4B50A0CAFC060F0B0C061F035
:10022800636B626B4FEC47F060C0ADF061C0AEF03D
:10023800040EAD19AE1101E1010CAE5103E1020E3D
:10024800AD5D01E30D0C20EE2BF0AF51D926B05176
:10025800DA22DECFA0F0DECFA1F0DECFA2F0DECF33
:10026800A3F03A0EAF250B6E000EB0210C6EDAEC3F
:100278005EF0020E0C180B1001E00D0C450E00018B
:10028800AF250B6E000EB0210C6EDAEC5EF00BC0E1
:10029800A9F00CC0AAF00001AB6BAC6BA951AA1174
:1002A800AB11AC1110E1530EAF250B6E000EB0214F
:1002B8000C6E01EC54F00BC0A9F00CC0AAF00DC0F4
:1002C800ABF00EC0ACF0000120EE17F0AF51D9260C
:1002D800B051DA22A9C0DEFFAAC0DEFFABC0DEFF44
:1002E800ACC0DEFF20EE3FF0AF51D926B051DA2284
:1002F80010EE02F0AF51E126B051E222DFCFE7FF66
:1003080020EE02F0AF51D926B051DA22DE040AE01D
:1003180020EE02F0AF51D926B051DA22020EDE18D3
:1003280001E00D0CA9C00BF0AAC00CF0ABC00DF099
:10033800ACC00EF020EE02F0AF51D926B051DA224F
:10034800DF500F6E106A116A126AC4EC57F00BC0C6
:10035800A9F00CC0AAF00DC0ABF00EC0ACF020EEB6
:100368003CF0AF51D926B051DA22DF50806F816B53
:1003780020EE09F0AF51D926B051DA2280C0DEFF55
:1003880081C0DDFF20EE09F0AF51D926B051DA2245
:10039800DE50DE10D8B40D0C20EE09F0AF51D9268E
:1003A800B051DA22DECF80F0DDCF81F08269836937
:1003B80020EE09F0AF51D926B051DA22DECF84F011
:1003C800DDCF85F08251842783518523805184179E
:1003D800815185178451851101E00D0C400EAF2520
:1003E8000B6E000EB0210C6EDAEC5EF0000120EE10
:1003F80007F0AF51D926B051DA220BC0DEFF0CC08E
:10040800DDFF20EE07F0AF51D926B051DA22DF50D8
:10041800806F0F0E801701E00D0C420EAF250B6E9A
:10042800000EB0210C6EDAEC5EF00BC09CF00CC034
:100438009DF000019E6B9F6B9C519D119E119F1119
:1004480010E14F0EAF250B6E000EB0210C6E01ECC3
:1004580054F00BC09CF00CC09DF00DC09EF00EC077
:100468009FF03D0E0001AF250B6E000EB0210C6E03
:10047800DAEC5EF00BC09AF00CC09BF000019A51C8
:100488009B1101E10D0C20EE07F0AF51D926B051B8
:10049800DA22DECF80F0DDCF81F0040E826FD890B3
:1004A80081338033822FFBD79A518025836F9B51EC
:1004B8008121846F856BD8B0852B866BA9518325E4
:1004C800946FAA518421956FAB518521966FAC51D9
:1004D8008621976F94519C5D95519D5996519E59CF
:1004E80097519F5901E20D0C94519C5D0B6E9551EB
:1004F8009D590C6E96519E590D6E97519F590E6ECF
:1005080020EE09F0AF51D926B051DA22DECF80F0C3
:10051800DDCF81F080C00FF081C010F0116A126A3F
:1005280044EC58F00BC0A5F00CC0A6F00DC0A7F025
:100538000EC0A8F00001A551A611A711A81101E14C
:100548000D0CAD6BAE6BF60EA55DFF0EA659FF0E3A
:10055800A7590F0EA85903E2AE6B030EAD6FA85151
:10056800A71108E1F60EA55DFF0EA65903E2AE6BD2
:10057800020EAD6FA851A71108E1F60EA55D0F0E8A
:10058800A65903E2AE6B010EAD6FAD51AE1101E19C
:100598000D0C020EA525806F000EA621816F000E9E
:1005A800A721826F000EA821836F20EE13F0AF51B0
:1005B800D926B051DA2280C0DEFF81C0DEFF82C0BA
:1005C800DEFF83C0DEFF20EE1BF0AF51D926B0510D
:1005D800DA22A0C0DEFFA1C0DEFFA2C0DEFFA3C0FA
:1005E800DEFF9A51A025806F9B51A121816F000EDB
:1005F800A221826F000EA321836F20EE1FF0AF515E
:10060800D926B051DA2280C0DEFF81C0DEFF82C069
:10061800DEFF83C0DEFF9451A025806F9551A12194
:10062800816F9651A221826F9751A321836F20EE8B
:1006380027F0AF51D926B051DA2280C0DEFF81C041
:10064800DEFF82C0DEFF83C0DEFF030EAD19AE11F0
:100658004DE1590EAF250B6E000EB0210C6EDAEC91
:100668005EF00B500C1001E00D0C000120EE07F0BD
:10067800AF51D926B051DA22DE50DE1001E00D0C60
:100688005B0EAF250B6E000EB0210C6E01EC54F022
:10069800000120EE23F0AF51D926B051DA220BC069
:1006A800DEFF0CC0DEFF0DC0DEFF0EC0DEFF20EE59
:1006B80013F0AF51D926B051DA22DECF80F0DECF69
:1006C80081F0DECF82F0DECF83F0020ED890803743
:1006D800813782378337E82EF9D780C090F081C000
:1006E80091F082C092F083C093F0B8D020EE07F06A
:1006F800AF51D926B051DA22DE50DE1001E10D0CDF
:1007080020EE1FF0AF51D926B051DA22DECF80F0AB
:10071800DECF81F0DECF82F0DECF83F0A9518025D5
:10072800846FAA518121856FAB518221866FAC51AC
:100738008321876F20EE23F0AF51D926B051DA22FA
:1007480084C0DEFF85C0DEFF86C0DEFF87C0DEFF17
:10075800020EAD19AE116BE020EE13F0AF51D926A1
:10076800B051DA22DECF80F0DECF81F0DECF82F02A
:10077800DECF83F0010E8015846F856B866B876BE7
:1007880020EE13F0AF51D926B051DA22DECF88F02F
:10079800DECF89F0DECF8AF0DECF8BF0030E880340
:1007A800F3CF8CF0F4CF8DF08E6B8F6B8903F35001
:1007B8008D27F4508E23000E8F238803F3508D2746
:1007C800F4508E23000E8F23030E8A03F3508E27D6
:1007D800F4508F23000E8903F3508E27F4508F2393
:1007E800000E8803F3508E27F4508F23030E8B03DB
:1007F800F3508F27000E8A03F3508F27000E8903CA
:10080800F3508F27000E8803F3508F27D8908F332B
:100818008E338D338C3384518C25906F85518D2187
:10082800916F86518E21926F87518F2116D020EEBD
:1008380013F0AF51D926B051DA22DECF80F0DECFE7
:1008480081F0DECF82F0DECF83F0D8908035906FD4
:100858008135916F8235926F8335936FFF0E9025A6
:10086800806F010E9121816F000E9221826F000E20
:100878009321836F0A0E05D0D89083338233813356
:100888008033E82EF9D720EE17F0AF51D926B051B2
:10089800DA228051DE5C8151DE588251DE58835164
:1008A800DE5801E20D0C20EE0FF0AF51D926B05101
:1008B800DA22DE68DE68DE68DD68DD52DD5210EEC1
:1008C8000BF0AF51E126B051E222DECFE6FFDECFDA
:1008D800E6FFDECFE6FFDECFE6FF20EE04F0AF5105
:1008E800D926B051DA22800EDF6E030EAD19AE1193
:1008F80001E090D05F0EAF250B6E000EB0210C6E9C
:10090800DAEC5EF00B040C1001E084D0AFC037F0D5
:10091800B0C038F0010E0001A025396E000EA121EB
:100928003A6E000EA2213B6E000EA3213C6EF6EC3F
:1009380054F000096FE1000120EE04F0AF51D92610
:10094800B051DA22DF6A2D0EAF250B6E020EB021F0
:100958000C6EDAEC5EF0550E0B185CE1AA0E0C1862
:1009680059E12F0E0001AF250B6E000EB0210C6E61
:1009780001EC54F0520E0B184DE1520E0C184AE1DE
:10098800610E0D1847E1410E0E1844E1130E0001E7
:10099800AF250B6E020EB0210C6E01EC54F0720EF6
:1009A8000B1838E1720E0C1835E1410E0D1832E1C2
:1009B800610E0E182FE1170E0001AF250B6E020E07
:1009C800B0210C6E01EC54F0000120EE0FF0AF5195
:1009D800D926B051DA220BC0DEFF0CC0DEFF0DC0F5
:1009E800DEFF0EC0DEFF1B0EAF250B6E020EB02120
:1009F8000C6E01EC54F0000120EE0BF0AF51D9263B
:100A0800B051DA220BC0DEFF0CC0DEFF0DC0DEFFE6
:100A18000EC0DEFFAFC0D9FFB0C0DAFFADC0DFFF48
:100A28000101844B852B000120EE05F0AF51D9263A
:100A3800B051DA2284C1DEFF85C1DDFF000C74C02D
:100A480077F075C078F001017A6B7B6B91D373C036
:100A580048F0770E496E76C04AF04950D96EDA6A86
:100A6800DECFF6FFDDCFF7FFF86A000EF86E08005C
:100A7800F550250AD8A45ED34950D96EDA6ADE2A21
:100A8800000EDD2201017C6B7D6B4B6A4C6A7E692E
:100A98007F694950D96EDA6ADECFF6FFDDCFF7FFFE
:100AA800F86A000EF86E0800F550640AD8B40FD042
:100AB8004950D96EDA6ADECFF6FFDDCFF7FFF86A64
:100AC800000EF86E0800F550690AD8A47ED1495086
:100AD800D96EDA6ADE2A000EDD224A50D96EDA6A49
:100AE800DF50DF2ADF2AD96EDA6ADECF62F0DDCF87
:100AF80063F00001000E63BFFF0E646F656F666FE1
:100B0800676F686F696F48C025F062C026F063C0E0
:100B180027F064C028F065C029F066C02AF067C0D5
:100B28002BF068C02CF069C02DF026C03EF027C01D
:100B38003FF028C040F029C041F02AC042F02BC045
:100B480043F02CC044F02DC045F045AE02D0010E54
:100B580001D0000E3C6E3D6A3C503D10D8B410D018
:100B6800451E441E431E421E411E401E3F1E3E6C33
:100B7800000E3F22402241224222432244224522A3
:100B880001017FBF01D04B927FBF05D07F5107E1A4
:100B98007E05D8B004D0396A010E386E04D07EC103
:100BA80038F07FC139F07CC13AF07DC13BF03C5050
:100BB8003D10D8A402D04BA403D03A06D8A03B06D7
:100BC800476A1F0E466E0201B86B6ED04606D8A063
:100BD8004706990E4624D96E020E4720DA6E3EC0AB
:100BE8000BF03FC00CF040C00DF041C00EF042C009
:100BF8000FF043C010F044C011F045C012F00A0EC7
:100C0800136E146A156A166A176A186A196A1A6AD4
:100C1800BFEC4AF00BC02EF00CC02FF00DC030F026
:100C28000EC031F00FC032F010C033F011C034F0F4
:100C380012C035F02EC01DF030C01EF025EC5FF05C
:100C48001D50300FDF6E3806D8A039063A06D8A0F6
:100C58003B063EC00BF03FC00CF040C00DF041C059
:100C68000EF042C00FF043C010F044C011F045C070
:100C780012F00A0E136E146A156A166A176A186A51
:100C8800196A1A6A12EC46F00BC03EF00CC03FF02D
:100C98000DC040F00EC041F00FC042F010C043F04C
:100CA80011C044F012C045F047BE1FD0475003E1C1
:100CB8004604D8A01AD03E503F10401041104210B0
:100CC800431044104510D8A481D739BE05D03950F7
:100CD80002E13804D8B07AD73BBE07D03B5003E1D5
:100CE8003A04D8A002D04BB271D73C503D10D8A4DA
:100CF80002D04BA415D04606D8A047063C503D105C
:100D0800D8A403D0376A2B0E02D0376A2D0E366E60
:100D1800990E4624D96E020E4720DA6E36C0DFFFE0
:100D280025C01AF0990E46241B6E020E47201C6E31
:100D38003AC01DF03BC01EF04BA008D01BC014F0F9
:100D48001CC015F01AC016F06BEC5FF01EBE05D083
:100D58001DC022F01EC023F002D0226A236A206A36
:100D6800216A0AD0000E0D6E200E0C6E1AC00EF00D
:100D78003DEC57F0204A212A2250205C2150800A5D
:100D88001F6E2350800A1F58D8A0ECD74BB008D04C
:100D98001BC014F01CC015F01AC016F06BEC5FF005
:100DA8001BC00BF01CC00CF01BEC5DF022500B2498
:100DB8001A6E23500C201B6E1AC025F01BC026F09B
:100DC80025C048F026C049F0CED14950D96EDA6A1C
:100DD800DECFF6FFDDCFF7FFF86A000EF86E0800E9
:100DE800F550780AD8B40FD04950D96EDA6ADECFF8
:100DF800F6FFDDCFF7FFF86A000EF86E0800F55031
:100E0800580AD8A46DD14950D96EDA6ADECFF6FFF8
:100E1800DDCFF7FFF86A000EF86E0800F5CF72F024
:100E28004950D96EDA6ADE2A000EDD224A50D96EA0
:100E3800DA6ADF50DF2ADF2AD96EDA6ADECF60F09D
:100E4800DDCF61F060C06AF061C06BF000016C6BCF
:100E58006D6B6E6B6F6B706B716B48C024F06AC002
:100E680025F06BC026F06CC027F06DC028F06EC06E
:100E780029F06FC02AF070C02BF071C02CF072C03E
:100E88002DF001017FBF01D04B927FBF05D07F516C
:100E980007E17E05D8B004D0376A010E366E04D05B
:100EA8007EC136F07FC137F07CC140F07DC141F092
:100EB8004BA804D0FE0E4026FF0E412225C038F074
:100EC80026C039F027C03AF028C03BF029C03CF0D2
:100ED8002AC03DF02BC03EF02CC03FF0456A1F0EE3
:100EE800446E0201B86B6DD04406D8A045060F0EBB
:100EF8003814426E436A43BE08D0435004E10A0ED8
:100F0800425CD8A002D0570E01D0300E4226000E07
:100F18004322BF0E2E6E2F682D50306E316A2E5030
:100F280030262F503122315005E11A0E305C02E292
:100F3800010E01D0000E326E336A32503310D8B42D
:100F480025D09F0E2E6E2F68200E4210306E000E98
:100F58004310316E2E5030262F503122315005E18A
:100F68001A0E305C02E2010E01D0000E346E356AB2
:100F780034503510D8B40AD042C011F043C012F032
:100F8800D8EC5CF011C042F012C043F0990E442432
:100F9800D96E020E4520DA6E42C0DFFF3606D8A0B1
:100FA80037064006D8A04106040E2E6ED8903F3270
:100FB8003E323D323C323B323A32393238322E2ED2
:100FC800F5D745BE20D0455004E1020E445CD8A0B8
:100FD8001AD0385039103A103B103C103D103E10D2
:100FE8003F10D8A481D737BE05D0375002E1360468
:100FF800D8B07AD741BE07D0415003E14004D8A009
:1010080002D04BB271D74BA816D04406D8A04506DB
:10101800990E4424D96E020E4520DA6E2DC0DFFFEA
:101028004406D8A04506990E4424D96E020E4520E0
:10103800DA6E300EDF6E24C01AF0990E44241B6E4F
:10104800020E45201C6E40C01DF041C01EF04BA092
:1010580008D01BC014F01CC015F01AC016F06BECB9
:101068005FF01EBE05D01DC022F01EC023F002D0C6
:10107800226A236A206A216A0AD0000E0D6E200EA9
:101088000C6E1AC00EF03DEC57F0204A212A22506F
:10109800205C2150800A1F6E2350800A1F58D8A058
:1010A800ECD74BB008D01BC014F01CC015F01AC008
:1010B80016F06BEC5FF01BC00BF01CC00CF01BECC7
:1010C8005DF022500B241A6E23500C201B6E1AC0A0
:1010D80024F01BC025F024C048F025C049F043D0B7
:1010E8004950D96EDA6ADECFF6FFDDCFF7FFF86A2E
:1010F800000EF86E0800F550250AD8A412D0495001
:10110800D96EDA6ADE2A000EDD22000E0D6E250E7B
:101118000C6E48C00EF03DEC57F0496A010E486E5F
:1011280022D04950D96EDA6ADE2A000EDD22486ADA
:10113800496A19D04950D96EDA6ADECFF6FFDDCF99
:10114800F7FFF86A000EF86E0800F5500C6E0D6A8D
:1011580048C00EF03DEC57F04950D96EDA6ADE2AE5
:10116800000EDD22DAD7485001017A2749507B2347
:1011780077C0F6FF78C0F7FF0800F55001E067D4A4
:101188007AC173F07BC174F0120097C0ADF098C0BB
:10119800AEF09B51D96EDA6ADE6ADD6A95C00CF052
:1011A80096C00DF0BD0E0E6E57EC53F00001AC6FFB
:1011B800AC510AE120EE0FF09551D9269651DA226A
:1011C800DF50AC6FAC5102E0AC51120020EE0EF0D3
:1011D8009551D9269651DA22DFA2070C20EE10F09D
:1011E8009551D9269651DA2210EE10F09551E12644
:1011F8009651E222E6CFA0F0E6CFA1F0E6CFA2F02A
:10120800E6CFA3F09951A025A46F9A51A121A56F0B
:10121800000EA221A66F000EA321A76FDE50A45DC9
:10122800DE50A559DE50A659DE50A75901E3DFD29A
:1012380020EE10F09551D9269651DA22DECF9CF097
:10124800DDCF9DF09C1D996F9D1D9A6FD0D220EE29
:1012580010F09551D9269651DA22FF0EDE149C6FB4
:10126800010EDE149D6F000EDE149E6F000EDE145C
:101278009F6F9C519D119E119F1101E0FDD120EEA1
:1012880010F09551D9269651DA22DECF9CF0DECFA8
:101298009DF0DECF9EF0DECF9FF00A0E05D0D890ED
:1012A8009F339E339D339C33E82EF9D7A069A169FB
:1012B80020EE09F0BD51D926BE51DA22DECFA2F0C8
:1012C800DDCFA3F0A051A227A151A3239C51A215C1
:1012D800AF6F9D51A315B06FAF1101E091D020EE13
:1012E80010F09551D9269651DA22DE50DE10DE1024
:1012F800DE101EE120EE06F09551D9269651DA222D
:10130800DECFB7F0DECFB8F0DECFB9F0DECFBAF07F
:10131800B751B811B911BA1127E195C078F096C044
:1013280079F07A6B7B6B7C6B7D6B10EC23F014D0BF
:1013380095C078F096C079F020EE14F09551D92632
:101348009651DA22DECF7AF0DECF7BF0DECF7CF06A
:10135800DECF7DF010EC23F078C0B7F079C0B8F09C
:101368007AC0B9F07BC0BAF0B751B811B911BA1147
:1013780001E141D2B705B811B911BA1109E120EE5E
:101388000FF09551D9269651DA22020EDF6E020C23
:10139800B7290FE1B8290DE1B9290BE1BA2909E10B
:1013A80020EE0FF09551D9269651DA22010EDF6E04
:1013B800010C20EE14F09551D9269651DA22B7C0C7
:1013C800DEFFB8C0DEFFB9C0DEFFBAC0DEFF20EE28
:1013D80006F09551D9269651DA22DE50DE10DE103D
:1013E800DE100EE120EE06F09551D9269651DA224C
:1013F800B7C0DEFFB8C0DEFFB9C0DEFFBAC0DEFF8F
:1014080020EE18F09551D9269651DA2210EE2BF0DD
:10141800BD51E126BE51E222DE50E61812E1DE504F
:10142800E6180FE1DE50E6180CE1DE50E61809E197
:10143800BDC024F0BEC025F014EC44F0000901E062
:1014480053D1BDC00BF0BEC00CF0000120EE14F06B
:101458009551D9269651DA22DECF0DF0DECF0EF067
:10146800DECF0FF0DECF10F04DEC4BF00BC0B3F039
:101478000CC0B4F00DC0B5F00EC0B6F00001B35109
:10148800B411B511B61101E17AD7AF51B327B051F4
:10149800B423000EB523B62399C09CF09AC09DF0E2
:1014A800090E9E6FD8909D339C339E2FFBD79CC00E
:1014B800B1F09DC0B2F0B151B21101E1A2D0B15169
:1014C800AF259C6FB251B0219D6F20EE09F0BD5140
:1014D800D926BE51DA229C51DE5C9D51DE5810E2BD
:1014E80020EE09F0BD51D926BE51DA22DECF9CF09C
:1014F800DDCF9DF0AF519C5DB16FB0519D59B26F7A
:10150800ADC01AF0AEC01BF0B3C01CF0B4C01DF0E3
:10151800B5C01EF0B6C01FF0B1C020F0B2C021F0B7
:1015280020EE01F0BD51D926BE51DA22DF50C0ECC1
:101538004FF0000901E0D8D00001B1519C6FB251C1
:101548009D6F9E6B9F6B20EE2BF0BD51D926BE512F
:10155800DA22DECFA0F0DECFA1F0DECFA2F0DECF20
:10156800A3F0B351A05DA46FB451A159A56FB551B3
:10157800A259A66FB651A359A76F9C51A45D9D515E
:10158800A5599E51A6599F51A7592CE22F0EBD254A
:101598000B6E000EBE210C6E20EE2BF0BD51D9262D
:1015A800BE51DA22DECF9CF0DDCF9DF0B3519C5FB7
:1015B800B4519D5B090ED8909C379D37E82EFBD718
:1015C8009C51AD250D6E9D51AE210E6E020E106E12
:1015D8000F6A3CEC5DF020EE03F0BD51D926BE51F8
:1015E800DA22DF6AB1C09CF0B2C09DF0090ED89033
:1015F8009C379D37E82EFBD79CC0BBF09DC0BCF044
:10160800A7D020EE0AF09551D9269651DA2210EE8D
:1016180010F09551E1269651E222DE50E65CDE504C
:10162800E658DE50E658DE50E65818E3BDC024F010
:10163800BEC025F014EC44F0000901E055D00001CB
:1016480020EE2BF0BD51D926BE51DA22B3C0DEFF01
:10165800B4C0DEFFB5C0DEFFB6C0DEFF20EE18F076
:101668009551D9269651DA22B3C0DEFFB4C0DEFF09
:10167800B5C0DEFFB6C0DEFF9C69010E9D6F20EE8F
:1016880010F09551D9269651DA22DECF9EF0DDCFA3
:101698009FF09C519E179D519F179E510008BB6F4C
:1016A8009F51D8A0E82A0208BC6FBB51995DBC5174
:1016B8009A5904E299C0BBF09AC0BCF0BDC037F09B
:1016C800BEC038F020EE18F09551D9269651DA228E
:1016D800DECF39F0DECF3AF0DECF3BF0DECF3CF0A4
:1016E800F6EC54F0000902E000015AD600019C69AA
:1016F800010E9D6F20EE10F09551D9269651DA22F1
:10170800DECF9EF0DDCF9FF09C519E179D519F1715
:10171800BDC0A0F0BEC0A1F09E51A0279F51A1233B
:101728002F0EA0250B6E000EA1210C6EADC00DF082
:10173800AEC00EF0BBC00FF0BCC010F03CEC5DF0CA
:1017480020EE03F0BD51D926BE51DA22010EDF6E1C
:10175800BB51995FBC519A5B9B51D96EDA6ABB51F8
:10176800DE26BC51DD22BB51AD27BC51AE2320EE95
:1017780010F09551D9269651DA22BB51DE26BC517C
:10178800DE22000EDE22DE2220EE10F09551D92650
:101798009651DA2210EE0AF09551E1269651E2228E
:1017A800DE50E65CDE50E658DE50E658DE50E6587D
:1017B80020EE0AF0D8A020EE10F09551D9269651C7
:1017C800DA22DECFA8F0DECFA9F0DECFAAF0DECF96
:1017D800ABF020EE0AF09551D9269651DA22A8C02E
:1017E800DEFFA9C0DEFFAAC0DEFFABC0DEFF995155
:1017F8009A1101E02CD520EE0EF09551D92696517C
:10180800DA22000EDB8C000C0C6E0B6AB3D20C5083
:1018180009E14F5007E00B6A0101836B0A0EA5D05E
:1018280083901AD3020E0C1807E14F5005E00B6A9B
:101838000101836B140E99D01F0E0C6437D0300E43
:101848000C6034D04F5032E00C50E00F506E0B6AF1
:101858000F0E501805E192C14EF00101926B6CD247
:101868005050220D0A0EF324D96E030EF420DA6EBE
:10187800DE50DE10DE10DE1003E0030E50645CD292
:10188800010E4E6E50501C0D1B0EF324D96E010E26
:10189800F420DA6E50501C0D1B0EF324E16E010E7D
:1018A800F420E26EE7501009DF6E46D23F0E0C645A
:1018B80028D0500E0C6025D04F5023E050501C0DFE
:1018C800000EF324D96E010EF420DA6E0C50C00F0E
:1018D800DF6E50501C0D000EF324D96E010EF4205B
:1018E800DA6EDF500CE050501C0D1B0EF324D96E3D
:1018F800010EF420DA6E100EDF6E010E4E6E0B6ACA
:101908001BD2310E0C1807E14F5005E00C0E0101F7
:10191800836F1D0E26D2340E0C1807E14F5005E0D8
:101928000101826B836B0B6A7BD7350E0C1808E1BB
:101938004F5006E00B6A0D0E0101836FAC0E15D0F7
:10194800370E0C1808E14F5006E083800E0E010197
:10195800836F750E06D20D0E0C1809E14F5007E083
:101968000B6A020E0101836FBC0E826F59D7100EED
:101978000C1807E14F5005E0030E0101836FE90ED3
:10198800F0D1180E0C1807E14F5005E0070E0101C1
:10199800836F090EE6D13B0E0C1807E14F5005E0A6
:1019A8000E0E0101836F7E0EDCD13E0E0C1801E095
:1019B80053D24F5001E150D20F0E0101836F3D0EFB
:1019C800D0D150501C0D010EF324D96E010EF42015
:1019D800DA6E0CC0DFFF030E0101836FEA0EC1D17E
:1019E80050501C0D020EF324D96E010EF420DA6E4D
:1019F8000CC0DFFF030E0101836FEB0EB2D1505014
:101A08001C0D030EF324D96E010EF420DA6E0CC0FF
:101A1800DFFF030E0101836FEC0EA3D150501C0DA4
:101A2800040EF324D96E010EF420DA6E0CC0DFFF29
:101A3800030E0101836FED0E94D150501C0D050E5D
:101A4800F324D96E010EF420DA6E0CC0DFFF030E0A
:101A58000101836FEE0E85D150501C0D060EF32444
:101A6800D96E010EF420DA6E0CC0DFFF50501C0D49
:101A7800060EF324D96E010EF420DA6EDF50606F83
:101A880060C061F0626B636B646B63C064F062C0DA
:101A980063F061C062F0616B61C065F062C066F0BE
:101AA80063C067F064C068F0696B68BF696969C042
:101AB8006AF069C06BF069C06CF050501C0D050EDF
:101AC800F324D96E010EF420DA6EDF506D6F6DC00D
:101AD8006EF06F6B706B716B6FC071F06EC070F0F1
:101AE8006F6B6E6B6EC072F06FC073F070C074F085
:101AF80071C075F0766B75BF766976C077F076C081
:101B080078F076C079F050501C0D040EF324D96E8D
:101B1800010EF420DA6EDF507A6F7AC07BF07C6BAE
:101B28007D6B7E6B7BC07EF07D6B7C6B7B6B7BC043
:101B38007FF07CC080F07DC081F07EC082F0836B36
:101B480082BF836983C084F083C085F083C086F038
:101B580050501C0D030EF324D96E010EF420DA6EDA
:101B6800DF50876F87C088F0896B8A6B8B6B8C6BB3
:101B78008D6B8E6B8F6B200ED890883789378A379C
:101B88008B378C378D378E378F37E82EF5D77F51C7
:101B98008825906F80518921916F81518A21926F98
:101BA80082518B21936F83518C21946F84518D21A5
:101BB800956F85518E21966F86518F21976F72513F
:101BC8009025986F73519121996F745192219A6F52
:101BD800755193219B6F765194219C6F7751952174
:101BE8009D6F785196219E6F795197219F6F65510E
:101BF8009825A06F66519921A16F67519A21A26F0C
:101C080068519B21A36F69519C21A46F6A519D2142
:101C1800A56F6B519E21A66F6C519F21A76F5050E5
:101C28001C0D070EF324D96E010EF420DA6EA0C045
:101C3800DEFFA1C0DEFFA2C0DEFFA3C0DEFFA4C09E
:101C4800DEFFA5C0DEFFA6C0DEFFA7C0DEFF8390D3
:101C58000101826B836B00D150501C0D1A0EF324C6
:101C6800D96E010EF420DA6E0CC0DFFF070E0101F9
:101C7800836F0A0E76D050501C0D190EF324D96EBE
:101C8800010EF420DA6E0CC0DFFF070E0101836F2E
:101C98000B0E67D050501C0D180EF324D96E010E90
:101CA800F420DA6E0CC0DFFF070E0101836F0C0E03
:101CB80058D050501C0D170EF324D96E010EF42085
:101CC800DA6E0CC0DFFF38D00101826B836B4E6A7D
:101CD800A7D50CC08FF20F0E0101836F3E0E41D0C5
:101CE8000CC090F20F0E0101836F3F0E3AD00CC06A
:101CF80091F20F0E0101836F400E33D00CC092F2A7
:101D08000F0E0101836F410E2CD00CC093F20F0E01
:101D18000101836F420E25D00CC094F20F0E010111
:101D2800836F430E1ED00CC095F20F0E0101836F16
:101D3800440E17D00CC096F20101826B836B70D5EC
:101D48000C0E0101836F1E0E0CD00C0E0101836F67
:101D58001C0E826F0A0E0B6E63D50E0E0101836F87
:101D6800760E826F79D00101826B836B090E0B6E40
:101D7800838072D082C160F083C161F0000161513B
:101D880011E0030A13E0040A25E00B0A31E0010A16
:101D980035E0030A39E0010A40E0130A58E03B0A3B
:101DA80059E05AD0605101E132D556D06051E90A64
:101DB80001E107D6030A01E113D6010A01E11FD6A2
:101DC800070A01E12BD6010A01E137D6030A01E12E
:101DD80043D642D06051090A01E13ED7030A01E126
:101DE8004AD7010A01E156D7070A01E162D734D080
:101DF80060511D0AA5E0030AA8E02ED06051480AE8
:101E080001E126D7E40A28D06051750AA6E0030A42
:101E1800AAE0080A01E158D71FD060513D0A01E144
:101E280058D7030A01E15CD7010A01E160D77F0AAC
:101E380001E164D7010A01E168D7030A01E16CD71F
:101E4800010A01E170D7070A01E174D705D0605192
:101E58002A0A02D060510F0A0B5012000C6A0B6A52
:101E6800A8EC60F00101FC6F966B070E8C6E010EFA
:101E7800FD6F9C6B0F0E0F01596F116B196B216B66
:101E8800266B2E6B886889688A688A8E8890889203
:101E98008382020E0201B96FC4EC5FF088948384D8
:101EA800889C839C889E838E8B688968CE0E0001EF
:101EB8009C6FF90E9D6FAC0E9E6FFF0E9F6FE40E28
:101EC800A06FFE0EA16F2F0EA26FFF0EA36FCAECBC
:101ED80060F08A988588F4EC5EF0A80E00019C6F8B
:101EE800FB0E9D6FFCC19EF09F6BCAEC60F0010178
:101EF800FC2901E1FC6B0F0EFC175CEC4CF00101B6
:101F0800FC6FC00E00019C6FFB0E9D6FFCC19EF024
:101F18009F6BCAEC60F00400520E0101F06F2B0EAB
:101F2800EF6F000EE82EFED7EF2FFCD7F02FFAD771
:101F380000F0D250F00B0109D26ED09E0E01C6916E
:101F4800CF0ECF16CF82CF80C2890F01138113899C
:101F58001489F28E0E01BA89D4EC59F083928394D5
:101F68004DEC4FF04DEC4FF0000E0B6E340E8BEC39
:101F78005CF05C0E0F6EFF0E106E07EC58F0AC0EA6
:101F88000F6EFF0E106E07EC58F0000E0B6E390E38
:101F98008BEC5CF08FA22FD0290E0101F06F960E0A
:101FA800EF6F7F0EE82EFED7EF2FFCD7F02FFAD772
:101FB800000E0B6E800E8BEC5CF0630E0F6EFE0E47
:101FC800106E07EC58F017D0A50E00019C6FFE0E9E
:101FD8009D6F8FCF9EF09F6BCAEC60F0290E0101B8
:101FE800F06F960EEF6F7F0EE82EFED7EF2FFCD71F
:101FF800F02FFAD704008FB2E7D78380040031ECC2
:102008004AF00101F46FE6EC31F00101F46FFD5183
:102018000CE0900E00019C6FFD0E9D6FCAEC60F005
:10202800020E01019A6F220E0BD0800E00019C6FE8
:10203800FD0E9D6FCAEC60F0010E01019A6F040E4F
:10204800996F955102E0FCEC3FF0FEC193FFA1ECC3
:102058002EF07BEC51F0000E0B6E800E8BEC5CF0DA
:10206800D9EC5FF0000E0B6E800E8BEC5CF001017A
:10207800FC510F0D350EF3240F6E0D0EF420106E6B
:1020880007EC58F001019CBF6FEC45F00101F36BC0
:10209800F96B000EF76F010EF66FF7BF05D0F75119
:1020A80066E1040EF65D63E20F0EF603F3CFEFF17F
:1020B800F4CFF0F1F703F350F027250EEF250B6E60
:1020C8000E0EF0210C6E1BEC5DF00C5003E1030EBC
:1020D8000B5C49E3ED0E00019C6FFD0E9D6F0F0E2A
:1020E8000101F603F3CFEFF1F4CFF0F1F703F3506A
:1020F800F027250EEF2500019E6F0E0E0101F0213D
:1021080000019F6FCAEC60F0220E0101F603F3CFC5
:10211800EFF1F4CFF0F1F703F350F027000EEF25BD
:102128000001C96F030E0101F0210001CA6F0F0EF3
:102138000101F603F3CFF1F1F4CFF2F1F703F35015
:10214800F227250EF1250001CB6F0E0E0101F221B9
:102158000001CC6F030ECD6F1CEC15F00101F46F7C
:10216800F4513AEC5CF00101F64BF72B96D7970542
:1021780002E1070E8C6E020E971901E03FD10F01A4
:10218800108B070E2D6F3AD18EA8899462EC60F0FF
:102198000B500C1001E107D1F9C1F5F1F80E0B6EE7
:1021A800010E0C6EF9EC56F00101F96FF8B9F99FC0
:1021B8009C511BE0350EF91907E1FC0E00019C6FDC
:1021C800F90E9D6FCAEC60F04A0E00019C6FFF0E7D
:1021D8009D6FF9C19EF09F6B0101010EF8A9000ED9
:1021E8000001A06FA16BCAEC60F00101F8A949D009
:1021F800600EF91946E15F0EF51943E19F0E0001E3
:102208009C6FFC0E9D6FF9C19EF09F6BF5C1A0F00D
:10221800A16B010E8EA2000EA26FA36B010E8EA4FD
:10222800000EA46FA56BCAEC60F00201B983380EEA
:1022380000019C6FFF0E9D6F9AC19EF09F6BCAECC8
:1022480060F0410E9C6FFF0E9D6F99C19EF09F6BD1
:10225800CAEC60F02BEE35F09AC1DFFF2BEE36F0BA
:1022680099C1DFFF83841F6A020E1E6E45EC38F0A9
:1022780083940201B993536A81EC60F00101F96B10
:10228800BDD0FD5145E0F851100B0001C26F000EA2
:10229800C36F0101F95126EC37F0C2C0FAF1C3C08F
:1022A800FBF1080E0101FA19FB1101E100F0070E1C
:1022B8000101FA19FB1102E10BEC5BF0FA05FB11C5
:1022C80002E1FBEC52F0020E0101FA19FB1102E1E6
:1022D80072EC3AF0030E0101FA19FB1104E10FEC5C
:1022E8002BF00101F36F050EFA19FB1103E119EC4C
:1022F8003FF0F36F090EFA19FB1102E19FEC52F05F
:102308000A0E0101FA19FB1179E1F3EC60F076D0BD
:10231800F851100B1E6E000E1F6EF951ADEC1CF03B
:102328001EC0FAF11FC0FBF1070E0101FA19FB11DB
:1023380002E177EC5AF0020EFA19FB1102E12CECDB
:1023480059F0FA05FB1102E16CEC1AF0030EFA19C8
:10235800FB1102E1A2EC50F0040EFA19FB1102E1A4
:102368003DEC5FF0050EFA19FB1102E1D7EC4BF0DA
:10237800060E0101FA19FB1102E1FBEC60F0080EF0
:10238800FA19FB1102E134EC3EF0090EFA19FB11BF
:1023980002E1D8EC4EF00A0E0101FA19FB112EE108
:1023A800BDEC5DF02BD05CEC4CF00101966F9751C1
:1023B80025E0FC51961922E0838E000E0B6EC00EAC
:1023C8008BEC5CF0D9EC5FF0000E0B6EC00E8BEC62
:1023D8005CF0070E0F6EFF0E106E07EC58F096C1FA
:1023E800FCF1000E486E030E496EFAEC5DF0E6EC67
:1023F80031F00101955102E0FCEC3FF08FB22ED094
:10240800050E0101F3192AE0BFD6A50E00019C6F45
:10241800FE0E9D6F8FCF9EF09F6BCAEC60F0290E69
:102428000101F06F960EEF6F7F0EE82EFED7EF2FAB
:10243800FCD7F02FFAD70400000E0B6EC00E8BEC01
:102448005CF0D9EC5FF0000E0B6EC00E8BEC5CF00C
:10245800640E0F6EFF0E106E07EC58F08FB2D5D7D2
:10246800090E0101F06F1E0EEF6FE40EE82EFED785
:10247800EF2FFCD7F02FFAD700F083948392000156
:10248800B16BB26BFE0EB36FF90EB46FB56B23EC84
:1024980056F0B4D595C00CF096C00DF0B30E0E6E84
:1024A80057EC53F00001B56FB55108E120EE0FF07D
:1024B8009551D9269651DA22DF50B56FB55102E011
:1024C800B551120020EE0AF09551D9269651DA221C
:1024D8009751DE5C9851DE589951DE589A51DE5872
:1024E80016E220EE0EF09551D9269651DA22DFB287
:1024F8000ED020EE0AF09551D9269651DA22DECF79
:1025080097F0DECF98F0DECF99F0DECF9AF020EE8C
:1025180010F09551D9269651DA22DECFABF0DECFF6
:10252800ACF0DECFADF0DECFAEF0AF6BB06BB16B21
:10253800B26B20EE10F09551D9269651DA22AFC031
:10254800DEFFB0C0DEFFB1C0DEFFB2C0DEFF9751D4
:10255800981199119A1101E100D220EE09F0B351B6
:10256800D926B451DA22DECF9BF0DDCF9CF09B5107
:102578009D6F9C519E6F9F6BA06B090ED8909D37E5
:102588009E379F37A037E82EF9D79DC0B6F09EC07A
:10259800B7F09FC0B8F0A0C0B9F0AB51AC11AD1105
:1025A800AE1101E196D0FF0E97250B6EFF0E982114
:1025B8000C6EFF0E99210D6EFF0E9A210E6EB6C09D
:1025C8000FF0B7C010F0B8C011F0B9C012F044EC69
:1025D80058F00BC09BF00CC09CF00DC09DF00EC0D5
:1025E8009EF0FF0E0001AB250B6EFF0EAC210C6EAA
:1025F800FF0EAD210D6EFF0EAE210E6EB6C00FF0B0
:10260800B7C010F0B8C011F0B9C012F044EC58F0DF
:102618000B5000019B5D0C509C590D509D590E505C
:102628009E5957E3FF0EB6259B6FFF0EB7219C6F8F
:10263800FF0EB8219D6FFF0EB9219E6F9B1D9F6FE6
:102648009C1DA06F9D1DA16F9E1DA26FFF0EAB2547
:10265800A36FFF0EAC21A46FFF0EAD21A56FFF0E77
:10266800AE21A66F9F51A315A76FA051A415A86FFF
:10267800A151A515A96FA251A615AA6F20EE10F0B9
:102688009551D9269651DA22A7C0DEFFA8C0DEFFF1
:10269800A9C0DEFFAAC0DEFF20EE10F09551D926B2
:1026A8009651DA22DE50975FDE50985BDE50995BD8
:1026B800DD509A5B20EE14F09551D9269651DA2216
:1026C800DECFBAF0DECFBBF0DECFBCF0DECFBDF0A0
:1026D80060D020EE06F09551D9269651DA22DECF49
:1026E800BAF0DECFBBF0DECFBCF0DECFBDF0BA5122
:1026F800BB11BC11BD113FE195C078F096C079F0CF
:102708007A6B7B6B7C6B7D6B10EC23F078C0BAF036
:1027180079C0BBF07AC0BCF07BC0BDF0BA05BB1174
:10272800BC11BD1109E120EE0FF09551D926965143
:10273800DA22020EDF6E020CBA290FE1BB290DE185
:10274800BC290BE1BD2909E120EE0FF09551D926EE
:102758009651DA22010EDF6E010C20EE06F095513B
:10276800D9269651DA22BAC0DEFFBBC0DEFFBCC054
:10277800DEFFBDC0DEFF20EE14F09551D92696513C
:10278800DA22BAC0DEFFBBC0DEFFBCC0DEFFBDC0C0
:10279800DEFFBA51BB11BC11BD1101E085D0DDD0FF
:1027A800B651975FB751985BB851995BB9519A5B2D
:1027B80020EE10F09551D9269651DA22B651DE2630
:1027C800B751DE22B851DE22B951DE2220EE0EF0DA
:1027D8009551D9269651DA22DFA220D095C078F0FB
:1027E80096C079F0BAC07AF0BBC07BF0BCC07CF070
:1027F800BDC07DF010EC23F078C0BAF079C0BBF012
:102808007AC0BCF07BC0BDF0BA51BB11BC11BD1180
:102818001BE1976B986B996B9A6B50D095C042F0FF
:1028280096C043F0BAC044F0BBC045F0BCC046F007
:10283800BDC047F0E2EC2CF042C0BAF043C0BBF098
:1028480044C0BCF045C0BDF00001BA2907E1BB296E
:1028580005E1BC2903E1BD2901E176D7BD51BC11D1
:10286800BB1104E1020EBA5D01E25DD720EE13F060
:10287800B351D926B451DA22DE50BA5DDE50BB59C5
:10288800DE50BC59DE50BD5901E34DD720EE14F09F
:102898009551D9269651DA22BAC0DEFFBBC0DEFFB9
:1028A800BCC0DEFFBDC0DEFF9751B65D9851B75979
:1028B8009951B8599A51B95901E272D720EE10F0DE
:1028C8009551D9269651DA229751DE269851DE2263
:1028D8009951DE229A51DE2297519B6F010E98156D
:1028E8009C6F9D6B9E6B9B119D119E1136E0B3C032
:1028F8000BF0B4C00CF0BAC00DF0BBC00EF0BCC0F9
:102908000FF0BDC010F04DEC4BF00BC0AFF00CC099
:10291800B0F00DC0B1F00EC0B2F00001AF51B0116F
:10292800B111B21101E1FFD697C09BF098C09CF09D
:1029380099C09DF09AC09EF00A0E05D0D8909E339B
:102948009D339C339B33E82EF9D79B51AF279C517D
:10295800B0239D51B1239E51B22320EE10F0955122
:10296800D9269651DA2210EE0AF09551E1269651B1
:10297800E222DE50E65CDE50E658DE50E658DE50D5
:10298800E6581CE220EE10F09551D9269651DA222D
:1029980010EE0AF09551E1269651E222DECFE6FFCD
:1029A800DECFE6FFDECFE6FFDECFE6FF20EE0EF05D
:1029B8009551D9269651DA22000EDB8C20EE10F0C4
:1029C8009551D9269651DA22FF0EDE149B6F010E1F
:1029D800DE149C6F000EDE149D6F000EDE149E6FD9
:1029E8009B519C119D119E1101E16AD520EE18F0B2
:1029F8009551D9269651DA22AF51DE180AE1B05125
:102A0800DE1807E1B151DE1804E1B251DE1801E128
:102A180057D520EE18F09551D9269651DA22AFC035
:102A2800DEFFB0C0DEFFB1C0DEFFB2C0DEFF48D5BA
:102A3800C951CA1101E1090C3F0ECD17CB0E7C6FAD
:102A4800B50E7D6F010E7E6FCDC07FF0AFEC00F04C
:102A58000101B76FB75101E0A8D2B5C1B8F1B6C14D
:102A6800B9F1B80E0001BB6F010EBC6FCBC0BDF051
:102A7800CCC0BEF0BEEC41F00101B76FB75104E124
:102A8800DFAF02D0060EB76FCDC0CEF01C0E00012E
:102A9800CE1701E1D1D00101B7510FE0040EB719EB
:102AA80009E1B80E0001BF6F010EC06F41EC52F092
:102AB8000101B76F0001CD870DD0BCC1CEF0110E5A
:102AC8000001CE1702E0070E03D0CDA503D0080EF3
:102AD8000101B76F0101B75101E0BDD00001CDA7D9
:102AE800BAD0B5C112F0B6C113F0D2C114F0D3C137
:102AF80015F0B9EC58F012C0A5F113C0A6F114C036
:102B0800A7F115C0A8F10E0E0101D2250B6E000E1B
:102B1800D3210C6E0D6A0E6A210E0F6E500E106EC8
:102B280041EC5AF0010120EE0BF0D251D926D351D5
:102B3800DA22200EDF6EB5C10FF0B6C110F0D2C197
:102B480011F0D3C112F0136A146A156A166A9DEC63
:102B58005DF01C0E0101D2250B6E000ED3210C6E08
:102B68000D6A0E6A0F6A106A41EC5AF0010120EEF4
:102B780003F0B551D926B651DA22010EDF6EA55100
:102B8800A611A711A81167E020EE2BF0B551D926A0
:102B9800B651DA22DECFA9F1DECFAAF1DECFABF152
:102BA800DECFACF1B80E0001786F010E796FA5C1C8
:102BB8007AF0A6C17BF0A7C17CF0A8C17DF07E6B3E
:102BC8007F6B806B816B8BEC42F00101B76FB75163
:102BD80042E1B5C137F0B6C138F0A9C139F0AAC190
:102BE8003AF0ABC13BF0ACC13CF0F6EC54F001015B
:102BF800B76FFF0EA5250001CE6FFF0E0101A621BC
:102C08000001CF6FFF0E0101A7210001D06FFF0E59
:102C18000101A8210001D16F010120EE0BF0B5518F
:102C2800D926B651DA22CEC0DEFFCFC0DEFFD0C033
:102C3800DEFFD1C0DEFF0FD00101B7510CE1BCA906
:102C480002D0040E07D00001CDA305D00101BCA11C
:102C580002D0070EB76F0101B75123E10001CDB7CC
:102C6800CD8D010120EE2BF0B551D926B651DA22CF
:102C7800000110EE1CF0C951E126CA51E222DECF54
:102C8800E6FFDECFE6FFDECFE6FFDECFE6FF20EE93
:102C980020F0C951D926CA51DA22D2C1DEFFD3C1E8
:102CA800DDFF0101B75101E080D1B5C112F0B6C115
:102CB80013F0D2C114F0D3C115F0B9EC58F00001EB
:102CC80020EE06F0C951D926CA51DA2212C0DEFF19
:102CD80013C0DEFF14C0DEFF15C0DEFF1C0E0101AD
:102CE800D2250B6E000ED3210C6E01EC54F00001BE
:102CF80020EE0AF0C951D926CA51DA220BC0DEFFEC
:102D08000CC0DEFF0DC0DEFF0EC0DEFFC9C0D9FF5C
:102D1800CAC0DAFFB5C1DEFFB6C1DDFF010120EE92
:102D280005F0B551D926B651DA22000110EE02F0AD
:102D3800C951E126CA51E222DECFE6FFDDCFE5FF29
:102D480020EE0EF0C951D926CA51DA22CDC0DFFFD4
:102D580020EE0FF0C951D926CA51DA22DF6A20EED7
:102D680018F0C951D926CA51DA22DE6ADE6ADE6A4B
:102D7800DD6A20EE10F0C951D926CA51DA22DE6A7E
:102D8800DE6ADE6ADD6ACDAB10D120EE0AF0C951E9
:102D9800D926CA51DA22DE50DE10DE10DE1001E13B
:102DA80004D120EE0AF0C951D926CA51DA2210EE10
:102DB80010F0C951E126CA51E222DECFE6FFDECF8C
:102DC800E6FFDECFE6FFDECFE6FF010120EE09F0E9
:102DD800B551D926B651DA22DECFCEF0DDCFCFF00D
:102DE8000001CE51D06FCF51D16FD26BD36B090E8A
:102DF800D890D037D137D237D337E82EF9D7D0C0CB
:102E0800A1F1D1C0A2F1D2C0A3F1D3C0A4F120EEA8
:102E180006F0C951D926CA51DA22DECFB1F1DECF88
:102E2800B2F1DECFB3F1DECFB4F120EE0AF0C95132
:102E3800D926CA51DA22DECFADF1DECFAEF1DECF30
:102E4800AFF1DECFB0F132D0C9C042F0CAC043F012
:102E5800B1C144F0B2C145F0B3C146F0B4C147F0C6
:102E6800E2EC2CF042C0B1F143C0B2F144C0B3F17E
:102E780045C0B4F10101B451B311B21105E1020E1C
:102E8800B15D02E2020EB76FB12908E1B22906E18D
:102E9800B32904E1B42902E1010EB76FA151AD5F76
:102EA800A251AE5BA351AF5BA451B05B0101B75116
:102EB80009E1AD51A15DAE51A259AF51A359B0512D
:102EC800A459C2E3000120EE14F0C951D926CA5111
:102ED800DA22B1C1DEFFB2C1DEFFB3C1DEFFB4C189
:102EE800DEFF0101B75161E1AD510001CE6F010E66
:102EF8000101AE150001CF6FD06BD16BCE11D0118F
:102F0800D11153E0B5C10BF0B6C10CF0B1C10DF051
:102F1800B2C10EF0B3C10FF0B4C110F04DEC4BF0DC
:102F28000BC0A9F10CC0AAF10DC0ABF10EC0ACF1F9
:102F38000101A951AA11AB11AC1103E1020EB76F3F
:102F480034D0ADC1CEF0AEC1CFF0AFC1D0F0B0C17A
:102F5800D1F00A0E06D00001D890D133D033CF3348
:102F6800CE33E82EF8D70101A9510001CE25D26F42
:102F78000101AA510001CF21D36F0101AB5100011A
:102F8800D021D46F0101AC510001D121D56F20EEC1
:102F980018F0C951D926CA51DA22D2C0DEFFD3C0EF
:102FA800DEFFD4C0DEFFD5C0DEFF0101B75106E069
:102FB800C9C0D9FFCAC0DAFFDE6ADD6AB75112009C
:102FC80076C091F077C092F07AC0D9FF7BC0DAFF63
:102FD800DE6ADD6A74C00CF075C00DF09D0E0E6ED1
:102FE80057EC53F000018C6F8C510AE120EE0FF082
:102FF8007451D9267551DA22DF508C6F8C5102E05A
:103008008C51120020EE0EF07451D9267551DA2237
:10301800DFA0070C20EE10F07451D9267551DA2282
:10302800DECF7CF0DECF7DF0DECF7EF0DECF7FF02E
:1030380020EE0AF07451D9267551DA22DECF80F0DD
:10304800DECF81F0DECF82F0DECF83F07C51805D71
:10305800886F7D518159896F7E5182598A6F7F515E
:1030680083598B6F78517C6F79517D6F7E6B7F6B45
:103078007C51885D7D5189597E518A597F518B5980
:1030880001E321D288C078F089C079F01CD220EE03
:1030980010F07451D9267551DA22FF0EDE147C6FB8
:1030A800010EDE147D6F000EDE147E6F000EDE143E
:1030B8007F6F7C517D117E117F1101E083D120EE5D
:1030C80010F07451D9267551DA22DECF7CF0DECFAC
:1030D8007DF0DECF7EF0DECF7FF00A0E05D0D890EF
:1030E8007F337E337D337C33E82EF9D7806981695D
:1030F80020EE09F09D51D9269E51DA22DECF82F0CA
:10310800DDCF83F080518227815183237C51821542
:10311800936F7D518315946F931166E120EE10F043
:103128007451D9267551DA22DE50DE10DE10DE1019
:103138000FE120EE06F07451D9267551DA22DECF60
:103148008DF0DECF8EF0DECF8FF0DECF90F01CD08A
:1031580074C042F075C043F020EE14F07451D926C3
:103168007551DA22DECF44F0DECF45F0DECF46F0EF
:10317800DECF47F0E2EC2CF042C08DF043C08EF079
:1031880044C08FF045C090F0000190518F118E110E
:103198000CE1020E8D5D09E220EE0FF07451D92684
:1031A8007551DA22020EDF6E020C8D290FE18E298D
:1031B8000DE18F290BE1902909E120EE0FF0745100
:1031C800D9267551DA22010EDF6E010C20EE14F0BB
:1031D8007451D9267551DA228DC0DEFF8EC0DEFF0C
:1031E8008FC0DEFF90C0DEFF9DC00BF09EC00CF0CC
:1031F80020EE14F07451D9267551DA22DECF0DF085
:10320800DECF0EF0DECF0FF0DECF10F04DEC4BF03E
:103218000BC095F00CC096F00DC097F00EC098F05A
:103228000001955196119711981101E1B5D7935165
:10323800952794519623000E9723982378C07CF005
:1032480079C07DF0090E7E6FD8907D337C337E2F58
:10325800FBD77CC099F07DC09AF099519A1101E191
:10326800A3D0995193257C6F9A5194217D6F20EEBC
:1032780009F09D51D9269E51DA227C51DE5C7D51A0
:10328800DE5810E220EE09F09D51D9269E51DA222F
:10329800DECF7CF0DDCF7DF093517C5D996F94514A
:1032A8007D599A6F91C01AF092C01BF095C01CF01E
:1032B80096C01DF097C01EF098C01FF099C020F06E
:1032C8009AC021F020EE01F09D51D9269E51DA22B4
:1032D800DF5055EC54F0000901E0ACD0000120EEBD
:1032E80003F09D51D9269E51DA22DF504EE09951C4
:1032F8007C6F9A517D6F7E6B7F6B20EE2BF09D511A
:10330800D9269E51DA22DECF80F0DECF81F0DECFE3
:1033180082F0DECF83F09551805D846F965181599C
:10332800856F97518259866F98518359876F7C5161
:10333800845D7D5185597E5186597F51875925E293
:1033480020EE2BF09D51D9269E51DA22DECF7CF05B
:10335800DDCF7DF095517C5F96517D5B090ED8904D
:103368007C377D37E82EFBD77C5191250B6E7D513C
:1033780092210C6E2F0E9D250D6E000E9E210E6E55
:10338800020E106E0F6A3CEC5DF099C07CF09AC09A
:103398007DF0090ED8907C377D37E82EFBD77CC0AE
:1033A8009BF07DC09CF072D020EE18F07451D926A5
:1033B8007551DA2295C0DEFF96C0DEFF97C0DEFFAA
:1033C80098C0DEFF7C69010E7D6F20EE10F074510D
:1033D800D9267551DA22DECF7EF0DDCF7FF07C5121
:1033E8007E177D517F177E5100089B6F7F51D8A0B3
:1033F800E82A02089C6F9B51785D9C51795904E238
:1034080078C09BF079C09CF09DC037F09EC038F022
:1034180020EE18F07451D9267551DA22DECF39F032
:10342800DECF3AF0DECF3BF0DECF3CF0F6EC54F0E6
:10343800000902E00001C1D691C00BF092C00CF067
:1034480000017C69010E7D6F20EE10F07451D926C1
:103458007551DA22DECF7EF0DDCF7FF07C517E170A
:103468007D517F179DC080F09EC081F07E518027DE
:103478007F5181232F0E80250D6E000E81210E6E47
:103488009BC00FF09CC010F03CEC5DF09B51785F46
:103498009C51795B7AC0D9FF7BC0DAFF9B51DE264D
:1034A8009C51DD229B5191279C51922320EE10F0D4
:1034B8007451D9267551DA229B51DE269C51DE22A1
:1034C800000EDE22DE227851791101E0E0D5000CF1
:1034D80050500C0D5F0EF324D96E020EF420DA6EF4
:1034E8000001C469C56950500C0D670EF324E16EE4
:1034F800020EF420E26EE6CFC6F0E5CFC7F0C45165
:10350800C627C551C723DE50C65DC751800AC86F9C
:10351800DE50800AC8594AE350500C0D610EF3245E
:10352800D96E020EF420DA6EDF50C26FC36BC46925
:10353800C56950500C0D690EF324D96E020EF420A3
:10354800DA6EDF50C66FC76BC451C627C551C72393
:10355800C251C65DC751800AC86FC351800AC85995
:1035680025E350500C0D620EF324D96E020EF420A0
:10357800DA6EDF50C26FC36BC469C56950500C0D59
:103588006A0EF324D96E020EF420DA6EDF50C66F8D
:10359800C76BC451C627C551C723C251C65DC751A1
:1035A800800AC86FC351800AC85961E21F0E010121
:1035B8008D6F010E8F6F8390250E00019C6FFA0EA0
:1035C8009D6F50500C0D5F0EF324D96E020EF4203F
:1035D800DA6EDECF9EF0DDCF9FF050500C0D670EF7
:1035E800F324D96E020EF420DA6EDECFC2F0DDCFFE
:1035F800C3F0FF0EC225A06FFF0EC321A16F50506C
:103608000C0D610EF324D96E020EF420DA6EDF5031
:10361800A26FA36B50500C0D690EF324D96E020EE5
:10362800F420DA6EDF50C46FFF0EC425A46FA56BBB
:10363800FF0EA52350500C0D620EF324D96E020E16
:10364800F420DA6EDF50A66FA76B50500C0D6A0E8F
:10365800F324D96E020EF420DA6EDF50C56FFF0E28
:10366800C525A86FA96BFF0EA923CAEC60F05050BE
:103678000C0D620EF324D96E020EF420DA6EDF50C0
:10368800C26FC2C0C3F0C46BC56BC66BC5C0C6F001
:10369800C4C0C5F0C3C0C4F0C36B50500C0D6A0E53
:1036A800F324D96E020EF420DA6EDF50C76FC7C05C
:1036B800C8F0C96BCA6BCB6B50500C0D610EF3246C
:1036C800D96E020EF420DA6EDF50CC6FCCC0CDF08C
:1036D800CE6BCF6BD06BCFC0D0F0CEC0CFF0CDC00B
:1036E800CEF0CD6BCD51C803F3CFD1F0F4CFD2F0EB
:1036F800D36BD46BC903F350D227F450D323000EF5
:10370800D423CE51C803F350D227F450D323000E4C
:10371800D423CD51CA03F350D327F450D423CE5128
:10372800C903F350D327F450D423CF51C803F3501F
:10373800D327F450D423CB51CD03F350D427CE5103
:10374800CA03F350D427CF51C903F350D427D0511B
:10375800C803F350D42750500C0D690EF324D96ECA
:10376800020EF420DA6EDF50D56FD5C0D6F0D76BD5
:10377800D86BD96B50500C0D6A0EF324D96E020E1B
:10378800F420DA6EDF50DA6FDAC0DBF0DC6BDD6B69
:10379800DE6B50500C0D5F0EF324D96E020EF42030
:1037A800DA6EDECFDFF0DDCFE0F0DFC0E1F0E0C0C1
:1037B800E2F0000EE2BFFF0EE36FE46FE151DB03BE
:1037C800F3CFE5F0F4CFE6F0E76BE86BDC03F350FA
:1037D800E627F450E723000EE823E251DB03F35019
:1037E800E627F450E723000EE823E151DD03F35008
:1037F800E727F450E823E251DC03F350E727F450BD
:10380800E823E351DB03F350E727F450E823DE51C4
:10381800E103F350E827E251DD03F350E827E351D1
:10382800DC03F350E827E451DB03F350E827E7C053
:10383800E8F0E6C0E7F0E5C0E6F0E56BE551D60351
:10384800F3CFE9F0F4CFEAF0EB6BEC6BD703F3506E
:10385800EA27F450EB23000EEC23E651D603F3508D
:10386800EA27F450EB23000EEC23E551D803F3507C
:10387800EB27F450EC23E651D703F350EB27F45031
:10388800EC23E751D603F350EB27F450EC23D9513E
:10389800E503F350EC27E651D803F350EC27E75142
:1038A800D703F350EC27E851D603F350EC27D15156
:1038B800E925ED6FD251EA21EE6FD351EB21EF6F7D
:1038C800D451EC21F06FC351ED25F26FC451EE21B4
:1038D800F36FC551EF21F46FC651F021F56F5050C9
:1038E800220D000EF324956F030EF420966FF2C09C
:1038F80097F0F3C098F0F4C099F0F5C09AF04EEC48
:1039080012F0F16FF15111E0900E9C6FFB0E9D6F5C
:10391800F2C09EF0F3C09FF0F4C0A0F0F5C0A1F093
:10392800F1C0A2F0A36BCAEC60F050500C0D630E0E
:10393800F324D96E020EF420DA6EF2C0DEFFF3C073
:10394800DEFFF4C0DEFFF5C0DEFF01018F6B839060
:103958001200236E1F5002E07BEC51F0226A1E50C9
:1039680001E1C9D1239E040E231802E14D5003E161
:10397800140E231807E10101806B816B1F6A070E83
:103988001E6E070C3F0E231807E14D6A0101806B7C
:10399800816B1E6A1F6A12005F0E231807E101017E
:1039A800906B806B816B1E6A1F6A12003F0E236446
:1039B8000BD05F0E236008D0400E231805E00101EC
:1039C800906B1E6A1F6A1200400E23180AE1010E4E
:1039D8000101906F4D6A0101806B816B1E6A1F6A3D
:1039E8001200200E231801E086D1010E4D6EF3D788
:1039F800600E231809E10101905106E08E51080E6E
:103A0800D8B4030E226E7CD0600E231809E14D5005
:103A180007E001018E5102E0090E15D0050E13D002
:103A2800680E231809E14D5007E01A0E0101816F55
:103A3800900E54D18380BCD1680E231806E1010191
:103A4800905103E0020E226E5BD06A0E231807E144
:103A58004D5005E01A0E0101816FF40E3FD16C0E36
:103A6800231807E14D5005E01A0E0101816F2C0E55
:103A780035D1700E231810E1010190510DE0880E28
:103A880000019C6FFF0E9D6FCAEC60F0040E226E61
:103A98000101806B816BCED7700E231801E088D1AD
:103AA8004D5001E185D11B0E0101816F620E16D1C7
:103AB8008380020E231805E11A0E0101816F920E10
:103AC800806F050E231805E11A0E0101816FAE0EF5
:103AD800806F070E231805E11A0E0101816FB80ED9
:103AE800806F080E231805E11A0E0101816FCC0EB4
:103AF800806F030E231802E0232806E1226A8390D0
:103B08000101806B816B54D1140E231805E11A0E44
:103B18000101816F9E0E806F160E231801E048D1B7
:103B28001A0E0101816FA40ECAD0050E231805E1F3
:103B38001A0E0101816FF50E806F080E231801E03F
:103B480037D11A0E0101816FCC0E806F010E8E6F76
:103B58002FD123C050F01A0E0101816F950EAFD0FE
:103B68002350216E206A50500C0D5F0EF324D96E3D
:103B7800020EF420DA6E20C0DEFF21C0DDFF1A0E2F
:103B88000101816F960E9BD02350206E216A505000
:103B98000C0D5F0EF324D96E020EF420DA6E20C0ED
:103BA800DEFF21C0DDFF1A0E0101816F970E87D05D
:103BB80050500C0D610EF324D96E020EF420DA6E0B
:103BC80023C0DFFF1A0E0101816F980E78D0505084
:103BD8000C0D620EF324D96E020EF420DA6E23C0A7
:103BE800DFFF0101806B816B010E37D01A0E0101D6
:103BF800816FB90E73D01A0E0101816FBA0E5FD0B2
:103C08001A0E0101816FBB0E806F710E00019C6F4F
:103C1800FE0E9D6FCAEC60F001018F6B806B816BAB
:103C280055D00101806B816B710E00019C6FFE0EF7
:103C38009D6FCAEC60F04AD0120E00019C6FFF0E17
:103C48009D6FCAEC60F00101806B816B010E8C6F77
:103C58003DD00101806B816B060E226EA9D023C076
:103C680050F00101806B816B226A30D001018E6BAC
:103C78001A0E816FF70E806F29D01A0E0101816F1D
:103C8800F70E1DD08390270E0101816F0F0E17D0FC
:103C9800180E231801E08CD01A0E0101816F2D0E29
:103CA8000ED01A0E0101816F2E0E09D01A0E0101D5
:103CB800816F2F0E04D01A0E0101816F300E806FB4
:103CC80077D00101806B816B0A0E226E839070D0D1
:103CD800040E226E270E0101816F0F0E806FAAD687
:103CE8008380010104D08390010E01018E6F806BE7
:103CF800816B226A5DD080C120F081C121F0215002
:103D080007E01A0A09E0010A4BE03C0A4FE050D0EC
:103D1800205001E16DD64CD020502C0AB9E0010AA0
:103D2800C0E0030AC3E0010AC6E01F0ACAE0A00A0D
:103D380001E1BED6020A01E10CD7070A01E110D75A
:103D4800030A01E121D7010A01E132D70F0A01E193
:103D58003ED7060A01E170D73A0A01E17AD70A0A82
:103D6800C2E0160A01E142D7010A01E144D7030A79
:103D780001E146D7010A01E154D7790A01E162D687
:103D88000E0A01E16CD7380A01E1CFD6010A01E138
:103D98006DD7030A01E171D7010A01E173D708D091
:103DA8002050580A95E03A0A9BE002D020500F0AAA
:103DB80022C01EF01F6A1200020E4A6E655164117D
:103DC800631104E1020E625D01E211D220EE13F0EC
:103DD8006051D9266151DA22DE50625DDE506359A6
:103DE800DE506459DE50655901E2EED100D262C05E
:103DF80048F063C049F0D89049306B6F48306A6F1B
:103E08006A5148266B51492260C037F061C038F0CA
:103E180020EE1FF06051D9266151DA22DECF6AF018
:103E2800DECF6BF0DECF6CF0DECF6DF048C06EF009
:103E380049C06FF0090E706FD8906F336E33702FD2
:103E4800FBD76E516A25396E6F516B213A6E000EA1
:103E58006C213B6E000E6D213C6EF6EC54F04A6E00
:103E68004A5001E0C4D100016A69010E6B6F48C075
:103E78006CF049C06DF06A516C176B516D1760C0DA
:103E88006EF061C06FF06C516E276D516F232F0E6D
:103E98006E25466E000E6F21476E484A492A62B168
:103EA80004D066C042F0436A1AD066516A6F6B6BE1
:103EB8006A3B6B3BF00E6B176A510F0B6B13F00EDE
:103EC8006A1746C0D9FF47C0DAFFDF500F0B6C6F87
:103ED8006D6B6A516C11426E6B516D11436E46C029
:103EE800D9FF47C0DAFF42C0DFFF20EE03F0605180
:103EF800D9266151DA22010EDF6E60C037F061C049
:103F080038F020EE1FF06051D9266151DA22DECF59
:103F18006AF0DECF6BF0DECF6CF0DECF6DF048C01C
:103F28006EF049C06FF0090E706FD8906F336E3322
:103F3800702FFBD76E516A25396E6F516B213A6E1F
:103F4800000E6C213B6E000E6D213C6EF6EC54F0B9
:103F58004A6E4A5001E04BD100016A69010E6B6F4D
:103F680048C06CF049C06DF06A516C176B516D1701
:103F780060C06EF061C06FF06C516E276D516F2399
:103F88002F0E6E25466E000E6F21476E62B10CD063
:103F980067C06AF00F0E6A1746C0D9FF47C0DAFF3C
:103FA800DF50F00B6A1112D066C06AF067C06BF080
:103FB80068C06CF069C06DF0050E05D0D8906D33FF
:103FC8006C336B336A33E82EF9D76A51446E456A0D
:103FD80046C0D9FF47C0DAFF44C0DFFF4FD060C0FA
:103FE80037F061C038F020EE1FF06051D9266151DA
:103FF800DA22DECF6AF0DECF6BF0DECF6CF0DECFF8
:104008006DF063516E6F64516F6F6551706F716BB6
:104018006A516E25396E6B516F213A6E6C51702161
:104028003B6E6D5171213C6EF6EC54F04A6E4A506D
:1040380001E0DDD000016A69010E6B6F62C06CF0AF
:1040480063C06DF0D8906C376D376A516C176B513F
:104058006D1760C06EF061C06FF06C516E276D51C6
:104068006F232F0E6E250B6E000E6F210C6E66C02F
:104078000DF067C00EF002EC60F0A4D020EE03F063
:104088006051D9266151DA22010EDF6EB0D060C0CE
:1040980037F061C038F020EE1FF06051D926615129
:1040A800DA22DECF6AF0DECF6BF0DECF6CF0DECF47
:1040B8006DF062C06EF063C06FF064C070F065C0F0
:1040C80071F0080E05D0D890713370336F336E33AA
:1040D800E82EF9D76A516E25396E6B516F213A6E09
:1040E8006C5170213B6E6D5171213C6EF6EC54F0B1
:1040F8004A6E4A507CE100016A69010E6B6F62C02A
:104108006CF063C06DF0D8906C376D37D8906C3711
:104118006D376A516C176B516D1760C06EF061C0D6
:104128006FF06C516E276D516F232F0E6E250B6E3D
:10413800000E6F210C6E01EC54F00001706B716B76
:10414800726BF00E0E14736F6651746F6751756F52
:104158006851766F0F0E6915776F70517411666F1D
:1041680071517511676F72517611686F73517711BC
:10417800696F6A69010E6B6F62C06CF063C06DF0A5
:10418800D8906C376D37D8906C376D376A516C178B
:104198006B516D1760C06EF061C06FF06C516E2787
:1041A8006D516F232F0E6E250B6E000E6F210C6E56
:1041B80066C00DF067C00EF068C00FF069C010F05F
:1041C80041EC5AF000015AD760C0D9FF61C0DAFF4C
:1041D800DF506A6F6B6B6B510AE16A51010A01E1AA
:1041E80006D6030A01E1FBD6010A01E150D74A507D
:1041F80012002A6E1BC041F01CC042F02A5001E098
:10420800040C010E3F6E54B0030CE9D19CEC60F035
:10421800000901E1FDD13F6AFBD1146A156A166AEB
:10422800176A090E6DEC5EF0000901E0F1D12B0E62
:104238000B6E0C6A0E6A100E0D6E3AEC5BF00009FC
:1042480001E1E6D12B44E846030BE8064DE132C014
:104258001DF03F0E1D161DC01EF01F6A206A216A40
:104268001FC021F01EC020F01F6A1E6A3350236E43
:10427800226A3450246E256A22502426235025228F
:1042880024501E24266E25501F20276E000E202045
:10429800286E000E2120296E26283B6E000E27204E
:1042A8003C6E000E28203D6E000E29203E6E3BC05D
:1042B8001DF03CC01EF03DC01FF03EC020F00A0EAD
:1042C800D8901D361E361F362036E82EF9D71BC06B
:1042D800D9FF1CC0DAFF1DC0DEFF1EC0DEFF1FC0F5
:1042E800DEFF20C0DEFF97D71D6A35AE01D01D2A3C
:1042F800010E1D1630C01EF00F0E1E163450030B93
:10430800020DF3501E241D24020F406E3150030B82
:104318001D6E1E6A0A0ED8901D361E36E82EFBD773
:1043280032501F6E206AD8901F362036D8901F361C
:1043380020363344E846030B216E226A1F5021269B
:10434800205022221D5021261E502222212A000EF2
:10435800222221C03BF022C03CF03D6A3E6A40C0A8
:104368001DF0F70E1D263BC01EF03CC01FF03DC0DF
:1043780020F03EC021F01D2A05D0D8901E361F36E9
:10438800203621361D2EF9D734D051A43FD0146AD7
:10439800156A166A176A8D0E6DEC5EF0000901E069
:1043A80037D1E6EC60F02B0E0B6E0C6A0E6A100E1D
:1043B8000D6E3AEC5BF0000901E12AD1300E406E37
:1043C80003D0E6EC60F040064050FBE135C01DF03C
:1043D8001D3A0F0E1D16100E1E6E1F6A206A216AE6
:1043E8001D2A05D0D8901E361F36203621361D2EA0
:1043F800F9D71BC0D9FF1CC0DAFF1EC0DEFF1FC0E3
:10440800DEFF20C0DEFF21C0DEFF05D7146A156A73
:10441800166A176A090E6DEC5EF0000901E0F8D023
:104428002B0E0B6E0C6A0E6A100E0D6E3AEC5BF0DA
:10443800000901E1EDD051A232D038C01DF0060EBE
:104448001E6ED8901D321E2EFCD7FF0E1D2635502D
:104458003F0B1F6E206AD8901F3620363644010B5A
:104468001F26000E20221F2A20221D2A03D0D890A2
:104478001F3620361D2EFBD71F50216E2050226E6E
:10448800236A246A1BC0D9FF1CC0DAFF21C0DEFFE3
:1044980022C0DEFF23C0DEFF24C0DEFFBCD63650BC
:1044A800030B1D6E1E6AD8901D361E36D8901D3619
:1044B8001E36D8901D361E363638E842070B1D26A4
:1044C800000E1E221D2A1E223540E8423F0B1F0BFC
:1044D8001F6E206A1F2A000E20221D501F02F3CFD4
:1044E80021F0F4CF22F02002F35022261E501F02A2
:1044F800F35022262150236E2250246E256A266A04
:104508001BC0D9FF1CC0DAFF23C0DEFF24C0DEFFBA
:1045180025C0DEFF26C0DEFF7ED641C0D9FF42C0DF
:10452800DAFF51C0DFFF77D6146A156A166A176A70
:10453800090E6DEC5EF000096BE141C00BF042C062
:104548000CF00E6A100E0D6E3AEC5BF0000901E0FB
:1045580062D65ED0146A156A166A176A0A0E6DEC7E
:104568005EF0000955E141C00BF042C00CF00E6A44
:10457800100E0D6E3AEC5BF0E9D7146A156A166AEC
:10458800176A3A0E6DEC5EF0000942E1040E406EC7
:104598000AD0E6EC60F041C0D9FF42C0DAFFDF6E16
:1045A800414A422A4006405001E135D6F2D7146A02
:1045B800156A166A176A8D0E6DEC5EF0000928E11F
:1045C800E6EC60F041C00BF042C00CF00E6A400E01
:1045D8000D6E3AEC5BF0BAD7040E3F6E19D01A5044
:1045E8001D6E1E6A1E50F8E11D5001E10FD6010A2A
:1045F80001E113D6020A01E1C8D6090A8EE0010AD0
:1046080093E0070AA7E0010AB8E0030AD0E0E4D77C
:10461800F7EC60F03F50120078C0D9FF79C0DAFF9C
:10462800DECF8FF0DDCF90F07A517B117C117D11B8
:1046380028E120EE0BF08F51D9269051DA22DECFF7
:1046480087F0DECF88F0DECF89F0DECF8AF08751A1
:10465800881189118A110FE020EE13F08F51D926A5
:104668009051DA22DE50875DDE508859DE50895934
:10467800DE508A5952E3010E876F886B896B8A6B0B
:104688004CD078C042F079C043F07AC044F07BC087
:1046980045F07CC046F07DC047F0E2EC2CF042C00B
:1046A80091F043C092F044C093F045C094F00001EB
:1046B80094519311921109E1020E915D06E2010EE7
:1046C800786F796B7A6B7B6B000C91290FE19229DB
:1046D8000DE193290BE1942909E191C078F092C08A
:1046E80079F093C07AF094C07BF0120020EE13F0BA
:1046F8008F51D9269051DA22DE50915DDE509259C1
:10470800DE509359DE509459E8E37AC087F07BC0B5
:1047180088F07CC089F07DC08AF020EE0FF08F51C0
:10472800D9269051DA22DE50DE10DE10DE1005E1C7
:10473800786B796B7A6B7B6B12008B6B8C6B8D6BE8
:104748008E6B7A51871909E17B51881906E17C51F2
:1047580089197DE17D518A19D8A479D087298B6F71
:10476800000E88218C6F000E89218D6F000E8A2122
:104778008E6F20EE13F08F51D9269051DA22DE5039
:104788008B5DDE508C59DE508D59DE508E5905E315
:10479800020E8B6F8C6B8D6B8E6B78C042F079C07C
:1047A80043F08BC044F08CC045F08DC046F08EC0FD
:1047B80047F0E2EC2CF042C091F043C092F044C0C4
:1047C80093F045C094F00001910592119311941152
:1047D80084E0912907E1922905E1932903E19429CD
:1047E80001E17BD7915192119311941130E020EEA1
:1047F8000BF08F51D9269051DA22DECF91F0DECF1F
:1048080092F0DECF93F0DECF94F094519311921191
:1048180003E1020E915D17E320EE13F08F51D926C4
:104828009051DA22DE50915DDE509259DE50935954
:10483800DE50945908E291C087F092C088F093C086
:1048480089F094C08AF08B6B8C6B8D6B8E6B8B515F
:104858008C118D118E1162E187C08BF088C08CF0AD
:1048680089C08DF08AC08EF08B2B000E8C238D238F
:104878008E2320EE13F08F51D9269051DA22DE5084
:104888008B5DDE508C59DE508D59DE508E590DE30C
:10489800020E8B6F8C6B8D6B8E6B8A518911881110
:1048A80004E1020E875D01E243D778C042F079C087
:1048B80043F08BC044F08CC045F08DC046F08EC0EC
:1048C80047F0E2EC2CF042C091F043C092F044C0B3
:1048D80093F045C094F000019151921193119411F5
:1048E8001DE0910592119311941101E1F6D69129D9
:1048F80007E1922905E1932903E1942901E1EDD625
:1049080087518B19B1E188518C19AEE189518D1904
:10491800ABE18A518E1901E10BD7A6D78FC060F0A1
:1049280090C061F08BC062F08CC063F08DC064F001
:104938008EC065F06669676968696969E0EC1EF0B0
:104948000001866F86511DE17A517B117C117D1122
:1049580018E08FC060F090C061F07AC062F07BC050
:1049680063F07CC064F07DC065F08BC066F08CC0DD
:1049780067F08DC068F08EC069F0E0EC1EF00001B1
:10498800866F865143E120EE0BF08F51D926905166
:10499800DA228BC0DEFF8CC0DEFF8DC0DEFF8EC04A
:1049A800DEFF20EE0FF08F51D9269051DA2210EE5B
:1049B80013F08F51E1269051E222FE0EE624826F19
:1049C800FF0EE620836FFF0EE620846FFF0EE620C1
:1049D800856FDE50825DDE508359DE508459DE508B
:1049E80085590BE320EE0FF08F51D9269051DA222A
:1049F800DE06000EDE5ADE5ADE5A20EE04F08F5133
:104A0800D9269051DA22000EDB800DD0860507E00A
:104A1800010E8B6F000E8C6B8D6B8E6B04D08B69C7
:104A28008C698D698E698BC078F08CC079F08DC0E7
:104A38007AF08EC07BF0120018C0F6FF19C0F7FF9D
:104A48000800F5CF9BF0184A192A00019B5101E193
:104A58001200250E9B1904E09B51BFEC60F0ECD7C7
:104A6800946B956B966B976B18C0F6FF19C0F7FFA0
:104A78000800F5CF9BF0184A192A300E9B190DE152
:104A8800976B010E966F18C0F6FF19C0F7FF080064
:104A9800F5CF9BF0184A192A06D02D0E9B1903E171
:104AA800976B020EEFD72A0E9B1943E11A50D96E65
:104AB800DA6A020EDF26DF5CD96EDA6ADECF8CF0A6
:104AC800DECF8DF08DAF0BD08C5100088C6F8D51DF
:104AD800D8A0E82A00088D6F976B020E966F8CC0DD
:104AE80094F08DC095F018C0F6FF19C0F7FF0800C4
:104AF800F5CF9BF0184A192A22D00A0E9403F3CF57
:104B08001BF0F4CF1CF09503F3501C269B511B2679
:104B1800000E1C22D00E1B24946FFF0E1C20956FD4
:104B280018C0F6FF19C0F7FF0800F5CF9BF0184A28
:104B3800192A2F0E9B6503D0390E9B65DED76C0EA4
:104B48009B1903E04C0E9B190AE1968518C0F6FFE5
:104B580019C0F7FF0800F5CF9BF0184A192A9B5196
:104B680001E112009BC09AF0600E9A6575D0200E84
:104B78009A5F72D01A50D96EDA6A020EDF26DF5CAD
:104B8800D96EDA6ADECF84F0DECF85F0926B936B54
:104B980003D00001924B932B925184251B6E9351A5
:104BA80085211C6E1BC0F6FF1CC0F7FF000EF86EB7
:104BB8000E0EF76403D00800F55005D0F6CFE9FFD4
:104BC800F7CFEAFFEF50000904E0E3D7200EBFEC6F
:104BD80060F0000196B30BD092511B6E93511C6E7E
:104BE800924B932B94511B5C95511C58EFE384C056
:104BF8000CF085C00DF0BEEC5BF003D0200EBFECCE
:104C080060F0000192511B6E93511C6E924B932BD6
:104C180094511B5C95511C5801E30ED7EFD71A50DD
:104C2800D96EDA6ADF50DF2ADF2AD96EDA6ADF50F6
:104C3800BFEC60F001D7876B020E08D0876B080EB7
:104C480005D0876B0A0E02D0876B100E866F1AD0BC
:104C58009B51BFEC60F0F0D69A511B6E1C6A1C5039
:104C6800F7E11B50420AE7E0010AD9E0070AE9E048
:104C78000B0AE4E01C0A01E17DD7060AE2E00D0A0E
:104C8800E3E0E6D796A511D01A50D96EDA6A040E79
:104C9800DF26DF5CD96EDA6ADECF8EF0DECF8FF0EA
:104CA800DECF90F0DECF91F027D0440E9A1913E0B2
:104CB8001A50D96EDA6ADF50DF2ADF2AD96EDA6A2B
:104CC800DECF1BF0DDCF1CF01BC08EF01CC08FF0B8
:104CD800906B916B11D01A50D96EDA6ADF50DF2AC7
:104CE800DF2AD96EDA6ADECF8EF0DDCF8FF0000EC4
:104CF8008FBFFF0E906F916F440E9A190CE191AF20
:104D08000AD08E6D8F1FD8B08F2B901FD8B0902BE4
:104D1800000E91579689986B996B8EC088F08FC05A
:104D280089F090C08AF091C08BF088C00BF089C0E0
:104D38000CF08AC00DF08BC00EF086C00FF087C053
:104D480010F0116A126AAAEC5AF00B5000019A6F1F
:104D580088C00BF089C00CF08AC00DF08BC00EF033
:104D680086C00FF087C010F0116A126A44EC58F040
:104D78000BC088F00CC089F00DC08AF00EC08BF013
:104D8800090E00019A650BD0780E9B1903E0816B20
:104D9800070E02D0816B270E806F80519A27985199
:104DA800600FD96EDA6A9A51300FDF6E984B992BE3
:104DB800885189118A118B1105E0995103E1200E60
:104DC800985DB3E396A908D09851600FD96EDA6A56
:104DD8002D0EDF6E984B992B98C092F099C093F0E6
:104DE80096B103D0836B200E02D0836B300E826F96
:104DF80082C09AF003D09A51BFEC60F0000196B3DC
:104E08000BD092511B6E93511C6E924B932B945165
:104E18001B5C95511C58EFE39807D8A09907985147
:104E2800600FD96EDA6ADF50BFEC60F0000198516C
:104E3800991104E0F1D7200EBFEC60F00001925107
:104E48001B6E93511C6E924B932B94511B5C955186
:104E58001C5801E3F1D5EFD750500C0D620EF32426
:104E6800D96E020EF420DA6EDF2A50500C0D620E55
:104E7800F324D96E020EF420DA6EDF500001C26FFF
:104E8800C36BC469C56950500C0D6A0EF324D96E02
:104E9800020EF420DA6EDF50C66FC76BC451C62706
:104EA800C551C723C251C65DC751800AC86FC351D7
:104EB800800AC8594BE250500C0D620EF324D96E8B
:104EC800020EF420DA6EDF6A50500C0D610EF324E6
:104ED800D96E020EF420DA6EDF2A50500C0D610EE6
:104EE800F324D96E020EF420DA6EDF50C26FC36B62
:104EF800C469C56950500C0D690EF324D96E020EB1
:104F0800F420DA6EDF50C66FC76BC451C627C5518F
:104F1800C723C251C65DC751800AC86FC351800AF2
:104F2800C85914E250500C0D610EF324D96E020ECC
:104F3800F420DA6EDF6A50500C0D5F0EF324D96E40
:104F4800020EF420DA6EDE2A000EDD2250500C0D1F
:104F5800620EF324D96E020EF420DA6EDF50C26FAF
:104F6800C2C0C3F0C46BC56BC66BC5C0C6F0C4C0B5
:104F7800C5F0C3C0C4F0C36B50500C0D6A0EF324C7
:104F8800D96E020EF420DA6EDF50C76FC7C0C8F0C2
:104F9800C96BCA6BCB6B50500C0D610EF324D96EE4
:104FA800020EF420DA6EDF50CC6FCCC0CDF0CE6BA1
:104FB800CF6BD06BCFC0D0F0CEC0CFF0CDC0CEF08D
:104FC800CD6BCD51C803F3CFD1F0F4CFD2F0D36B72
:104FD800D46BC903F350D227F450D323000ED42343
:104FE800CE51C803F350D227F450D323000ED42354
:104FF800CD51CA03F350D327F450D423CE51C9035B
:10500800F350D327F450D423CF51C803F350D327F8
:10501800F450D423CB51CD03F350D427CE51CA0337
:10502800F350D427CF51C903F350D427D051C80324
:10503800F350D42750500C0D690EF324D96E020E8C
:10504800F420DA6EDF50D56FD5C0D6F0D76BD86BA9
:10505800D96B50500C0D6A0EF324D96E020EF42051
:10506800DA6EDF50DA6FDAC0DBF0DC6BDD6BDE6B3B
:1050780050500C0D5F0EF324D96E020EF420DA6E38
:10508800DECFDFF0DDCFE0F0DFC0E1F0E0C0E2F03E
:10509800000EE2BFFF0EE36FE46FE151DB03F3CFD5
:1050A800E5F0F4CFE6F0E76BE86BDC03F350E627B6
:1050B800F450E723000EE823E251DB03F350E62720
:1050C800F450E723000EE823E151DD03F350E7270E
:1050D800F450E823E251DC03F350E727F450E823C7
:1050E800E351DB03F350E727F450E823DE51E103F3
:1050F800F350E827E251DD03F350E827E351DC03DE
:10510800F350E827E451DB03F350E827E7C0E8F061
:10511800E6C0E7F0E5C0E6F0E56BE551D603F3CF6E
:10512800E9F0F4CFEAF0EB6BEC6BD703F350EA2726
:10513800F450EB23000EEC23E651D603F350EA2794
:10514800F450EB23000EEC23E551D803F350EB2782
:10515800F450EC23E651D703F350EB27F450EC233B
:10516800E751D603F350EB27F450EC23D951E5036C
:10517800F350EC27E651D803F350EC27E751D70357
:10518800F350EC27E851D603F350EC27D151E92529
:10519800ED6FD251EA21EE6FD351EB21EF6FD4516D
:1051A800EC21F06FC351ED25F16FC451EE21F26F80
:1051B800C551EF21F36FC651F021F46F50500C0D1B
:1051C800630EF324D96E020EF420DA6EF1C0DEFF0E
:1051D800F2C0DEFFF3C0DEFFF4C0DEFF5050220D48
:1051E800000EF324956F030EF420966F50500C0DAB
:1051F800630EF324D96E020EF420DA6EDECF97F038
:10520800DECF98F0DECF99F0DECF9AF04EEC12F0B8
:10521800F56FF55119E0900E9C6FFB0E9D6F505085
:105228000C0D630EF324D96E020EF420DA6EDECF75
:105238009EF0DECF9FF0DECFA0F0DECFA1F0F5C06C
:10524800A2F0A36BCAEC60F001018F6B1200000E94
:105258000001746F030E756F350E766F0B0E776F46
:10526800020E796F786BF30E7A6F7B6BE4EC17F0B4
:1052780001019B6FB00E00019C6FFD0E9D6FF3C086
:105288009EF0F4C09FF0CAEC60F0F56BF66BF16B22
:10529800F26BF76BF86BF751D30FD96EDA6ADF6AE6
:1052A800F751E20FD96EDA6A000EDF6EF74BF82B72
:1052B800F8BFF1D7F85103E10F0EF75DECE3F96B96
:1052C800FA6B30D1350EF925D96E0B0EFA21DA6E4C
:1052D8000D0EDE1801E0EBD09A0E0B6EFF0E0C6E71
:1052E800D30E0D6E44EC55F00B500C1007E1E20E96
:1052F800126E61EC4DF012500101FD6F940E0B6EB1
:10530800FF0E0C6ED30E0D6E44EC55F00B500C10C6
:1053180007E1E20E126E61EC4DF0125001019C6F34
:10532800730E0B6EFF0E0C6ED30E0D6E44EC55F023
:105338000B500C1007E1E20E126E61EC4DF01250AA
:105348000101976FD80E0B6EFF0E0C6ED30E0D6E0B
:1053580044EC55F00B500C1007E1E20E126E61ECB4
:105368004DF012500101956FDC0E0B6EFF0E0C6EA6
:10537800D30E0D6E44EC55F00B500C1007E1E20E05
:10538800126E61EC4DF012500101FE6F0001FB6BD3
:10539800FC6BC40E796F7A6B7A0E7B6FFF0E7C6F95
:1053A800FBC07DF0FCC07EF017EC5EF0C40E0B6E07
:1053B8000C6AD30E0D6E44EC55F00B500C1018E12E
:1053C8000F0E0001FB03F3CFC2F0F4CFC3F0FC03D0
:1053D800F350C327350EC2250B6E0D0EC3210C6E7C
:1053E800E20E0D6E0E6A106A0F0E0F6E69EC5BF01E
:1053F8000001FB4BFC2BFCBFCCD7FC5103E1100E8A
:10540800FB5DC7E3FC6B010EFB6FC40E796F7A6B13
:10541800810E7B6FFF0E7C6FFBC07DF0FCC07EF0C1
:1054280017EC5EF0C40E0B6E0C6AD30E0D6E44ECD6
:1054380055F00B500C1018E10F0E0001FB03F3CFD1
:10544800C2F0F4CFC3F0FC03F350C327250EC225E6
:105458000B6E0E0EC3210C6EE20E0D6E0E6A106AF4
:105468000F0E0F6E69EC5BF00001FB4BFC2BFCBFD1
:10547800CCD7FC5103E1040EFB5DC7E3F76BF86B77
:10548800F751D30FD96EDA6ADF6AF751E20FD96E96
:10549800DA6A000EDF6EF74BF82BF8BFF1D7F85138
:1054A80003E10F0EF75DECE3F16BF26B15D0350EEF
:1054B800F925D96E0B0EFA21DA6E0A0EDE1830E0E5
:1054C800350EF925D96E0B0EFA21DA6E200EDE188C
:1054D80006E1F26B010EF16FF56BF66B21D0F1511D
:1054E800F21109E0350EF925D96E0B0EFA21DA6EA4
:1054F800F551E20F08D0350EF925D96E0B0EFA21B9
:10550800DA6EF551D30FE16EE26ADFCFE7FFF6BF3F
:1055180005D0F65105E10F0EF55D02E2F54BF62BCD
:10552800F94BFA2BF351F95DF451FA5901E2CAD655
:10553800A00E9C6FFD0E9D6F97C19EF09F6BCAECED
:1055480060F01A0E9C6FFE0E9D6FFDC19EF09F6B62
:10555800CAEC60F0FC0E9C6FFD0E9D6F9CC19EF026
:105568009F6BCAEC60F00B0E9C6FFE0E9D6FFEC128
:105578009EF09F6BCAEC60F0FB6BFC6B1D0E9C6F82
:10558800FD0E9D6FFBC09EF0FCC09FF00F0EFB034D
:10559800F3CFC2F0F4CFC3F0FC03F350C327350EAA
:1055A800C225A06F0D0EC321A16FCAEC60F0FB4BA2
:1055B800FC2BFCBFE3D7FC5103E1100EFB5DDEE3DF
:1055C800FA6B010EF96F2E0E9C6FFD0E9D6FF9C0E0
:1055D8009EF0FAC09FF00F0EF903F3CFC2F0F4CF9C
:1055E800C3F0FA03F350C327250EC225A06F0E0E91
:1055F800C321A16FCAEC60F0F94BFA2BFABFE3D7CD
:10560800FA5103E1040EF95DDEE3FC0E9C6FF90E1E
:105618009D6FCAEF60F0838E83806DEC3BF00101D3
:10562800AB6FAB5118E050501C0D1B0EF324D96E14
:10563800010EF420DA6E50501C0D1B0EF324E16E9F
:10564800010EF420E26EE7500409DF6E54EC5FF0BF
:105658000101AB511200955154E070517111721152
:1056680073114FE050504DE150501C0D070EF324BC
:10567800D96E010EF420DA6E70C1F0F071C1F1F04C
:1056880072C1F2F00001EF6B000EEF25F36F010E0F
:10569800F021F46F000EF121F56F000EF221F66F84
:1056A800F76BF86BF96BFA6BDE50F3192AE1DE50F1
:1056B800F41927E1DE50F51924E1DE50F61921E14D
:1056C800DE50F7191EE1DE50F8191BE1DE50F9191A
:1056D80018E1DE50FA1915E1350E286E0B0E296E09
:1056E800010195515FEC4EF00201B993010E1F6E56
:1056F8001E6A45EC38F00201B9934E6A83904E5009
:10570800120050501C0D170EF324D96E010EF42010
:10571800DA6EDECFE7F0DECFE8F0DECFE9F0DECFFD
:10572800EAF0E8C0E7F0E9C0E8F0EAC0E9F0000113
:10573800EA6BE7C09FF1E8C0A0F1E9C0A1F1EAC0B7
:10574800A2F150501C0D170EF324D96E010EF4204F
:10575800DA6EDECFE7F0DDCFE8F0E7510101A56FA3
:10576800A66B0201B9930101A76BA86BA96BAA6B81
:10577800A36BA46B98D0A3C1E7F0A4C1E8F0000E16
:10578800E8BFFF0EE96FEA6FFF0E01019F250001D8
:10579800EB6FFF0E0101A0210001EC6FFF0E01016C
:1057A800A1210001ED6FFF0E0101A2210001EE6FA2
:1057B800E751EB190FE1E851EC190CE1E951ED194A
:1057C80009E1EA51EE1906E10101A551A61102E12C
:1057D8000201B9835050220D000EF3240001746FAA
:1057E800030EF420756F350E766F0B0E776F010E72
:1057F800796F786BAC0E7A6F010E7B6FE4EC17F063
:105808000101AE6FAE5101E00ED7AC51AD1101E10F
:105818000AD7ACC11EF0ADC11FF045EC38F001014C
:10582800AC51A727AD51A823000EA923AA23505095
:105838001C0D070EF324D96E010EF420DA6E000E4B
:10584800DE240001E76F010EDE20E86F000EDE2087
:10585800E96F000EDE20EA6F000EDE20EB6F000E0F
:10586800DE20EC6F000EDE20ED6F000EDE20EE6F06
:1058780050501C0D070EF324D96E010EF420DA6E79
:10588800E7C0DEFFE8C0DEFFE9C0DEFFEAC0DEFFFA
:10589800EBC0DEFFECC0DEFFEDC0DEFFEEC0DEFFDA
:1058A8000101A34BA42BA3C1E7F0A4C1E8F0000EAB
:1058B8000001E8BFFF0EE96FEA6F01019F51000187
:1058C800E75D0101A0510001E8590101A151000162
:1058D800E9590101A2510001EA5901E24CD701013D
:1058E800A551A61165E05050220D000EF3240001C9
:1058F800746F030EF420756F350E766F0B0E776F8D
:10590800A5C178F0A6C179F0AC0E7A6F010E7B6F55
:10591800E4EC17F00101AE6FAE5101E084D602014C
:10592800B983A5C11EF0A6C11FF045EC38F00101EE
:10593800AC51A727AD51A823000EA923AA23505084
:105948001C0D070EF324D96E010EF420DA6E000E3A
:10595800DE240001E76F010EDE20E86F000EDE2076
:10596800E96F000EDE20EA6F000EDE20EB6F000EFE
:10597800DE20EC6F000EDE20ED6F000EDE20EE6FF5
:1059880050501C0D070EF324D96E010EF420DA6E68
:10599800E7C0DEFFE8C0DEFFE9C0DEFFEAC0DEFFE9
:1059A800EBC0DEFFECC0DEFFEDC0DEFFEEC0DEFFC9
:1059B8000201B9934E6A8390839EA1D642C0D9FF53
:1059C80043C0DAFFDECF72F0DDCF73F047504610E8
:1059D800451003E1020E445C10E3000120EE13F0D1
:1059E8007251D9267351DA22DE50445CDE50455894
:1059F800DE504658DE50475808E3010E00016C6F30
:105A0800000E6D6B6E6B6F6B8FD16C696D696E6913
:105A18006F6976D144C070F045C071F0D89071318B
:105A2800616F7031606F605170276151712372C06E
:105A380037F073C038F020EE1FF07251D926735139
:105A4800DA22DECF60F0DECF61F0DECF62F0DECFAB
:105A580063F070C064F071C065F0090E666FD8908D
:105A680065336433662FFBD764516025396E655101
:105A780061213A6E000E62213B6E000E63213C6E7E
:105A8800F6EC54F0000901E04FD100016069010E05
:105A9800616F70C062F071C063F06051621761514C
:105AA800631772C064F073C065F062516427635174
:105AB80065232F0E6425D96E000E6521DA6EDF503E
:105AC8006A6F6B6B704B712B72C037F073C038F014
:105AD80020EE1FF07251D9267351DA22DECF60F022
:105AE800DECF61F0DECF62F0DECF63F070C064F02D
:105AF80071C065F0090E666FD89065336433662F00
:105B0800FBD764516025396E655161213A6E000EEC
:105B180062213B6E000E63213C6EF6EC54F00009E6
:105B280001E002D100016069010E616F70C062F08E
:105B380071C063F0605162176151631772C064F0FD
:105B480073C065F062516427635165232F0E642585
:105B5800D96E000E6521DA6EDF50676F666B66518D
:105B68006A1367516B1344B006D06A51686F0F0E01
:105B78006B15696F0FD06AC060F06BC061F0040EDE
:105B8800626FD89061336033622FFBD760C068F0D2
:105B980061C069F068C06CF069C06DF04ED072C029
:105BA80037F073C038F020EE1FF07251D9267351C8
:105BB800DA22DECF60F0DECF61F0DECF62F0DECF3A
:105BC80063F04550646F4650656F4750666F676B6A
:105BD80060516425396E615165213A6E62516621C2
:105BE8003B6E635167213C6EF6EC54F0000901E00E
:105BF8009BD000016069010E616F44C062F045C02E
:105C080063F0D89062376337605162176151631748
:105C180072C064F073C065F06251642763516523F4
:105C28002F0E64250B6E000E65210C6EDAEC5EF00B
:105C38000BC06CF00CC06DF000016E6B6F6B74D014
:105C480072C037F073C038F020EE1FF07251D926B9
:105C58007351DA22DECF60F0DECF61F0DECF62F082
:105C6800DECF63F044C064F045C065F046C066F01E
:105C780047C067F0080E05D0D890673366336533A0
:105C88006433E82EF9D760516425396E6151652176
:105C98003A6E625166213B6E635167213C6EF6ECA9
:105CA80054F0000941E100016069010E616F44C0D0
:105CB80062F045C063F0D89062376337D890623796
:105CC8006337605162176151631772C064F073C023
:105CD80065F062516427635165232F0E64250B6EAE
:105CE800000E65210C6E01EC54F00B5000016C6F36
:105CF8000C506D6F0D506E6F0F0E0E146F6F14D029
:105D080072C0D9FF73C0DAFFDF50606F616B6151F9
:105D180001E073D66051010A01E17CD6030A01E172
:105D28003ED7010A8DE069D66CC042F06DC043F0E1
:105D38006EC044F06FC045F01200506A0101916BCB
:105D4800506A030E506401D090D1505003E11E6A8E
:105D58001F6A03D01F6A010E1E6E50501C0D1B0EC9
:105D6800F324D96E010EF420DA6EDF6A50501C0D50
:105D7800000EF324D96E010EF420DA6EDF6A50505B
:105D88001C0D070EF324D96E010EF420DA6E070EEF
:105D9800DE6AE806FDE20D0E1E02F3CF9FF1F4CF96
:105DA800A0F11F02F3500101A027310E9F25D96EE3
:105DB800020EA021DA6EDF50A16FA1C1A2F1A36B80
:105DC800A46BA56BA4C1A5F1A3C1A4F1A2C1A3F1C1
:105DD800A26BA2C1A6F1A3C1A7F1A4C1A8F1A5C154
:105DE800A9F1AA6BA9BFAA69AAC1ABF1AAC1ACF172
:105DF800AAC1ADF10D0E1E02F3CFAEF1F4CFAFF193
:105E08001F02F350AF27300EAE25D96E020EAF2118
:105E1800DA6EDF50B06FB0C1B1F1B26BB36BB46B77
:105E2800B2C1B4F1B1C1B3F1B26BB16BB1C1B5F1EB
:105E3800B2C1B6F1B3C1B7F1B4C1B8F1B96BB8BF6B
:105E4800B969B9C1BAF1B9C1BBF1B9C1BCF10D0E9B
:105E58001E02F3CFBDF1F4CFBEF11F02F350BE27EF
:105E68002F0EBD25D96E020EBE21DA6EDF50BF6F30
:105E7800BFC1C0F1C16BC26BC36BC0C1C3F1C26B00
:105E8800C16BC06BC0C1C4F1C1C1C5F1C2C1C6F10B
:105E9800C3C1C7F1C86BC7BFC869C8C1C9F1C8C108
:105EA800CAF1C8C1CBF10D0E1E02F3CFCCF1F4CF6D
:105EB800CDF11F02F350CD272E0ECC25D96E020E40
:105EC800CD21DA6EDF50CE6FCEC1CFF1D06BD16B62
:105ED800D26BD36BD46BD56BD66B200ED890CF37E3
:105EE800D037D137D237D337D437D537D637E82E4E
:105EF800F5D7C451CF25D76FC551D021D86FC6511A
:105F0800D121D96FC751D221DA6FC851D321DB6FA4
:105F1800C951D421DC6FCA51D521DD6FCB51D621AF
:105F2800DE6FB551D725DF6FB651D821E06FB75175
:105F3800D921E16FB851DA21E26FB951DB21E36F62
:105F4800BA51DC21E46FBB51DD21E56FBC51DE2184
:105F5800E66FA651DF25E76FA751E021E86FA8514A
:105F6800E121E96FA951E221EA6FAA51E321EB6F20
:105F7800AB51E421EC6FAC51E521ED6FAD51E62159
:105F8800EE6F50501C0D0F0EF324D96E010EF42045
:105F9800DA6EE7C1DEFFE8C1DEFFE9C1DEFFEAC174
:105FA800DEFFEBC1DEFFECC1DEFFEDC1DEFFEEC1BF
:105FB800DEFFB40E00019C6FFA0E9D6F50C09EF07C
:105FC8009F6B50501C0D0F0EF324D96E010EF42058
:105FD800DA6EDECF9FF1DECFA0F1DECFA1F1DECF0A
:105FE800A2F1DECFA3F1DECFA4F1DECFA5F1DECFA3
:105FF800A6F19FC1A0F0A0C1A1F0A1C1A2F0A2C1C9
:10600800A3F0A3C1A4F0A4C1A5F0A5C1A6F0A6C1A0
:10601800A7F050501C0D0F0EF324D96E010EF4207A
:10602800DA6EDECFA7F1DECFA8F1DECFA9F1DECFA1
:10603800AAF1DECFABF1DECFACF1DECFADF1DECF32
:10604800AEF1A7C1A8F0A8C1A9F0A9C1AAF0AAC138
:10605800ABF0ABC1ACF0ACC1ADF0ADC1AEF0AEC110
:10606800AFF0CAEC60F0502A6CD60101946B4F6A0D
:10607800936B826B836B020E4E6E926F8390020C51
:1060880095C0D9FF96C0DAFFDECFADF0DDCFAEF018
:1060980020EE0EF09551D9269651DA22DECF99F0EE
:1060A800DECF9AF0DECF9BF0DECF9CF0200E992554
:1060B800A96F000E9A21AA6F000E9B21AB6F000EEC
:1060C8009C21AC6FAC5103E1200EAB5D0AE320EEDE
:1060D80016F09551D9269651DA22DE6ADE6ADE6A12
:1060E800DD6A20EE16F09551D9269651DA22DE5057
:1060F800DE10DE10DE1001E1040CA951996F010ECB
:10610800AA159A6F9B6B9C6B99119B119C1101E0CE
:1061180029D120EE16F09551D9269651DA22DE2A99
:10612800000EDE22DE22DE2220EE12F09551D92664
:106138009651DA22DE50DE10DE10DE102CE120EE61
:1061480007F0AD51D926AE51DA22DECF99F0DDCF76
:106158009AF099519B6F9A519C6F9D6B9E6BA9C049
:106168009FF0AAC0A0F0ABC0A1F0ACC0A2F0060E90
:1061780005D0D890A233A133A0339F33E82EF9D7A6
:106188009B519F5D9C51A0599D51A1599E51A25967
:1061980001E2E8D06ED099699A6920EE09F0AD5114
:1061A800D926AE51DA22DECF9BF0DDCF9CF0995193
:1061B8009B279A519C23A9C09DF0AAC09EF0ABC012
:1061C8009FF0ACC0A0F00A0E05D0D890A0339F3342
:1061D8009E339D33E82EF9D79B519D15A16F9C5195
:1061E8009E15A26FA36BA46BA111A311A41101E0CA
:1061F800B9D095C042F096C043F020EE12F0955108
:10620800D9269651DA22DECF44F0DECF45F0DECF34
:1062180046F0DECF47F0E2EC2CF042C0AFF043C0CE
:10622800B0F044C0B1F045C0B2F00001B251B111B4
:10623800B01104E1020EAF5D01E2020CAF2907E1E3
:10624800B02905E1B12903E1B22901E1010C20EEF1
:1062580013F0AD51D926AE51DA22DE50AF5DDE50D3
:10626800B059DE50B159DE50B25950E397519811E8
:106278000BE120EE16F09551D9269651DA22DE6A06
:10628800DE6ADE6ADD6A040C95C078F096C079F0A3
:1062980020EE12F09551D9269651DA22DECF7AF007
:1062A800DECF7BF0DECF7CF0DECF7DF010EC23F08C
:1062B80078C0AFF079C0B0F07AC0B1F07BC0B2F06E
:1062C800AF51B011B111B21101E1070CAF05B01116
:1062D800B111B21101E1020CAF2907E1B02905E1C2
:1062E800B12903E1B22901E1010CADC037F0AEC01C
:1062F80038F0AFC039F0B0C03AF0B1C03BF0B2C02E
:106308003CF0DFEC4CF0000901E0010C000120EE4C
:1063180012F09551D9269651DA22AFC0DEFFB0C0EF
:10632800DEFFB1C0DEFFB2C0DEFFADC00BF0AEC015
:106338000CF0AFC00DF0B0C00EF0B1C00FF0B2C09D
:1063480010F04DEC4BF0000120EE16F09551D926D7
:106358009651DA220BC0DEFF0CC0DEFF0DC0DEFF57
:106368000EC0DEFF20EE0EF09551D9269651DA22A6
:10637800A9C0DEFFAAC0DEFFABC0DEFFACC0DEFFF7
:106388009969010E9A6FA9C09BF0AAC09CF0995117
:106398009B179A519C17ADC09DF0AEC09EF09B51C3
:1063A8009D279C519E232F0E9D27000E9E2320EE95
:1063B8001AF09551D9269651DA229DC0DEFF9EC06B
:1063C800DDFF000C000E0001DB6F250EDA6F000EFA
:1063D800D96F050ED86F0101FD5105E1000E0001CE
:1063E800DB6F280EDA6F010197510DE1FC6B350E5A
:1063F8000001796F0D0E7A6FBF0E7B6FFE0E7C6FFA
:1064080017EC5EF00DD0F20E00019C6FFA0E9D6F36
:1064180097C19EF09F6BFCC1A0F0A16BCAEC60F025
:10642800380E9C6FFE0E9D6F0101FC510F0D350E4D
:10643800F32400019E6F0D0EF4209F6FCAEC60F0EC
:10644800050E0001D76F0F0ED66FF10EE82EFED79E
:10645800D62FFCD7D72FFAD7E3D00C0E0C6EFD0E33
:106468000D6EBEEC5BF0030E0101FE6105D0965087
:10647800FE19F00BFE1905D0FEC193FF9650F00BE4
:106488000A09966E000E0001C96F030ECA6FB20E9C
:10649800CB6FFE0ECC6F010ECD6F1CEC15F0010119
:1064A8009B6F9B513AEC5CF001019B510AE1FCECBB
:1064B80035F0000E486E030E496EFAEC5DF00101EE
:1064C8009B6F9B513AEC5CF0DB6B280EDA6FA4D023
:1064D8000101FC510F0D350EF324D96E0D0EF42079
:1064E800DA6E200EDE1806E1FC2B0F0EFC6594D048
:1064F800FC6B92D01D0E00019C6FFC0E9D6F01017C
:10650800FC510F0D350EF32400019E6F0D0EF42083
:106518009F6FCAEC60F0000EC96F030ECA6F0101CD
:10652800FC510F0D350EF3240001CB6F0D0EF42036
:10653800CC6F030ECD6F1CEC15F001019B6F9B51C6
:106548003AEC5CF001019B5104E10001DB6B3C0E6D
:10655800DA6F040E01019B1904E10001DB6B320EB6
:10656800DA6F050E0001D76F0F0ED66FF10EE82E09
:10657800FED7D62FFCD7D72FFAD74ED0D80E9C6F80
:10658800FC0E9D6F0101FC510F0D350EF324000127
:106598009E6F0D0EF4209F6FCAEC60F0000EC96F5D
:1065A800030ECA6F0101FC510F0D350EF3240001D3
:1065B800CB6F0D0EF420CC6F070ECD6F1CEC15F0D1
:1065C80001019B6F9B51CDE10001DB6B3C0EC8D7ED
:1065D800B30E9C6FFC0E9D6F0101FC510F0D350E23
:1065E800F32400019E6F0D0EF4209F6FCAEC60F03B
:1065F80013D0DAC0D6F0DBC0D7F0D7510DE1D651B1
:10660800250A01E12AD70D0A01E162D7050A04E04B
:106618001F0AB4E00E0ADCE00001D807D8A0D907A9
:106628000001D9BF08D0D95102E1D80504E33C0ED6
:10663800DA19DB11DEE1030E010197193BE1839EB4
:10664800000E0B6EC00E8BEC5CF0D9EC5FF0000E08
:106658000B6EC00E8BEC5CF03C0E0001DA19DB11FE
:1066680016E102014B510CE04B0E0F6E020E106E3C
:1066780007EC58F0D60E0F6EFE0E106E07EC58F0B1
:10668800A00E0F6EFF0E106E07EC58F0000C350EC2
:10669800796F0D0E7A6F530E7B6FFF0E7C6F9BC167
:1066A8007DF07E6B17EC5EF0350E0F6E0D0E106EE2
:1066B80007EC58F0000C74C0D9FF75C0DAFFDECFC4
:1066C80090F0DDCF91F0795109E1200E785DD8B0D6
:1066D800020C76C07AF01F0E7A1701E0020C20EE49
:1066E8000EF07451D9267551DA2276C0DEFF77C0D4
:1066F800DEFF78C0DEFF79C0DEFF20EE06F07451C1
:10670800D9267551DA22DECF8CF0DECF8DF0DECFC0
:106718008EF0DECF8FF08C518D118E118F1115E117
:1067280090C0D9FF91C0DAFF020EDF640ED020EED0
:1067380023F09051D9269151DA22DECF8CF0DECFAA
:106748008DF0DECF8EF0DECF8FF08C518D118E1153
:106758008F1140E120EE07F09051D9269151DA22AD
:10676800DECF7AF0DDCF7BF07A517C6F7B517D6F85
:106778007E6B7F6B76C080F077C081F078C082F046
:1067880079C083F0060E05D0D890833382338133E5
:106798008033E82EF9D77C51805D7D5181597E5137
:1067A80082597F51835901E3020C20EE23F0905166
:1067B800D9269151DA2210EE16F07451E12675515E
:1067C800E222DECFE6FFDECFE6FFDECFE6FFDECF5A
:1067D800E6FF87D020EE09F09051D9269151DA22B0
:1067E800DECF7AF0DDCF7BF07A517C6F7B517D6F05
:1067F8007E6B7F6B090ED8907C377D377E377F376D
:10680800E82EF9D77CC088F07DC089F07EC08AF078
:106818007FC08BF040D074C042F075C043F08CC08C
:1068280044F08DC045F08EC046F08FC047F0E2ECD2
:106838002CF042C08CF043C08DF044C08EF045C0AF
:106848008FF000018C2907E18D2905E18E2903E1EC
:106858008F2901E1010C8F518E118D1104E1020E77
:106868008C5DD8A0020C20EE13F09051D9269151DE
:10687800DA22DE508C5DDE508D59DE508E59DE50A6
:106888008F5901E3020C8851765F8951775B8A51F1
:10689800785B8B51795B8851765D895177598A513C
:1068A80078598B517959B7E290C00BF091C00CF030
:1068B8008CC00DF08DC00EF08EC00FF08FC010F0A0
:1068C8004DEC4BF0000120EE16F07451D9267551AD
:1068D800DA220BC0DEFF0CC0DEFF0DC0DEFF0EC0EB
:1068E800DEFF20EE12F07451D9267551DA228CC0E1
:1068F800DEFF8DC0DEFF8EC0DEFF8FC0DEFF20EE24
:1069080016F07451D9267551DA22DE50DE10DE10E9
:10691800DE1001E1020C76C07AF077C07BF078C017
:106928007CF079C07DF00A0E05D0D8907D337C3399
:106938007B337A33E82EF9D720EE16F07451D92636
:106948007551DA227A51DE267B51DE227C51DE2215
:106958007D51DE227A69010E7B6F76C07CF077C0AC
:106968007DF07A517C177B517D1790C07EF091C0E5
:106978007FF07C517E277D517F232F0E7E27000ECE
:106988007F2320EE1AF07451D9267551DA227EC081
:10699800DEFF7FC0DDFF000C1550D96EDA6ADECF4E
:1069A8001FF0DDCF20F01C0E1324236E000E1420E0
:1069B800246E23C00BF024C00CF00E6A200E0D6E5E
:1069C800106A0B0E0F6E3CEC60F0256A266A216A8D
:1069D800226A1E6A080E1D6E21501F24166E225050
:1069E8002020176E16C0F6FF17C0F7FF000EF86ECE
:1069F8000E0EF76403D00800F55005D0F6CFE9FF76
:106A0800F7CFEAFFEF50276E214A222A210E27608E
:106A180001D0BED02F0E271806E05C0E271803E021
:106A280036D0214A222A21501F24166E22502020B7
:106A3800176E16C0F6FF17C0F7FF000EF86E0E0EA1
:106A4800F76403D00800F55005D0F6CFE9FFF7CF7B
:106A5800EAFFEF502F0AE5E021501F24166E22505E
:106A68002020176E16C0F6FF17C0F7FF000EF86E4D
:106A78000E0EF76403D00800F55005D0F6CFE9FFF5
:106A8800F7CFEAFFEF505C0A01E082D0CAD72E0E9A
:106A9800271805E01D50255C1E5026580FE30B0EE5
:106AA8001D181E10D8B4060C2E0E271801E0060C6F
:106AB800266A080E256E1E6A0B0E8DD7275063ECCA
:106AC8005CF00B500C1044E021501F24166E22502D
:106AD8002020176E16C0F6FF17C0F7FF000EF86EDD
:106AE8000E0EF76403D00800F55005D0F6CFE9FF85
:106AF800F7CFEAFFEF501C6E214A222A1C509CEC6B
:106B080059F00B500C10D8B4060C166817681DC045
:106B180018F01EC019F016501826175019221850D0
:106B2800255C1950265801E3060C25502324D96EFC
:106B380026502420DA6E27C0DFFF254A262A255052
:106B48002324D96E26502420DA6E1CC0DFFF1DD006
:106B5800DE0E0B6EFD0E0C6E27C00DF00E6A51ECAA
:106B68005EF00B500C1001E0060C600E276405D097
:106B78007B0E276002D0200E275E25502324D96E75
:106B880026502420DA6E27C0DFFF254A262A24D77C
:106B980021501F24166E22502020176E1550D96ED2
:106BA800DA6A16C0DEFF17C0DDFF2550261001E1A6
:106BB800060C23C0D9FF24C0DAFFE50EDE1806E173
:106BC80023C0D9FF24C0DAFF050EDF6E200E27642C
:106BD80003D01A6A1B6A03D01B6A040E1A6E20EED1
:106BE8000BF02350D9262450DA221AC0DFFF000CFC
:106BF8003B0EF66EF90EF76E0900F5CFC5F00A00E8
:106C0800F5CFC6F00001CB6B02014B6B030E0101FF
:106C1800FE6105D09650FE19F00BFE1905D0FEC195
:106C280093FF9650F00B0A09966ECD6ACE6AEED0A5
:106C3800CC6B350E146E0B0E156EC50E166E8FECE2
:106C480055F014C0C9F015C0CAF0C9C0D9FFCAC0F0
:106C5800DAFF3B0EDE1801E0D4D0D8D0CC5109E1E0
:106C6800C9C00FF0CAC010F064EC59F00001CB6F36
:106C7800BDD0CC051BE10101FC510001CB1903E09B
:106C88007F0ECB1913E1C9C00FF0CAC010F064EC35
:106C980059F001019A6F380E00019C6FFF0E9D6F2D
:106CA8009AC19EF09F6BCAEC60F0A0D0020ECC197E
:106CB8001BE10101FC510001CB1903E07F0ECB1948
:106CC80013E1C9C00FF0CAC010F064EC59F001011B
:106CD800996F410E00019C6FFF0E9D6F99C19EF048
:106CE8009F6BCAEC60F082D0020ECC651FD0080EF4
:106CF800CC611CD00101FC510001CB1903E07F0ECF
:106D0800CB1914E1550EC76F020EC86FC9C00FF03A
:106D1800CAC010F064EC59F00001C26FCC51C7250D
:106D2800C36F000EC821C46FFD0E40D0070ECC659E
:106D38001FD01B0ECC611CD00101FC510001CB19E6
:106D480003E07F0ECB1914E1000EC76F020EC86F67
:106D5800C9C00FF0CAC010F064EC59F00001C26F4E
:106D6800CC51C725C36F000EC821C46FF80E1ED0C2
:106D7800280ECC6123D00101FC510001CB1903E09E
:106D88007F0ECB191BE1260EC76F020EC86FC9C054
:106D98000FF0CAC010F064EC59F00001C26FCC517A
:106DA800C725C36F000EC821C46FE50EC325D96E71
:106DB800FF0EC421DA6EC2C0DFFF18D0280ECC192E
:106DC80015E10101FC510001CB1903E07F0ECB193D
:106DD8000DE14B0E0B6E020E0C6EC9C00DF0CAC051
:106DE8000EF0106A080E0F6E69EC5BF0CC2B146A7B
:106DF800156AC50E166E8FEC55F014C0C9F015C093
:106E0800CAF00001C951CA1101E028D7350E0001A6
:106E18009F6F0B0EA06FA26B910EA16F000EA36F58
:106E2800030EA46FD9EC55F09F51A01101E000D7D3
:106E3800440E9C6FFB0E9D6F4B0E9E6F020E9F6F54
:106E4800CAEF60F0276E0001C35102E0A1EC2EF0FA
:106E5800266A0001C25101E1FAD0040E271802E1A6
:106E68004F5003E1140E271809E10101936B826B5F
:106E7800836B0001C36B070EC26F070C3F0E271808
:106E880007E14F6A0101936B0001C26BC36B1200EB
:106E98005F0E271807E10101946B936B0001C26B29
:106EA800C36B12003F0E276406D05F0E276003D025
:106EB800400E2718F0E1400E271809E1010E0101E4
:106EC800946F0101936B0001C26BC36B1200200E1B
:106ED800271803E1010E4F6EF4D7650E271809E154
:106EE8004F5007E00101826B836B010E936F838023
:106EF800EAD76E0E271803E1020E0101936F700E98
:106F0800271807E10101945104E0826B836B030E9B
:106F1800936F700E271808E14F5006E08380010137
:106F2800826B836B040E0FD0720E271801E08FD08E
:106F38004F5001E18CD083800101916B1C0E836F4F
:106F48002A0E826F050E936FBED7275008EC0CF0FF
:106F5800266E92D08380275081EC57F0266E01016F
:106F6800936B8AD08380D40E00019C6FFA0E9D6FBC
:106F7800CECF9EF09F6BCDCFA0F0A16B4EC0A2F0FC
:106F8800A36BCAEC60F0350E0B6E0B0E0C6E0E6A1E
:106F98000D6A010E106E0F6A7EEC48F00201B9838B
:106FA8002BEE35F04EC0DFFF1F6A010E1E6E45EC5A
:106FB80038F00201B993080E266E0101936B4E6AF0
:106FC8005BD08390266A58D0080E271822E1839058
:106FD800266A4E6A030E916522D00F0E91191FE0A2
:106FE800010E4E6E50501C0D1B0EF324D96E010E6F
:106FF800F420DA6E50501C0D1B0EF324E16E010EC6
:10700800F420E26EE7501009DF6E09D0826B836BC3
:1070180033D0090E271805E18390266A4E6A936BD0
:10702800F5D71F0E276428D0300E276025D0060E0E
:1070380000019C6FFC0E9D6F27C09EF09F6BCAECF1
:1070480060F027500F0B0101916F266AB8D7010134
:107058009351246E256A25500FE124500DE0010A52
:1070680001E173D7030A01E175D7010A01E17AD773
:10707800070AA7E0010AA8E026C0C2F00001C36B16
:10708800120001019E6B886B896BFF0E1E24226E15
:10709800FF0E1F20236E89868980898289848988CA
:1070A8008B68849084928494849883500F01139100
:1070B800350EE82EFED700F007D0FC0E00019C6FBD
:1070C800FF0E9D6FCAEC60F08EA8F7D7E3D08EA8AC
:1070D8008EAA14D0FD5112E1885189110FE03F0E9C
:1070E80000019C6FFD0E9D6F88C19EF089C19FF0C5
:1070F800CAEC60F0630E01019E6FD2D0100E746F5F
:10710800270E756F766B776BADD08EB28EA410D0CC
:107118007407000E755B765B775B742906E1752949
:1071280004E1762902E17729D8A4B4D0620E86D08A
:10713800010E84D08EA8AED0020E80D0350E8825E0
:10714800D96E0B0E8921DA6EDF1C866E88512218E3
:1071580006E18951231803E10201B9B3899A0101B3
:10716800884B892B8B6A030E9E6F100E746F270E47
:10717800756F766B776B06D08EA204D08990050E5A
:107188009E6F0ED07407000E755B765B775B742973
:10719800F3E17529F1E17629EFE177297BE0ECD776
:1071A800100E746F270E756F766B776B0DD08EA4EB
:1071B8000BD0898A89808B681E50885D1F50895939
:1071C800BBE3630E01013AD07407000E755B765B72
:1071D800775B7429ECE17529EAE17629E8E17729FA
:1071E80059E0E5D78EB20DD07407000E755B765B5B
:1071F800775B74294FE175294DE176294BE17729B1
:1072080049E1040E1BD08990050E9E6F100E746F15
:10721800270E756F766B776B3DD089848EB40DD051
:107228007407000E755B765B775B742933E175290B
:1072380031E176292FE177292DE1060E9E6F2AD0BC
:10724800898A89808B681E50885D1F50895901E2A0
:107258006FD7B7D7A60E00019C6FFF0E9D6FCAECC3
:1072680060F0AFD79E51206E216A215013E1205063
:1072780001E14BD7010A01E15DD7030A01E15ED7BD
:10728800010AB0E0070ABFE0010AC7E0030AD8E034
:10729800640AE0E0630E01019E1902E08EBC17D774
:1072A8008980898289848988898A8B680F011381FA
:1072B80088C11EF089C11FF01200350EFE6F0B0E3B
:1072C800FF6FE4C00BF0E5C00CF01BEC5DF00B5059
:1072D8000001F26FC20E956F966B976B986B996B66
:1072E8009A6B4EEC12F0FB6FFB510BE05E0E9C6F3D
:1072F800FB0E9D6FCAEC60F0C26BC36BC46BC56BB1
:107308001200C20E746F756BFEC076F0FFC077F086
:10731800010E796F786BF90E7A6F7B6BE4EC17F0DE
:10732800FB6FFB5107E0EF0E9C6FFB0E9D6FCAECE5
:1073380060F0E2D7FEC0D9FFFFC0DAFF800EDE188A
:1073480007E0FB0E9C6FFC0E9D6FCAEC60F0D4D773
:1073580020EE0AF0FE51D926FF51DA22DF50E76FFE
:10736800E66B20EE0BF0FE51D926FF51DA22DF50F2
:10737800E625F76F000EE721F86FD80E9C6FFB0E1D
:107388009D6FF7C09EF0F8C09FF0CAEC60F0C20E87
:10739800956F966BF751E76FE66BE6C097F0E7C01D
:1073A80098F0996B9A6B4EEC12F0FB6FFB51A4E1CD
:1073B800C20E746F756BFEC076F0FFC077F0010ED9
:1073C800796F786BF90E7A6F7B6BE4EC17F0FB6FD3
:1073D800FB5192E1FC6BFD6BE4C00BF0E5C00CF0D7
:1073E800FCC0E6F0FDC0E7F0050ED890E637E737B9
:1073F800E82EFBD7E651FE250D6EE751FF210E6EF4
:10740800F2C00FF0106A6BEC56F00B500C105AE1FA
:10741800FCC0E6F0FDC0E7F0050ED890E637E73788
:10742800E82EFBD7FEC0E8F0FFC0E9F0E651E827F8
:10743800E751E9230E0EE825D96E000EE921DA6E30
:10744800DF50EB6FEA6BFCC0ECF0FDC0EDF0050E11
:10745800D890EC37ED37E82EFBD7FEC0EEF0FFC032
:10746800EFF0EC51EE27ED51EF230F0EEE25D96E1C
:10747800000EEF21DA6EDF50F06FF16BEA51F02762
:10748800EB51F123F0C0F3F0F1C0F4F0000EF4BFBB
:10749800FF0EF56FF66FC00E9C6FFD0E9D6FF3C06B
:1074A8009EF0F4C09FF0F5C0A0F0F6C0A1F0CAECC1
:1074B80060F0F3C0C2F0F4C0C3F0F5C0C4F0F6C089
:1074C800C5F01200FC4BFD2BFDBF86D7FD5105E131
:1074D8000F0EFC5D01E310D77FD70ED70201B983E9
:1074E800350E0B6E0B0E0C6E0E6A0D6A010E106EC9
:1074F8000F6A7EEC48F0000EE8CF35FBFF0EE8CFB0
:1075080036FB50501C0D1B0EF324D96E010EF420CF
:10751800DA6E0101DFA403D0010EE8CF37FB50502B
:107528001C0D1B0EF324D96E010EF420DA6EDFA8B1
:1075380003D0020EE8CF37FB50501C0D1B0EF3246E
:10754800D96E010EF420DA6EDFA003D0020EE8CF68
:1075580039FB50501C0D1B0EF324D96E010EF4207C
:10756800DA6EDFA203D0020EE8CF39FB50501C0DB3
:107578001B0EF324D96E010EF420DA6EDFA603D0B9
:10758800800EE8CF38FB8FA403D0080EE8CF3BFB72
:10759800266A276A8F0E2624D96E020E2720DA6EF5
:1075A800DF1C256E370E2624D96E0B0E2720DA6EC7
:1075B800370E2624E16E0B0E2720E26EE7502514C5
:1075C800DF6E264A272A27BEE5D7275003E1070E94
:1075D800265CE0E34E6A020E916548D050501C0DBF
:1075E800010EF324D96E010EF420DA6EDF50246EFA
:1075F80024C040FB50501C0D020EF324D96E010E1E
:10760800F420DA6EDF50246E24C041FB50501C0D6C
:10761800030EF324D96E010EF420DA6EDF50246EC7
:1076280024C042FB50501C0D040EF324D96E010EE9
:10763800F420DA6EDF50246E24C043FB50501C0D3A
:10764800050EF324D96E010EF420DA6EDF50246E95
:1076580024C044FB50501C0D060EF324D96E010EB5
:10766800F420DA6EDF50246E24C045FB1F6A140E26
:107678001E6E45EC38F0260E00019C6FFF0E9D6FC4
:10768800CAEC60F0266A276A3D0E9C6FFF0E9D6F5C
:10769800350E2624D96E0B0E2720DA6EDF509E6F2A
:1076A8009F6BCAEC60F0264A272A27BEEDD72750E1
:1076B80003E1130E265CE8E350501C0D1B0EF32467
:1076C800D96E010EF420DA6EDF6A0201B993839055
:1076D800000C50501C0D070EF324D96E010EF42037
:1076E800DA6EDECFE2F0DECFE3F0DECFE4F0DECF1D
:1076F800E5F050501C0D070EF324D96E010EF4204E
:10770800DA6E50501C0D0F0EF324E16E010EF420BA
:10771800E26EDE50E65CDE50E658DE50E658DE509B
:10772800E658DE50E658DE50E658DE50E658DE50A1
:10773800E65815E2010E4E6E50501C0D1B0EF32438
:10774800D96E010EF420DA6E50501C0D1B0EF32476
:10775800E16E010EF420E26EE7500409DF6E50502E
:107768001C0D070EF324D96E010EF420DA6EDECF5D
:10777800BEF0DECFBFF0DECFC0F0DECFC1F0DECF8F
:10778800C2F0DECFC3F0DECFC4F0DECFC5F050507C
:107798001C0D170EF324D96E010EF420DA6EDECF1D
:1077A800C6F0DECFC7F0DECFC8F0DECFC9F00001EB
:1077B800C651CA6FC751CB6FC851CC6FC951CD6F75
:1077C800CE6BCF6BD06BD16BBE51CA25D26FBF5178
:1077D800CB21D36FC051CC21D46FC151CD21D56FEE
:1077E800C251CE21D66FC351CF21D76FC451D021FA
:1077F800D86FC551D121D96F50501C0D0F0EF324ED
:10780800D96E010EF420DA6ED251DE5CD351DE5807
:10781800D451DE58D551DE58D651DE58D751DE58EE
:10782800D851DE58D951DE5815E2010E4E6E50502F
:107838001C0D1B0EF324D96E010EF420DA6E505085
:107848001C0D1B0EF324E16E010EF420E26EE750CE
:107858000409DF6E4E6A5050220D000EF324956F16
:10786800030EF420966FE2C097F0E3C098F0E4C0EE
:1078780099F0E5C09AF04EEC12F0E66FE65115E08B
:10788800010E4E6E50501C0D1B0EF324D96E010EC6
:10789800F420DA6E50501C0D1B0EF324E16E010E1D
:1078A800F420E26EE7500409DF6E4E5012008EA6F7
:1078B80004D0D50E1E6EFE0E03D0BB0E1E6EFF0E3C
:1078C8001F6E8EAA04D0D50E206EFE0E03D0B60E03
:1078D800206EFF0E216E8EA804D0D50E226EFE0EED
:1078E80003D0020E226EFF0E236E8EAE04D0D50E8C
:1078F800246EFE0E03D0C00E246EFF0E256E8EACD5
:1079080004D0D50E266EFE0E03D0B10E266EFF0EE5
:10791800276E8EA404D0D50E286EFE0E03D0CA0E94
:10792800286EFF0E296E8EA204D0D50E2A6EFE0E8A
:1079380003D0CF0E2A6EFF0E2B6E8EA004D0D50E6C
:107948002C6EFE0E03D0C50E2C6EFF0E2D6E90AE63
:1079580004D0D50E2E6EFE0E03D0F90E2E6EFF0E3D
:107968002F6E90AC04D0D50E306EFE0E03D0F60EFE
:10797800306EFF0E316E90AA04D0D50E326EFE0E18
:1079880003D0F30E326EFF0E336E90A804D0D50EDE
:10799800346EFE0E03D0F00E346EFF0E356E90A6D8
:1079A80004D0D50E366EFE0E03D0ED0E366EFF0EE9
:1079B800376E90A404D0D50E386EFE0E03D0EA0EB2
:1079C800386EFF0E396E90A204D0D50E3A6EFE0EB8
:1079D80003D0E70E3A6EFF0E3B6E90A004D0D50E92
:1079E8003C6EFE0E03D0E40E3C6EFF0E3D6E820E22
:1079F80000019C6FF90E9D6F901C9E6F9F6B8ECF40
:107A0800A0F0A16B3CC0A2F03DC0A3F03AC0A4F026
:107A18003BC0A5F038C0A6F039C0A7F036C0A8F022
:107A280037C0A9F034C0AAF035C0ABF032C0ACF012
:107A380033C0ADF030C0AEF031C0AFF02EC0B0F002
:107A48002FC0B1F02CC0B2F02DC0B3F02AC0B4F0F2
:107A58002BC0B5F028C0B6F029C0B7F026C0B8F0E2
:107A680027C0B9F024C0BAF025C0BBF022C0BCF0D2
:107A780023C0BDF020C0BEF021C0BFF01EC0C0F0C2
:107A88001FC0C1F0CAEF60F0070E0B241A6E000E7B
:107A98000C201B6E0BC0D9FF0CC0DAFFDF500F6E35
:107AA8000F380F0B0A0DF3CF10F0F4CF11F00BC005
:107AB800D9FF0CC0DAFFDF500F0B1026000E112281
:107AC8001028186E000E1120196E1D6A010E1C6E0A
:107AD8001E6A1F6A206A216AB2D01C501D1054E029
:107AE8001EC00FF01FC010F020C011F021C012F00E
:107AF8000A0E0F02F3CF13F0F4CF14F0156A166ACA
:107B08001002F3501426F4501522000E16220F020C
:107B1800F3501426F4501522000E16220A0E1102F4
:107B2800F3501526F4501622000E1002F3501526B5
:107B3800F4501622000E0F02F3501526F4501622A8
:107B48000A0E1202F3501626000E1102F3501626E2
:107B5800000E1002F3501626000E0F02F3501626E0
:107B68001AC0D9FF1BC0DAFFDF50176E17380F0B8A
:107B780013241E6E000E14201F6E000E1520206E9A
:107B8800000E1620216E54D01EC00FF01FC010F03A
:107B980020C011F021C012F00A0E0F02F3CF13F02B
:107BA800F4CF14F0156A166A1002F3501426F45034
:107BB8001522000E16220F02F3501426F450152237
:107BC800000E16220A0E1102F3501526F450162242
:107BD800000E1002F3501526F4501622000E0F0264
:107BE800F3501526F45016220A0E1202F3501626E8
:107BF800000E1102F3501626000E1002F35016263E
:107C0800000E0F02F35016261AC0D9FF1BC0DAFF68
:107C1800DF500F0B13241E6E000E14201F6E000E73
:107C28001520206E000E1620216E1A06D8A01B06FD
:107C38001C501D10010ED8A4000E1C6E1D6A1806DB
:107C4800D8A01906182802E11928D8A446D71EC0BA
:107C58000BF01FC00CF020C00DF021C00EF0120078
:107C68000001D16B010ED06F838E8380D26BD36BF2
:107C7800D46BD56BD0D05050220D000EF324746F06
:107C8800030EF420756F350E766F0B0E776F010EAD
:107C9800796F786BD80E7A6F7B6BE4EC17F0DA6F3C
:107CA800DA5118E0180E01018D6F010E8F6F000177
:107CB800D96BD86F920E9C6FFA0E9D6F50C09EF0D4
:107CC8009F6BDAC0A0F0A16BD8C0A2F0D9C0A3F016
:107CD800CAEC60F00101955135E0705171117211D3
:107CE800731130E050500C0D630EF324D96E020E60
:107CF800F420DA6E70C1C7F071C1C8F072C1C9F062
:107D08000001C66B000EC625CA6F010EC721CB6FD6
:107D1800000EC821CC6F000EC921CD6FDE50CA19E4
:107D280011E1DE50CB190EE1DE50CC190BE1DE502B
:107D3800CD1908E1350E286E0B0E296E01019551FB
:107D48005FEC4EF00201B99301018D5102E002018E
:107D5800B983D8C01EF0D9C01FF045EC38F01EC05A
:107D6800D6F01FC0D7F00001D651D227D751D32360
:107D7800000ED423D5238EAC53D0D851D61903E1A5
:107D8800D951D7190CE0D06BD16B7E0E9C6FFE0ECB
:107D98009D6FD6C09EF0D7C09FF0CAEC60F081EC12
:107DA80060F062EC60F00B500C1004E0010E010171
:107DB8008F6F36D00001CF6B050ECE6F1CD0D00E62
:107DC8000001C26FC90EE82EFED7C22FFCD700D023
:107DD80062EC60F00B500C100EE00001D06BD16B20
:107DE800500E9C6FFD0E9D6FCEC09EF0CFC09FF0D1
:107DF800CAEC60F008D00001CE07D8A0CF07CE2982
:107E0800DEE1CF29DCE162EC60F00B500C1003E0FE
:107E18000001D06BD16B0001D051D11101E02BD7FB
:107E280001018F6B839E83901200838E83804E6A3C
:107E38006DEC3BF00101BB6FBB5102E0BB5112007E
:107E4800536AB36BB46BB56BB66BBA6B010EB96F93
:107E5800BE6BC3D0BC6BBD6B1CD062EC60F00B502A
:107E68000C1013E0BE0E0B6E010E0C6EF9EC56F002
:107E78000101B86F000E5324D96EDA6A040EDA22B3
:107E8800B8C1DFFF532ABC4BBD2B0101BEAB8EAC82
:107E980002D0BD05E2E3BC51B327BD51B423000EA7
:107EA800B523B62350501C0D170EF324D96E010EBE
:107EB800F420DA6EDE50B35DDE50B459DE50B559A9
:107EC800DE50B65902E3B96BBA6BBEAB02D0B96BE0
:107ED800BA6B8EBC02D0B96BBA6BBD0519E2000E45
:107EE80053240B6E0C6A040E0C22FF0E5324D96E19
:107EF800DA6A030EDA22DF500D6E0E6A535000085C
:107F08000F6E000ED8A0E82A0108106E7EEC48F02B
:107F18000101955145E0705171117211731140E0E2
:107F280050503EE150501C0D070EF324D96E010E3F
:107F3800F420DA6E70C1A8F171C1A9F172C1AAF179
:107F4800A76B000EA725AB6F010EA821AC6F000E22
:107F5800A921AD6F000EAA21AE6FAF6BB06BB16BEC
:107F6800B26BDE50AB191CE1DE50AC1919E1DE50E2
:107F7800AD1916E1DE50AE1913E1DE50AF1910E16C
:107F8800DE50B0190DE1DE50B1190AE1DE50B21928
:107F980007E1000E226E040E236E9551B2EC56F0E6
:107FA800ADEC53F00101B76FB75117E0010E4E6EFB
:107FB80050501C0D1B0EF324D96E010EF420DA6EFE
:107FC80050501C0D1B0EF324E16E010EF420E26EDE
:107FD800E7500409DF6E4E501200B951BA1101E0A2
:107FE80039D78FA402D0010E4E6E8390839E000C69
:107FF8009551D8B41200700E00019C6FFD0E9D6F54
:10800800CAEC60F0A7EC54F01EC0A5F11FC0A6F1A1
:1080180020C0A7F121C0A8F10101A551A611A711FF
:10802800A81117E14B0E00019C6FFC0E9D6FA5C1B6
:108038009EF0A6C19FF0A7C1A0F0A8C1A1F0CAEC0C
:1080480060F00A0E0E6E000E0F6A106A116AE8ECF4
:108058005BF00101A96BAA6BE00E00019C6FFF0E9B
:108068009D6FA50E0101A925D96E010EAA21DA6E10
:10807800DF5000019E6F9F6BCAEC60F00101A94BB5
:10808800AA2BAABFE9D7AA5103E1040EA95DE4E32C
:10809800FC0E00019C6FF90E9D6FCAEC60F02A0E71
:1080A8009C6FFB0E9D6FCAEC60F023EE00F000EEB3
:1080B800C2F0210EDBCFEBFFE806FCE2D80EE46F3E
:1080C800FF0EE56F61EC39F0C2C070F1C3C071F109
:1080D800C4C072F1C5C073F1010170517111721100
:1080E8007311D8B41200100E00019C6FFB0E9D6F27
:1080F80070C19EF071C19FF072C1A0F073C1A1F070
:10810800CAEC60F0000E956F030E966F70C1A0F177
:1081180071C1A1F172C1A2F101019F6B000E9F25EF
:108128000001976F010E0101A0210001986F000E58
:108138000101A1210001996F000E0101A221000196
:108148009A6F4EEC12F001019B6F000E0001746FE4
:10815800030E756F350E766F0B0E776F796B080E01
:10816800786FA30E7A6F010E7B6FE4EC17F00101B4
:108178009B6FAB6BAC6B3D0E00019C6FFF0E9D6F50
:10818800350E0101AB25D96E0B0EAC21DA6EDF502E
:1081980000019E6F9F6BCAEC60F00101AB4BAC2BEA
:1081A800ACBFE9D7AC5105E1080EAB5DD8B0120001
:1081B800E2D7120043C024F044C025F014EC44F088
:1081C800456E455001E0D4D043C0D9FF44C0DAFF22
:1081D800030EDE1801E0BCD020EE04F04350D9268F
:1081E8004450DA22DE0401E0B3D02F0E43240B6E94
:1081F800000E44200C6E0E6A0D6A020E106E0F6A95
:108208003CEC60F02D0E43240B6E020E44200C6EE5
:10821800AA0E0E6E550E0D6E02EC60F02F0E432462
:108228000B6E000E44200C6E520E0D6E0E6E610E1B
:108238000F6E410E106E41EC5AF0130E43240B6E74
:10824800020E44200C6E720E0D6E0E6E410E0F6EF5
:10825800610E106E41EC5AF0170E43240B6E020E9D
:1082680044200C6E20EE0FF04350D9264450DA22F9
:10827800DECF0DF0DECF0EF0DECF0FF0DECF10F048
:1082880041EC5AF01B0E43240B6E020E44200C6E78
:1082980020EE0BF04350D9264450DA22DECF0DF001
:1082A800DECF0EF0DECF0FF0DECF10F041EC5AF04B
:1082B80020EE1BF04350D9264450DA22DECF60F07E
:1082C800DECF61F0DECF62F0DECF63F0010E000199
:1082D8006025646F000E6121656F000E6221666F74
:1082E800000E6321676F20EE2BF04350D9264450CF
:1082F800DA2264C0DEFF65C0DEFF66C0DEFF67C04D
:10830800DEFF2F0E43241A6E000E44201B6E20EE53
:108318002BF04350D9264450DA22DECF1CF0DECFB2
:108328001DF0DECF1EF0DECF1FF0216A010E206E99
:1083380020EE01F04350D9264450DA22DF50C0EC39
:108348004FF020EE04F04350D9264450DA22DF6A79
:108358001A6A1B6A1C6A20EE01F04350D926445061
:10836800DA22DF50FDEC20F0000902E0010E456E34
:1083780045501200BBC0D9FFBCC0DAFFDECFC5F044
:10838800DDCFC6F003D00001BD4BBE2BBDC0F6FF4C
:10839800BEC0F7FF000EF86E0E0EF76403D008009B
:1083A800F55005D0F6CFE9FFF7CFEAFFEF502F0AD7
:1083B800EAE0BDC0F6FFBEC0F7FF000EF86E0E0E75
:1083C800F76403D00800F55005D0F6CFE9FFF7CFE2
:1083D800EAFFEF505C0AD7E0000120EE06F0BB513F
:1083E800D926BC51DA22DE6ADE6ADE6ADD6ABDC0E1
:1083F800F6FFBEC0F7FF000EF86E0E0EF76403D04E
:108408000800F55005D0F6CFE9FFF7CFEAFFEF50A7
:108418000001BF6F200EBF6114D020EE27F0BB51C2
:10842800D926BC51DA22800EDF6EBBC074F0BCC006
:1084380075F0000E766F776F786F796F5FEC33F0B9
:1084480023D0BBC013F0BCC014F0BD0E156ED0EC29
:1084580034F00001C86FC85158E1BBC0B3F0BCC0CC
:10846800B4F014EC49F0C86F20EE27F0BB51D926C0
:10847800BC51DA22DF50C76FC85108E0040EC81992
:1084880044E1C7B542D0050EC86F3FD0C7B53DD04F
:1084980020EE04F0BB51D926BC51DA22DFA8F3D76D
:1084A800C5C012F0C6C013F0BF69010EC06F20EE40
:1084B8000EF0BB51D926BC51DA22DECFC1F0DDCF98
:1084C800C2F0BF51C117C051C217C5C0C3F0C6C062
:1084D800C4F0C151C327C251C4232F0EC325146E43
:1084E800000EC421156EB9EC58F0000120EE06F01C
:1084F800BB51D926BC51DA2212C0DEFF13C0DEFF01
:1085080014C0DEFF15C0DEFF9CD7C851120078C02A
:10851800D9FF79C0DAFFDECF8FF0DDCF90F07D5143
:108528007C117B1104E1020E7A5DD8A0020C20EECA
:1085380013F08F51D9269051DA22DE507A5DDE5041
:108548007B59DE507C59DE507D5901E3020C7E5187
:108558007F118011811118E08FC060F090C061F028
:108568007EC062F07FC063F080C064F081C065F0B7
:108578006669676968696969E0EC1EF000018E6FD9
:108588008E5102E08E51120078C042F079C043F05B
:108598007AC044F07BC045F07CC046F07DC047F00F
:1085A800E2EC2CF042C08AF043C08BF044C08CF05F
:1085B80045C08DF000018A518B118C118D1171E02D
:1085C8008A058B118C118D1101E1020C8A2907E1B2
:1085D8008B2905E18C2903E18D2901E1010C8FC06C
:1085E80060F090C061F07AC062F07BC063F07CC03C
:1085F80064F07DC065F0666B676B686B696BE0EC77
:108608001EF000018E6F8E51BDE120EE13F08F51E8
:10861800D9269051DA22FE0EDE24826FFF0EDE206C
:10862800836FFF0EDE20846FFF0EDE20856F20EE45
:108638000FF08F51D9269051DA228251DE5C835196
:10864800DE588451DE588551DE5813E220EE0FF0D3
:108658008F51D9269051DA22DE2A000EDE22DE2240
:10866800DE2220EE04F08F51D9269051DA22000E36
:10867800DB808AC07AF08BC07BF08CC07CF08DC028
:108688007DF020EE13F08F51D9269051DA22DE507A
:108698007A5DDE507B59DE507C59DE507D5901E20F
:1086A80073D7000C1B6E1B5001E0010C54A202D0C2
:1086B80054501200000EEEEC5FF00A0E266E03D046
:1086C800E6EC60F026062650FBE1236A000E146AE9
:1086D800156A166A176A6DEC5EF0E80601E097D035
:1086E800AA0E146E010E156E166A176A080E6DEC46
:1086F8005EF0E80651E1266A26501C0FD96EDA6A48
:10870800E6EC60F0DF6E262A030E2664F5D71E0419
:108718007EE1AA0E1F187BE1030E256EE80E246E7B
:1087280015D0146A156A166A400E176EA90E6DECFC
:108738005EF000090EE0150E1A6EC60EE82EFED782
:108748001A2EFCD700D02406D8A0250624502510C0
:10875800E8E1245025105BE0146A156A166A176A66
:108768003A0E6DEC5EF0000952E1266A26501C0FA5
:10877800D96EDA6AE6EC60F0DF6E262A030E26640C
:10878800F5D71CBC03D0216A040E02D0216A0C0E56
:10879800206E20C023F03BD0146A156A166A176A47
:1087A800A90E6DEC5EF01A6E020E1A6003D0236EED
:1087B800A90E02D0010E236E226E030E256EE80E5E
:1087C800246E14D0146A156A166A176A22506DEC62
:1087D8005EF000090EE0150E1A6EC60EE82EFED7E2
:1087E8001A2EFCD700D02406D8A025062450251020
:1087F800E9E1245025100AE0146A020E156E166A83
:10880800176A100E6DEC5EF0000901E0236A23C0C0
:1088180051F0F7EC60F0235001E14AD7549048D763
:10882800366A20EE03F02450D9262550DA22DF508C
:1088380001E1A7D02F0E24241A6E000E25201B6EEE
:1088480020EE2BF02450D9262550DA22DECF1CF05A
:10885800DECF1DF0DECF1EF0DECF1FF0216A010E45
:10886800206E20EE01F02450D9262550DA22DF5060
:10887800C0EC4FF0000901E082D020EE03F0245054
:10888800D9262550DA22DF6A20EE17F02450D9269F
:108898002550DA2210EE1FF02450E1262550E2225E
:1088A800E6CF2AF0E6CF2BF0E6CF2CF0E6CF2DF07E
:1088B80010EE2BF02450E1262550E222E6CF2EF0D0
:1088C800E6CF2FF0E6CF30F0E6CF31F02A502E5C1D
:1088D800326E2B502F58336E2C503058346E2D502A
:1088E8003158356EDE50325CDE503358DE50345825
:1088F800DE50355846E220EE02F02450D9262550A5
:10890800DA22020EDE183DE12F0E24241A6E000E24
:1089180025201B6E20EE17F02450D9262550DA2288
:10892800DECF26F0DECF27F0DECF28F0DECF29F02D
:1089380020EE2BF02450D9262550DA22DECF2AF05B
:10894800DECF2BF0DECF2CF0DECF2DF026502A2400
:108958001C6E27502B201D6E28502C201E6E29506F
:108968002D201F6E216A010E206E20EE01F024508A
:10897800D9262550DA22DF50C0EC4FF002D0010E84
:10898800366E3650120046C00CF047C00DF06D0E22
:108998000E6E57EC53F000016C6F6C5101E099D0EA
:1089A80020EE0EF04650D9264750DA22DFAC91D09F
:1089B8006DC037F06EC038F020EE1CF04650D92656
:1089C8004750DA22DECF39F0DECF3AF0DECF3BF087
:1089D800DECF3CF0F6EC54F000016C6F6C5179E19D
:1089E80020EE20F04650D9264750DA22DECF6FF02D
:1089F800DDCF70F020EE0BF06F51D9267051DA22DE
:108A0800000EDB8A46C0D9FF47C0DAFFDECF0FF081
:108A1800DDCF10F06FC011F070C012F020EE06F03C
:108A28004650D9264750DA22DECF13F0DECF14F0B5
:108A3800DECF15F0DECF16F09DEC5DF01C0E0001C8
:108A48006F250B6E000E70210C6E20EE0AF046505A
:108A5800D9264750DA22DECF0DF0DECF0EF0DECF7A
:108A68000FF0DECF10F041EC5AF0160E00016F2522
:108A78000B6E000E70210C6E0D6A0E6A210E0F6EC1
:108A8800500E106E41EC5AF0120E00016F250B6E5D
:108A9800000E70210C6E000E0E6A0D6A02EC60F07A
:108AA800000120EE03F06D51D9266E51DA22010E35
:108AB800DF6E6DC043F06EC044F0DEEC40F00001A4
:108AC8006C6F20EE0EF04650D9264750DA22BF0EC2
:108AD800DF166C51120089688B688E280BE1770EBF
:108AE80000019C6FFB0E9D6F8ECF9EF09F6BCAECB2
:108AF80060F00AD04A0E00019C6FFA0E9D6F8ECF6F
:108B08009EF09F6BCAEC60F090280AE1340E9C6FCF
:108B1800FC0E9D6F8ECF9EF09F6BCAEC60F009D063
:108B28006F0E9C6FFA0E9D6F8ECF9EF09F6BCAECF6
:108B380060F0290E3F6E960E3E6E7F0EE82EFED731
:108B48003E2EFCD73F2EFAD700F0980E00019C6FFE
:108B5800FE0E9D6FCAEC60F089988498090E3F6EEE
:108B68001E0E3E6EE40EE82EFED73E2EFCD73F2E9C
:108B7800FAD700D08B0E00019C6FFE0E9D6FCAECD9
:108B880060F0899A849A090E3F6E1E0E3E6EE40EBE
:108B9800E82EFED73E2EFCD73F2EFAD700D0F00E97
:108BA80000019C6FFE0E9D6FCAEC60F088908D905E
:108BB80090280AE0340E9C6FFC0E9D6F90CF9EF0BB
:108BC8009F6BCAEC60F009D0FF0E9C6FF90E9D6F89
:108BD80090CF9EF09F6BCAEC60F08D80A30E3F6E25
:108BE800570E3E6E020EE82EFED73E2EFCD73F2EC5
:108BF800FAD700D089688B688A6883928382290EA5
:108C08003F6E960E3E6E7F0EE82EFED73E2EFCD7A8
:108C18003F2EFAD700F05BEC3CF0EFD71C6A1AAE97
:108C280012D01A1E191E181E171E161E151E141EE7
:108C3800136C000E1422152216221722182219224C
:108C48001A22010E1C6E12AE12D0121E111E101E18
:108C58000F1E0E1E0D1E0C1E0B6C000E0C220D227C
:108C68000E220F22102211221222010E1C1A1D6A36
:108C78001E6A1F6A206A216A226A236A246A1350BC
:108C88001410151016101710181019101A1045E0A6
:108C9800010E1B6E0AD0D8901336143615361636C8
:108CA8001736183619361A361B2A1AAEF4D7D89042
:108CB8001D361E361F3620362136223623362436F8
:108CC80013500B5C14500C5815500D5816500E5874
:108CD80017500F5818501058195011581A50125848
:108CE80011E313500B5E14500C5A15500D5A1650C0
:108CF8000E5A17500F5A1850105A1950115A1A5024
:108D0800125A1D80D8901A32193218321732163278
:108D18001532143213321B2ECAD71C5010E0241EF1
:108D2800231E221E211E201E1F1E1E1E1D6C000E2D
:108D38001E221F22202221222222232224221DC079
:108D48000BF01EC00CF01FC00DF020C00EF021C0AB
:108D58000FF022C010F023C011F024C012F012004E
:108D6800166817680B50D96EDA6ADECF18F0DDCFB7
:108D780019F018C013F019C014F01850191003E1B5
:108D88000B680C68120013C0F6FF14C0F7FF000E42
:108D9800F86E0E0EF76403D00800F55005D0F6CF34
:108DA800E9FFF7CFEAFFEF50156E134A142A200E99
:108DB800156403D03A0E1518E6E13A0E151868E165
:108DC800000E126E010E116E18C0F6FF19C0F7FFE3
:108DD800000EF86E0E0EF76403D00800F55005D0AB
:108DE800F6CFE9FFF7CFEAFFEF500D6E2F0E0D64B7
:108DF80039D018C0F6FF19C0F7FF000EF86E0E0E36
:108E0800F76403D00800F55005D0F6CFE9FFF7CF97
:108E1800EAFFEF500D6E3A0E0D6024D0020E1824B2
:108E28000D6E000E19200E6E13500D181BE1145014
:108E38000E1818E118C0F6FF19C0F7FF000EF86EFB
:108E48000E0EF76403D00800F55005D0F6CFE9FF01
:108E5800F7CFEAFFEF500D6ED00E0D24116E126A97
:108E6800FF0E122212BE04D012500DE111040BE2C3
:108E780011C016F012C017F00B50D96EDA6A13C081
:108E8800DEFF14C0DDFF16C00BF017C00CF0120097
:108E98000B6A0C6A120060C042F061C043F0446A79
:108EA800456A466A476AE2EC4DF042C078F043C032
:108EB80079F0020E0001781979110DE0795106E177
:108EC800030E785D03E26251631105E178C060F03A
:108ED80079C061F012007A6B7B6B7AC064F07BC05A
:108EE80065F0643B653BF00E651764510F0B651325
:108EF800F00E641760C066F061C067F064516627C1
:108F080065516723F50E66250B6E010E67210C6E01
:108F180001EC54F000017A51040DF350680FD96E3A
:108F2800DA6A0BC0DEFF0CC0DEFF0DC0DEFF0EC02C
:108F3800DEFF7A4B7B2B7B5103E1040E7A5DCDE398
:108F48006251631103E17A6B7B6B06D0FF0E6225D9
:108F58007A6FFF0E63217B6F7A51040DF350680F0F
:108F6800D96EDA6ADE50DE10DE10DE1004E1796BAD
:108F7800030E786F18D060C042F061C043F07A5198
:108F8800040DF350680FD96EDA6ADECF44F0DECFF5
:108F980045F0DECF46F0DECF47F0E2EC4DF042C0C0
:108FA80078F043C079F00001625163118FE1795183
:108FB80003E1020E785D8AE37A4B7B2B7B5186E1D5
:108FC800040E7A5D83E2C8D72F6C696664617461A8
:108FD800302E62696E20002F6C696664617461319D
:108FE8002E62696E20002F6C696664617461322E8E
:108FF80062696E20002F6C696664617461332E6249
:10900800696E20002F6C696664617461342E626930
:109018006E20002F6C696664617461352E62696E1A
:1090280020002F6C696664617461362E62696E2057
:10903800002F6C696664617461372E62696E200066
:109048002F6C696664617461382E62696E20002F26
:109058006C696664617461392E62696E20002F6CD8
:10906800696664617461612E62696E20002F6C69A3
:109078006664617461622E62696E20002F6C696695
:1090880064617461632E62696E20002F6C69666486
:10909800617461642E62696E20002F6C6966646178
:1090A8007461652E62696E20002F6C696664617454
:1090B80061662E62696E200000000000000000005A
:1090C8000000000000000000000000000000000098
:1090D8000000000000000000000000000000000088
:1090E8000000000000000000000000000000000078
:1090F800000000000BC015F00CC016F00F50101047
:1091080001E1120015C0D9FF16C0DAFF0DC0DFFF5C
:109118000F501524116E10501620126EFF0E1124D8
:10912800D96EFF0E1220DA6E0DC0DFFF105004E179
:10913800030E0F5C01E2120020EE01F01550D92653
:109148001650DA220DC0DFFF20EE02F01550D926A6
:109158001650DA220DC0DFFF0F501524116E105083
:109168001620126EFE0E1124D96EFF0E1220DA6E32
:109178000DC0DFFF0F501524116E10501620126E0F
:10918800FD0E1124D96EFF0E1220DA6E0DC0DFFF1E
:10919800105004E1070E0F5C01E2120020EE03F00C
:1091A8001550D9261650DA220DC0DFFF0F501524AE
:1091B800116E10501620126EFC0E1124D96EFF0E7F
:1091C8001220DA6E0DC0DFFF105004E1090E0F5CAB
:1091D80001E2120015C011F016C012F0111E121E85
:1091E800114A122A030E1114136E146A135015260D
:1091F8001450162213500F5E1450105AFC0E0F16FE
:109208000BD015C0D9FF16C0DAFF0DC0DFFF0F065F
:10921800D8A01006154A162A0F501010F2E11200B5
:10922800B3C0D9FFB4C0DAFFDECFB7F0DDCFB8F0F6
:10923800B3C074F0B4C075F0000E766F776F786FB6
:10924800796F5FEC33F0BA6FBA5103E00001BA519D
:109258001200B7C037F0B8C038F020EE16F0B3519E
:10926800D926B451DA22DECF39F0DECF3AF0DECF9C
:109278003BF0DECF3CF0F6EC54F00001BA6FBA5187
:10928800E5E120EE1AF0B351D926B451DA22DECF47
:10929800B5F0DDCFB6F0B5C0D9FFB6C0DAFFDF5004
:1092A800B96FB95103E1040EBA6FD0D720EE04F0BC
:1092B800B351D926B451DA2210EE1AF0B351E1268F
:1092C800B451E22200EE0BF0E650E926E550EA221E
:1092D800EF503F0BDF6E20EE1AF0B351D926B45190
:1092E800DA2210EE0BF0DE50E126DD50E222E7B67E
:1092F80018D020EE1AF0B351D926B451DA22DECFB5
:109308000BF0DDCF0CF01C0EB3250D6E000EB42152
:109318000E6E106A0B0E0F6E0BEC5AF00B500C1001
:1093280095E0B3C095F0B4C096F00001986B976BC8
:1093380044EC30F00001BA6FBA5188E18AD718C0FE
:109348000BF019C00CF00E6A0D6A106A080E0F6E49
:109358007EEC48F0236A020E226E22501824D96E41
:1093680023501920DA6E225018241E6E235019201B
:109378001F6E1E28E16E000E1F20E26EE750206E61
:10938800203AF00E2016201622501824E16E2350A1
:109398001920E26EE750216E21380F0B2010DF6E86
:1093A800224A232A23BED9D7235003E1070E225C81
:1093B800D4E322501824D96E23501920DA6E1AC02B
:1093C8000BF01BC00CF01CC00DF01DC00EF00A0EF7
:1093D8000F6E106A116A126AAAEC5AF00B3AF00E74
:1093E8000B1622501824E16E23501920E26EE75024
:1093F8001E6E1E380F0B0B10DF6E18C0D9FF19C078
:10940800DAFFDF2A1AC00BF01BC00CF01CC00DF0ED
:109418001DC00EF00A0E0F6E106A116A126A44EC33
:1094280058F00BC01AF00CC01BF00DC01CF00EC099
:109438001DF01A501B101C101D108CE118C0D9FF0C
:1094480019C0DAFFDF06090EDF64090C18C0D9FF5E
:1094580019C0DAFF100EDF6E100C000E0101E36F69
:109468000A0EE26F000EE16F050EE06F7DD001017C
:10947800E36B140EE26F70D08B0E0C6EFC0E0D6E4B
:10948800BEEC5BF08FB204D00101E36B1E0EE26FFD
:10949800090E0001FE6F1E0EFD6FE40EE82EFED7CA
:1094A800FD2FFCD7FE2FFAD700F056D0D80E0C6E41
:1094B800FE0E0D6EBEEC5BF0060E0001B16F090EDC
:1094C800B26FFE0EB36FF90EB46FB56B23EC56F0A6
:1094D80001019B6F9B513AEC5CF001019B51D8E173
:1094E800E36B230ED4D7290E0C6EFE0E0D6EBEEC68
:1094F8005BF0000E0001C96F030ECA6F400ECB6F00
:10950800020ECC6F010ECD6F1CEC15F001019B6FA4
:109518009B513AEC5CF001019B510AE12BEC29F0DC
:10952800000E486E030E496EFAEC5DF001019B6F68
:109538009B513AEC5CF0010CE2C1FDF0E3C1FEF096
:109548000001FE5109E1FD510A0A91E01E0A94E06A
:109558000A0AACE03D0AC7E0140E0101E219E31162
:1095680003E0E007D8A0E107E1BF000CE151E4E126
:10957800E005E2E2000C1C6A12AE12D0121E111EA7
:10958800101E0F1E0E1E0D1E0C1E0B6C000E0C2244
:109598000D220E220F22102211221222010E1C6E01
:1095A8001AAE10D01A1E191E181E171E161E151ECA
:1095B800141E136C000E14221522162217221822CC
:1095C80019221A22135014101510161017101810FB
:1095D80019101A103BE0010E1B6E0AD0D8901336F2
:1095E8001436153616361736183619361A361B2A13
:1095F8001AAEF4D713500B5C14500C5815500D5874
:1096080016500E5817500F58185010581950115816
:109618001A50125810E313500B5E14500C5A155080
:109628000D5A16500E5A17500F5A1850105A1950F2
:10963800115A1A50125AD8901A321932183217324F
:1096480016321532143213321B2ED4D71C5010E0A8
:10965800121E111E101E0F1E0E1E0D1E0C1E0B6C50
:10966800000E0C220D220E220F221022112212228D
:109678000BC00BF00CC00CF00DC00DF00EC00EF0BE
:109688000FC00FF010C010F011C011F012C012F08E
:109698001200020E0D5E000E0E5A0F5A105A20EEDE
:1096A80013F00B50D9260C50DA22FE0EDE24116E70
:1096B800FF0EDE20126EFF0EDE20136EFF0EDE2080
:1096C800146E11500D5C12500E5813500F58145050
:1096D800105805E30B6A0C6A0D6A0E6A120020EE38
:1096E80027F00B50D9260C50DA22DECF11F0DECF4E
:1096F80012F0DECF13F0DECF14F020EE09F00B509D
:10970800D9260C50DA22DECF15F0DDCF16F0155031
:10971800176E1650186E196A1A6A17500D02F3CF91
:109728001BF0F4CF1CF01D6A1E6A0E02F3501C26B3
:10973800F4501D22000E1E2218500D02F3501C2654
:10974800F4501D22000E1E2217500F02F3501D2642
:10975800F4501E2218500E02F3501D26F4501E22FB
:1097680019500D02F3501D26F4501E2210501702F6
:10977800F3501E2618500F02F3501E2619500E02E1
:10978800F3501E261A500D02F3501E2611501B24AA
:109798000B6E12501C200C6E13501D200D6E1450B1
:1097A8001E200E6E1200838E83800001F76BF86B0B
:1097B8007FEC58F01EC0F9F01FC0FAF0040E00014B
:1097C800FA5D07E3000EF925F76FFC0EFA21F86F32
:1097D80004D0F9C0F7F0FAC0F8F00101955133E070
:1097E80070517111721173112EE050500C0D630EEF
:1097F800F324D96E020EF420DA6E70C1A4F171C19F
:10980800A5F172C1A6F1A36B000EA325A76F010EE7
:10981800A421A86F000EA521A96F000EA621AA6F8A
:10982800DE50A71910E1DE50A8190DE1DE50A91984
:109838000AE1DE50AA1907E1000E226E040E236E1B
:109848009551B2EC56F08FB415D05050220D000E41
:10985800F3240001956F030EF420966F000E976FA6
:10986800040E986F010E9A6F996BF70E9B6FC9ECF7
:1098780008F0F66F0001F65109E0600E9C6FFD0ECE
:109888009D6FF6C09EF09F6BCAEC60F030EC27F03D
:109898008F6B8390839EEA0E00019C6FFC0E9D6F78
:1098A800CECF9EF09F6BCDCFA0F0A16BCAEF60F03A
:1098B800FCC120F071D04FEC60F0206EFC1979E00B
:1098C800290E1F6E960E1E6E7F0EE82EFED71E2ED8
:1098D800FCD71F2EFAD700F06CD0B3EC5CF0216EE9
:1098E800215067E021B0522A21B252060F0E5216BB
:1098F800000E0B6EC00E8BEC5CF0D9EC5FF0000E26
:109908000B6EC00E8BEC5CF052500F0D350EF3242D
:109918000F6E0D0EF420106E07EC58F0110E1F6E2E
:109928003C0E1E6ECB0EE82EFED71E2EFCD71F2E29
:10993800FAD700F021A43DD00C6A0B6A52C00DF092
:1099480034EC5EF0770E00019C6FFC0E9D6F52C0E8
:109958009EF09F6BCAEC60F052C020F0000E0B6EB8
:10996800800E8BEC5CF0D9EC5FF0000E0B6E800E75
:109978008BEC5CF052500F0D350EF3240F6E0D0E6C
:10998800F420106E07EC58F0000E0B6EC00E8BEC36
:109998005CF0D9EC5FF00DD0010197511E6E1F6A83
:1099A8001F5007E11E50010A86E0030A84E0010AFD
:1099B80094E02050120037C024F038C025F014EC91
:1099C80044F0000901E0010C37C00BF038C00CF07E
:1099D80039C00DF03AC00EF03BC00FF03CC010F09B
:1099E8004DEC4BF00BC041F00CC042F00DC043F001
:1099F8000EC044F020EE2BF03750D9263850DA222A
:109A080041C0DEFF42C0DEFF43C0DEFF44C0DEFFD0
:109A18002F0E37240B6E000E38200C6E0E6A0D6A5E
:109A2800020E106E0F6A3CEC60F02F0E37243F6E6A
:109A3800000E3820406E466A010E456E476A486A35
:109A480004D0455047264650482220EE09F03750AA
:109A5800D9263850DA22DE50475CDE5048581FE2DB
:109A68003FC01AF040C01BF0475041241C6E4850BC
:109A780042201D6E000E43201E6E000E44201F6EF5
:109A880045C020F046C021F020EE01F03750D9261D
:109A98003850DA22DF50C0EC4FF00009D2E020EE57
:109AA80009F03750D9263850DA224750DE1803E13A
:109AB8004850DE18D8A4010C000C1F6A206A186AE6
:109AC800196A01D0122A010E1E6E1250D96EDA6A76
:109AD800200EDE1813E0F70E146E15681250D96EBA
:109AE800DA6ADF50166E176A1450162615501722B8
:109AF800175003E1050E165C01E31E6A1EC01AF03A
:109B08001B6A1A501B1006E0DDD7196A010E186E81
:109B1800122A25D01250D96EDA6ADF50146E156AEF
:109B280015501DE114502B0AF3E0060AEEE017D099
:109B38000A0E1F02F3CF14F0F4CF15F02002F350F1
:109B480015261250D96EDA6ADF50145E000E155AC7
:109B5800300E14241F6E000E1520206ED9D7D00E9B
:109B6800146E15681250D96EDA6ADF50166E176ACD
:109B78001450162615501722175005E10A0E165CC8
:109B880002E2010E01D0000E1C6E1D6A1C501D1051
:109B9800CFE1185019100DE11FC014F020C015F0C6
:109BA800141E151E144A152A14C012F015C013F0FD
:109BB80012001FC012F020C013F0120020EE03F0B4
:109BC8004250D9264350DA22DF6A20EE2BF0425069
:109BD800D9264350DA22DE68DE68DE68DD6842C0D6
:109BE80037F043C038F044C039F045C03AF046C0B9
:109BF8003BF047C03CF0F6EC54F0000904E0436A3F
:109C0800040E426E040C2D0E42240B6E020E4320ED
:109C18000C6EDAEC5EF0550E0B1803E1AA0E0C1868
:109C280004E0436A030E426E030C20EE2FF042500C
:109C3800D9264350DA22E90EDE1812E020EE2FF082
:109C48004250D9264350DA22EB0EDE1809E020EE06
:109C58002FF04250D9264350DA22E80EDE1827E1C9
:109C6800650E42240B6E000E43200C6ED40E0D6E52
:109C7800FF0E0E6E106A030E0F6E0BEC5AF00B50AF
:109C88000C1003E1426A436A1200810E42240B6EF3
:109C9800000E43200C6E8E0E0D6EFF0E0E6E106AB7
:109CA800050E0F6E0BEC5AF00B500C10EBE0436AEC
:109CB800020E426E020C2C6EC60E00019C6FFC0E4A
:109CC8009D6F2CC09EF09F6B28C0A0F029C0A1F00A
:109CD800CAEC60F05DD0A7EC54F01EC02DF01FC098
:109CE8002EF020C02FF021C030F028C0D9FF29C0A5
:109CF800DAFFDF6A20EE01F02850D9262950DA224F
:109D080030C0DFFF20EE02F02850D9262950DA2291
:109D1800DF6A20EE03F02850D9262950DA222FC016
:109D2800DFFF20EE04F02850D9262950DA22DF6A16
:109D380020EE05F02850D9262950DA222EC0DFFF60
:109D480020EE06F02850D9262950DA22DF6A20EEC4
:109D580007F02850D9262950DA222DC0DFFF12003B
:109D6800A7EC54F01EC02DF01FC02EF020C02FF01D
:109D780021C030F028C018F029C019F02DC01AF001
:109D88002EC01BF02FC01CF030C01DF0A3EF49F00F
:109D98002C502A6E2B6A2B50D8A412002A50010A84
:109DA8009AE0030ADDE012000001F86B8380838EDD
:109DB8006AD07FEC58F01EC0F6F01FC0F7F0040E12
:109DC8000001F75D03E3010EF86F03D0FBC0F9F063
:109DD800FA6B8FB414D05050220D000EF324956FF7
:109DE800030EF420966F000E976F040E986F010E05
:109DF8009A6F996BF90E9B6FC9EC08F0FB6FFB51DA
:109E080009E0600E9C6FFD0E9D6FFBC09EF09F6B7E
:109E1800CAEC60F00101955133E070517111721173
:109E280073112EE050500C0D630EF324D96E020E00
:109E3800F420DA6E70C1A4F171C1A5F172C1A6F166
:109E4800A36B000EA325A76F010EA421A86F000E17
:109E5800A521A96F000EA621AA6FDE50A71910E14F
:109E6800DE50A8190DE1DE50A9190AE1DE50AA1941
:109E780007E1000E226E040E236E9551B2EC56F0E7
:109E880030EC27F08F6B0001F85193E0839E8390AC
:109E980012000F015969116B196B216B8C948C920C
:109EA8008C90889A110E106E3C0E0F6ECB0EE82E19
:109EB800FED70F2EFCD7102EFAD700F0110E106E19
:109EC8003C0E0F6ECB0EE82EFED70F2EFCD7102EB1
:109ED800FAD700F0020E106EA00E0F6E920EE82E4A
:109EE800FED70F2EFCD7102EFAD700D0000E0B6E1F
:109EF800300E8BEC5CF02A0E0F6E8E0EE82EFED71D
:109F08000F2EFCD7000E0B6E300E8BEC5CF0000EA3
:109F18000B6E300E8BEC5CF0000E0B6E390E8BEC7A
:109F28005CF0000E0B6E140E8BEC5CF0000E0B6EEA
:109F3800560E8BEC5CF0000E0B6E6D0E8BEC5CF02D
:109F4800000E0B6E700E8BEC5CF0000E0B6E0C0EA0
:109F58008BEC5CF0000E0B6E060E8BEC5CF0000ECA
:109F68000B6E010E8BEC5CF0D00E0F6ECA0EE82E55
:109F7800FED70F2EFCD71200236E2350D8A4040C52
:109F88002050211001E1040C54B0030C54B4020C0D
:109F980051B608D0090ED8901C361D361E361F360D
:109FA800E82EF9D7200421101AE11CC014F01DC0B6
:109FB80015F01EC016F01FC017F0180E6DEC5EF0FD
:109FC800000945E11AC00DF01BC00EF0FE0E0F6E21
:109FD80094EC5BF000093BE0206A216A38D051C05C
:109FE80022F0060E221609E020C014F021C015F058
:109FF800166A176A970E6DEC5EF01CC014F01DC04F
:10A0080015F01EC016F01FC017F0190E6DEC5EF0AB
:10A0180000091DE11AC00DF01BC00EF0FC0E0F6EFA
:10A0280094EC5BF0000908E0020E1B262006D8A07D
:10A03800210620502110EEE10D6A0E6AFD0E0F6E0A
:10A0480094EC5BF0000903E1216A010E206EF7EC45
:10A0580060F020502110D8A4010C000CB3C0D9FF27
:10A06800B4C0DAFFDECFBAF0DDCFBBF0B3C074F016
:10A07800B4C075F0000E766F776F786F796F5FEC0C
:10A0880033F0BE6FBE5153E1BC6BBD6BBAC037F045
:10A09800BBC038F020EE16F0B351D926B451DA22FD
:10A0A800DECF39F0DECF3AF0DECF3BF0DECF3CF04A
:10A0B800F6EC54F00001BE6FBE5139E120EE1AF003
:10A0C800B351D926B451DA22DECFB7F0DDCFB8F0DC
:10A0D800B7C0D9FFB8C0DAFFE50EDE1810E020EEF1
:10A0E8001AF0B351D926B451DA22DECFB7F0DDCF5A
:10A0F800B8F0B7C0D9FFB8C0DAFFDF5009E1BC4BF0
:10A10800BD2BB551BC1906E1B651BD1910E002D0FE
:10A11800BC6BBD6BB3C095F0B4C096F0986B010EE4
:10A12800976F44EC30F00001BE6FBE51AFE0040EF3
:10A13800BE1902E1070EBE6FBE511200838E8380E6
:10A148000001D16BD26BD36BD46B5050220D000E33
:10A15800F324746F030EF420756F350E766F0B0EB3
:10A16800776F010E796F786BD50E7A6F7B6BE4ECA5
:10A1780017F0D06F0101955135E0705171117211CE
:10A18800731130E050500C0D630EF324D96E020E9B
:10A19800F420DA6E70C1C7F071C1C8F072C1C9F09D
:10A1A8000001C66B000EC625CA6F010EC721CB6F12
:10A1B800000EC821CC6F000EC921CD6FDE50CA1920
:10A1C80011E1DE50CB190EE1DE50CC190BE1DE5067
:10A1D800CD1908E1350E286E0B0E296E0101955137
:10A1E8005FEC4EF00201B993D5C01EF0D6C01FF047
:10A1F80045EC38F01EC0CEF01FC0CFF00001CE51A4
:10A20800D127CF51D223000ED323D42301018F6B42
:10A21800839E83901200818E819CD00EF66E8F0EE5
:10A22800F76E000EF86E0DEE35F011EE2CF0090009
:10A23800F5CFEEFFE550E150FAE1E250F8E1B60E55
:10A24800F66EB50EF76E000EF86E02EE00F010EE28
:10A258005FF00900F5CFEEFFE550E150FAE1100E8E
:10A26800F66EC20EF76E000EF86E0900F5CFFEF11D
:10A278000900F5CFFFF1140EF66EC20EF76E000E50
:10A28800F86E0900F5CF54F005EE00F018EE35F041
:10A29800EE6AE550E150FCE1E250FAE104EE00F02C
:10A2A80011EE00F0EE6AE550E150FCE1E250FAE10F
:10A2B80003EE00F0AA0EEE6AE806FDE102EE5FF09A
:10A2C8005A0EEE6AE806FDE101EE00F09F0EEE6A16
:10A2D800E806FDE100EE4BF0090EEE6AE806FDE146
:10A2E80055905592000EF86E000132EF0FF0010103
:10A2F800906B4D6A806B816B020E8F6F83908E6BB3
:10A308008D6B506A030E506401D049D050500C0D2B
:10A31800620EF324D96E020EF420DA6EDF6A505012
:10A328000C0D610EF324D96E020EF420DA6EDF6A8A
:10A3380050500C0D5F0EF324D96E020EF420DA6E25
:10A34800DE6ADD6A50500C0D630EF324D96E020EDE
:10A35800F420DA6EDE6ADE6ADE6ADD6A50500C0DC1
:10A368006A0EF324D96E020EF420DA6E100EDF6E38
:10A3780050500C0D690EF324D96E020EF420DA6EDB
:10A38800020EDF6E50500C0D670EF324D96E020ECC
:10A39800F420DA6E240EDE6EDD6A502AB3D7100E72
:10A3A80002016A6F020E696F686B240E676F506A4C
:10A3B80001018C6B120050501C0D070EF324D96E4E
:10A3C800010EF420DA6E000EDE24BE6F010EDE20D0
:10A3D800BF6F000EDE20C06F000EDE20C16F000EC2
:10A3E800DE20C26F000EDE20C36F000EDE20C46FB9
:10A3F800000EDE20C56F50501C0D070EF324D96ED9
:10A40800010EF420DA6EBEC0DEFFBFC0DEFFC0C0A2
:10A41800DEFFC1C0DEFFC2C0DEFFC3C0DEFFC4C0B6
:10A42800DEFFC5C0DEFF50501C0D070EF324D96EA9
:10A43800010EF420DA6EDECFC6F0DECFC7F0DECF35
:10A44800C8F0DECFC9F05050220D000EF324956FEE
:10A45800030EF420966FC6C097F0C7C098F0C8C026
:10A4680099F0C9C09AF04EEC12F0CA6FCA5103E0D5
:10A47800010E4E6E010C4E6A1200BFC0D9FFC0C05B
:10A48800DAFFDECFC1F0DDCFC2F0BFC0B3F0C0C08D
:10A49800B4F0000EB66F010EB56F32EC50F0C36F1A
:10A4A800C35147E1C1C037F0C2C038F020EE16F002
:10A4B800BF51D926C051DA22DECF39F0DECF3AF0CB
:10A4C800DECF3BF0DECF3CF0F6EC54F00001C36F7A
:10A4D800C3512FE120EE1AF0BF51D926C051DA221C
:10A4E800DECF0BF0DDCF0CF00E6A0D6A106A200E7D
:10A4F8000F6E3CEC60F0000120EE1AF0BF51D92637
:10A50800C051DA22DECF0BF0DDCF0CF01C0EBF25D8
:10A518000D6E000EC0210E6E106A0B0E0F6E3CEC15
:10A528005DF020EE03F0C151D926C251DA22010EA6
:10A53800DF6EC35112008380838E000E0B6E040EF3
:10A548000C6E0E6AF60E0D6E010E106E0F6A7EEC22
:10A5580048F0470E00019C6FFE0E9D6FCAEC60F03C
:10A56800C66BC76BC6C0C2F0010EC217C233C23376
:10A578008350C2197F0BC219836E2E0EBFEC60F098
:10A588008FB415D05050220D000EF3240001956FA2
:10A59800030EF420966F000E976F040E986F010E4D
:10A5A8009A6F996BC30E9B6FC9EC08F0C56F0001D9
:10A5B800C55109E06C0E9C6FFF0E9D6FC5C09EF0E3
:10A5C8009F6BCAEF60F0C64BC72BC7BFCBD7C7512D
:10A5D80003E1640EC65DC6E31C0E9C6FFF0E9D6F03
:10A5E800CAEC60F0839E839083904E6A1200020149
:10A5F800B983505028E1350E0B6E0B0E0C6E550EBC
:10A608000D6E020E0E6E106A050E0F6EFAEC5CF0FF
:10A618003A0E0B6E0B0E0C6E000E0D6E020E0E6EC9
:10A62800106A130E0F6EFAEC5CF04D0E0B6E0B0EEB
:10A638000C6E260E0D6E020E0E6E106A0D0E0F6E4B
:10A64800FAEC5CF027D0350E0B6E0B0E0C6E5A0E22
:10A658000D6E020E0E6E106A050E0F6EFAEC5CF0AF
:10A668003A0E0B6E0B0E0C6E130E0D6E020E0E6E66
:10A67800106A130E0F6EFAEC5CF04D0E0B6E0B0E9B
:10A688000C6E330E0D6E020E0E6E106A0D0E0F6EEE
:10A69800FAEC5CF01F6A250E1E6E45EC38F00201DC
:10A6A800B99383901200090E156E0C500D103BE003
:10A6B8000CC0D9FF0DC0DAFFDE50DE1034E00CC04C
:10A6C800D9FF0DC0DAFFDECF0FF0DDCF10F00FC0DD
:10A6D800D9FF10C0DAFFDF5026E00CC0D9FF0DC04B
:10A6E800DAFF10EE05F0DE50E126DD50E22220EE22
:10A6F80002F00C50D9260D50DA22E650DE1813E18C
:10A70800E650DE1810E10CC0D9FF0DC0DAFF10EEDC
:10A7180001F0DE50E126DD50E222E750EDEC60F07A
:10A728000F6E0FA0156A155003E0136A146A08D05B
:10A738000CC0D9FF0DC0DAFFDECF13F0DDCF14F067
:10A748000E50D96EDA6A13C0DEFF14C0DDFF155053
:10A75800120050501C0D070EF324D96E010EF42080
:10A76800DA6EDECFE7F0DECFE8F0DECFE9F0DECF5D
:10A77800EAF0DECFEBF0DECFECF0DECFEDF0DECFAF
:10A78800EEF0E8C0E7F0E9C0E8F0EAC0E9F0EBC0B5
:10A79800EAF0ECC0EBF0EDC0ECF0EEC0EDF000013B
:10A7A800EE6BE7C0EFF0E8C0F0F0E9C0F1F0EAC006
:10A7B800F2F06DEC3BF0F56FF55102E0F551120047
:10A7C8008FB414D05050220D000EF324956F030E51
:10A7D800F420966F000E976F040E986F010E9A6F13
:10A7E800996BF30E9B6FC9EC08F0F66FF65102E017
:10A7F800F6511200DFEC51F0000C20EE03F00B5084
:10A80800D9260C50DA22DF50136E146A156A166ABC
:10A8180020EE02F00B50D9260C50DA22DF5013C07C
:10A8280010F014C011F015C012F00F6A0F10136E5B
:10A838001050146E1150156E1250166E20EE01F065
:10A848000B50D9260C50DA22DF5013C010F014C078
:10A8580011F015C012F00F6A0F10136E1050146E1D
:10A868001150156E1250166E0BC0D9FF0CC0DAFFCE
:10A87800DF5013C010F014C011F015C012F00F6AA9
:10A888000F10136E1050146E1150156E1250166E74
:10A8980013C00BF014C00CF015C00DF016C00EF06C
:10A8A8001200226E2250D8A4040C2050211001E17D
:10A8B800040C54B0030C51B608D0090ED8901C36BD
:10A8C8001D361E361F36E82EF9D7215006E1020E36
:10A8D800205C03E2246A110E02D0246A120E236E51
:10A8E80023C025F01CC014F01DC015F01EC016F0C2
:10A8F8001FC017F025506DEC5EF000091DE11AC06D
:10A908000BF01BC00CF0020E0E6E0D6A3AEC5BF0F9
:10A91800000908E0020E1B262006D8A021062050B8
:10A928002110EDE1120E251807E1146A156A166A5E
:10A93800176A0C0E6DEC5EF0F7EC60F020502110F9
:10A94800D8A4010C000C89EC5EF0CC0E8FEC60F002
:10A95800660E8FEC60F072EC60F0246E245005E116
:10A968001E6A1F6A206A216A1200226A236A22501C
:10A97800240FD96EDA6A72EC60F0DF6E224A232A5D
:10A9880023BEF5D7235003E1040E225CF0E3620EE8
:10A9980000019C6FFC0E9D6F24C09EF09F6B25C02C
:10A9A800A0F0A16B26C0A2F0A36B27C0A4F0A56BF2
:10A9B80024C0A6F025C0A7F026C0A8F027C0A9F09B
:10A9C800CAEC60F027502610251003E1060E245C1F
:10A9D800C7E324C01EF025C01FF026C020F027C002
:10A9E80021F01200416A20EE2BF03750D92638505A
:10A9F800DA223950DE1809E13A50DE1806E13B50F8
:10AA0800DE1803E13C50DE1839E037C024F038C0C6
:10AA180025F014EC44F0416E415030E12F0E3724FC
:10AA28001A6E000E38201B6E39C01CF03AC01DF09B
:10AA38003BC01EF03CC01FF0216A010E206E20EEC4
:10AA480001F03750D9263850DA22DF5055EC54F04F
:10AA5800000906E039683A683B683C68010E416EB7
:10AA680020EE2BF03750D9263850DA2239C0DEFFD5
:10AA78003AC0DEFF3BC0DEFF3CC0DEFF41501200A3
:10AA880003D00B4A0C2A0D2A0D50D96EDA6ADF5012
:10AA98000E6E0BC0F6FF0CC0F7FF000EF86E0E0E20
:10AAA800F76403D00800F55005D0F6CFE9FFF7CFDB
:10AAB800EAFFEF500E1813E10BC0F6FF0CC0F7FFCA
:10AAC800000EF86E0E0EF76403D00800F55005D09E
:10AAD800F6CFE9FFF7CFEAFFEF500009D2E10BC04C
:10AAE800F6FF0CC0F7FF000EF86E0E0EF76403D0E9
:10AAF8000800F55005D0F6CFE9FFF7CFEAFFEF5091
:10AB08000E6E0D50D96EDA6ADF500E5C0B6E0C6A51
:10AB1800D8A00C061200145015100AE178C114F0E0
:10AB280079C115F01450151003E1146A156A120062
:10AB380014C00FF015C010F016C011F05DEC5DF0F8
:10AB48000F5014261050152214C0D9FF15C0DAFF73
:10AB5800DF5006E10101786B796B146A156A1200FF
:10AB680014C00FF015C010F016C011F07DEC5DF0A8
:10AB78000F5014240101786F10501520796F78C197
:10AB8800D9FF79C1DAFFDF5009E078C1D9FF79C16F
:10AB9800DAFF000EDF6A784B792B02D0786B796B7D
:10ABA80014C014F015C015F01200A96BAA6B9FC051
:10ABB800ABF0A0C0ACF0A107D8A0A20727D0A3C0D3
:10ABC80074F0A4C075F0A50E766F776B796B010EE3
:10ABD800786FB10E7A6F7B6BE4EC17F0B105B211A8
:10ABE8001EE1A551AD6FAE6BAF6BB06BABC0D9FFBB
:10ABF800ACC0DAFFADC0DFFFAB4BAC2BA94BAA2B27
:10AC08000A0EAD19AE11AF11B01109E0A151A95D3D
:10AC1800AA51800A486EA251800A4858D0E3ABC0B6
:10AC2800D9FFACC0DAFFDF6AA951AA1103E19F6B13
:10AC3800A06B12009FC09FF0A0C0A0F01200B3C08C
:10AC4800B7F0B4C0B8F0B70E0B6EB4EC46F00BC05A
:10AC5800BBF00CC0BCF00001BCBF0B0CD890BB35DE
:10AC6800D96EBC35DA6E860ED926010EDA22DECF11
:10AC7800B9F0DDCFBAF0B951BA1105E0B9C0D9FFC2
:10AC8800BAC0DAFFDF6AB151B21105E0B1C0D9FF2D
:10AC9800B2C0DAFFDF6AD890BB35D96EBC35DA6E40
:10ACA800860ED926010EDA22B1C0DEFFB2C0DDFF62
:10ACB800B55101E1000CB30E7C6FB10E7D6F7E6B58
:10ACC8007F6BAFEC00F00001B66FB65112000BC0FD
:10ACD80012F00CC013F00DC014F00EC015F00F06E2
:10ACE800D8A010060F280CE110280AE10B6A0C6A9C
:10ACF8001200124A132A144A152A0F06D8A0100661
:10AD080012C0F6FF13C0F7FF0800F55015E014C095
:10AD1800D9FF15C0DAFFDF500FE00F5010100CE01C
:10AD280014C0D9FF15C0DAFF12C0F6FF13C0F7FF31
:10AD3800DE500900F518DDE012C0F6FF13C0F7FF7A
:10AD48000800F5CF11F014C0D9FF15C0DAFFDF50A5
:10AD5800115C0B6E0C6AD8A00C061200266E39D056
:10AD680020EE01F02250D9262350DA22DF502A6E35
:10AD780020EE03F02250D9262350DA22DF50296E24
:10AD880020EE05F02250D9262350DA22DF50286E13
:10AD980020EE07F02250D9262350DA22DF50276E02
:10ADA80027C00EF028C00FF029C010F02AC011F0FB
:10ADB800E8EF5BF022C00BF023C00CF048EC3DF04C
:10ADC8000BC027F00CC028F00DC029F00EC02AF0E7
:10ADD800E7D72650246E256A2550D8A4120024509F
:10ADE800010ABEE0030AE6E0120025EE04F0DE5098
:10ADF800DE10FBE000C513F001C514F0060E1324A5
:10AE0800D96E050E1420DA6EDF50116E060E13246B
:10AE1800D96E070E1420DA6EDF50126E134A142A08
:10AE28000D68010E0E6E13C00FF014C010F00D5017
:10AE38000F160E5010160FC000F510C001F5F29E47
:10AE480025EE04F0DE06000EDD5AF28E0BC0D9FFA7
:10AE58000CC0DAFF12C0DFFF25EE04F0010EDBBEE6
:10AE680005D0000EDE5C020EDE5801E28982115028
:10AE780012000E5002E00E5003E10C50B4EF60F0E7
:10AE88000E50D96EDA6A040ED926DE50DE1014E0B0
:10AE98000E50D96EDA6A040ED9260E50E16EE26AB7
:10AEA800020EE126DE50E65CE650800A136EDE50A4
:10AEB800800A1358D8B012000E50D96EDA6A020E02
:10AEC800D926DECF0FF0DDCF10F00E50D96EDA6A3A
:10AED800DECF11F0DDCF12F00F501124D96E1050D3
:10AEE8001220DA6E0CC0DFFF0E50D96EDA6A020E3D
:10AEF800D926DE2A000EDD22000CCF0E00019C6F41
:10AF0800FD0E9D6F82C19EF083C19FF0CAEC60F078
:10AF180011D0030E0BD0050E206E0101826B836BDE
:10AF28002DD00A0E03D0010E01D0020E206E26D0BD
:10AF3800206A24D082C11EF083C11FF01F5009E08F
:10AF4800020A0DE00E0A0FE0010A11E02A0A13E0D6
:10AF5800EFD71E500A0ADDE01E0ADDE0E9D71E50D1
:10AF6800BC0AE3E0E5D71E501C0ADBE0E1D71E501F
:10AF7800AC0AD9E0DDD71E500F0ADAE120501200E2
:10AF88000B500F02F3CF13F0F4CF14F0156A166AC2
:10AF98000B501002F3501426F4501522000E1622FE
:10AFA8000C500F02F3501426F4501522000E1622EE
:10AFB8000B501102F3501526F45016220C501002B3
:10AFC800F3501526F45016220D500F02F350152693
:10AFD800F450162212500B02F35016260C50110290
:10AFE800F35016260D501002F35016260E500F027D
:10AFF800F350162613C00BF014C00CF015C00DF05A
:10B0080016C00EF01200150E116EC60EE82EFED7F1
:10B01800112EFCD700D020D0150E116EC60EE82ECA
:10B02800FED7112EFCD700D0010E0B6E0FC0F6FF15
:10B0380010C0F7FF000EF86E0E0EF76403D008007C
:10B04800F55005D0F6CFE9FFF7CFEAFFEF508BECCC
:10B058005CF00F4A102AD7D70FC0F6FF10C0F7FFD1
:10B06800000EF86E0E0EF76403D00800F55005D0F8
:10B07800F6CFE9FFF7CFEAFFEF500009CDE1120064
:10B08800136A146A156A166A0F50101011101210FC
:10B0980029E0010E176E06D0D8900F3610361136FB
:10B0A8001236172A12AEF8D7D8901336143615363A
:10B0B80016360F500B5C10500C5811500D5812508A
:10B0C8000E5809E30F500B5E10500C5A11500D5AD0
:10B0D80012500E5A1380D8901232113210320F3299
:10B0E800172EE2D713C00BF014C00CF015C00DF0EA
:10B0F80016C00EF01200216A226A536A236A2ED003
:10B1080062EC60F00B500C101EE0230E0B6E0C6A04
:10B11800F9EC56F0206E23A80BD0FC0E00019C6FB2
:10B12800FE0E9D6F20C09EF09F6BCAEC60F00BD0A6
:10B13800000E5324D96EDA6A040EDA2220C0DFFF2B
:10B14800532A214A222A23AA07D0000E21241E6E40
:10B15800040E22201F6E12008EAC02D02204D0E30F
:10B1680021C01EF022C01FF012001A0E14240B6E0C
:10B17800000E15200C6EDAEC5EF00BC01AF00CC055
:10B188001BF01C6A1D6A12C0D9FF13C0DAFF030E38
:10B19800DE181CE1140E14240B6E000E15200C6E24
:10B1A800DAEC5EF00B50166E0C50176E186A196ABE
:10B1B80017C019F016C018F0176A166A16501A1236
:10B1C80017501B1218501C1219501D121AC012F0D9
:10B1D8001BC013F01CC014F01DC015F01200136E34
:10B1E8000C0E131807E0F7EC60F09CEC60F0000917
:10B1F80001E1FF0C13504009DDEC60F01050DDEC6C
:10B2080060F00F50DDEC60F00E50DDEC60F00D509A
:10B21800DDEC60F0010E126E135002E1950E126E15
:10B22800080E131802E1870E126E1250DDEC60F062
:10B238000C0E131802E1E6EC60F00A0E126EE6EC52
:10B2480060F0116E11AE02D0122EF9D71150120013
:10B2580083800201B98301018C050DE1000EE8CF5E
:10B2680035FB500EE8CF36FB000EE8CF37FBE8CFB2
:10B2780038FB8C6B1AD02BEE35F08DC1DFFF000E3A
:10B28800E8CF36FB0D0EE8CF37FB000EE8CF38FBD2
:10B298008FA403D0600EE8CF38FB8FA406D037CB3D
:10B2A80024F0200E241224C037FB1F6A040E1E6EE1
:10B2B80045EC38F00201B99301018D6B83901200BF
:10B2C8000F501010D8B4000C0FC0D9FF10C0DAFF0F
:10B2D800DF5001E1000C0FC00BF010C00CF01BECAC
:10B2E8005DF00BC011F00CC012F0020E1118121014
:10B2F80001E0000C130E0B6E0FC0D9FF10C0DAFF6F
:10B30800DF5011EC5CF00009D8B4000C140E0B6E81
:10B3180020EE01F00F50D9261050DA22DF5011EC40
:10B328005CF0000901E1000C1338F00B1410120056
:10B338000D6E350EF66EF90EF76E0900F5500D5CC0
:10B348002CE3360EF66EF90EF76E0D500900F55C1B
:10B3580004E30C6A010E0B6E010C370EF66EF90E43
:10B36800F76E0900F5500D5C08E3380EF66EF90E1D
:10B37800F76E0D500900F55CECE2390EF66EF90E29
:10B38800F76E0900F5500D5C08E33A0EF66EF90EFB
:10B39800F76E0D500900F55CDCE20B6A0C6A1200CE
:10B3A800866A846A8B688968536A839283940101E8
:10B3B8008A6B8B6B09D0000E8A25D96E040E8B21FF
:10B3C800DA6EDF6A8A4B8B2B8BBFF5D78B05F3E3DD
:10B3D8008A6B8B6B09D0350E8A25D96E0B0E8B21A3
:10B3E800DA6EDF6A8A4B8B2B8BBFF5D78B05F3E3BD
:10B3F8000F011769D6501F0B4009D66ED6980F0E4D
:10B40800D612D588D5120E01C29BD58E0F0C0BC053
:10B4180012F00CC013F00DC014F00EC015F012C0DD
:10B42800D9FF13C0DAFFDF50116E14C0F6FF15C044
:10B43800F7FF000EF86E0E0EF76403D00800F55003
:10B4480005D0F6CFE9FFF7CFEAFFEF50115C166E93
:10B45800176AD8A01706144A152A124A132A0F0683
:10B46800D8A010060F50101003E016501710D7E0A0
:10B4780016C00BF017C00CF012000BC0D9FF0CC09F
:10B48800DAFF0DC0DFFF0B4A0C2A0E500D6E0F506D
:10B498000E6E10500F6E106A0BC0D9FF0CC0DAFF89
:10B4A8000DC0DFFF0B4A0C2A0E500D6E0F500E6EAA
:10B4B80010500F6E106A0BC0D9FF0CC0DAFF0DC018
:10B4C800DFFF0B4A0C2A0E500D6E0F500E6E1050F7
:10B4D8000F6E106A0BC0D9FF0CC0DAFF0DC0DFFF7A
:10B4E8000B4A0C2A1200506A030E506401D02AD06D
:10B4F80050500C0D620EF324D96E020EF420DA6E51
:10B50800DF6A50500C0D610EF324D96E020EF42040
:10B51800DA6EDF6A50500C0D5F0EF324D96E020EFE
:10B52800F420DA6EDE6ADD6A50500C0D630EF324E7
:10B53800D96E020EF420DA6EDE6ADE6ADE6ADD6A31
:10B54800502AD2D7506A83908F6B12000F50101078
:10B558001110121023E0010E136E06D0D8900F368A
:10B56800103611361236132A12AEF8D70F500B5C6C
:10B5780010500C5811500D5812500E5808E30F5027
:10B588000B5E10500C5A11500D5A12500E5AD8908A
:10B598001232113210320F32132EE8D70BC00BF0D3
:10B5A8000CC00CF00DC00DF00EC00EF01200010919
:10B5B8001220010001001700002D119420D00F0067
:10B5C8000101091220010001001700002D1194202B
:10B5D800D00F000100004F01000F0000000009FF1C
:10B5E8000000004F01000F0000000009FF00687014
:10B5F8006469736B2E636667004850393132314491
:0DB60800000000800102E805800102E80555
:10B616000B6A0C6A50501C0D070EF324D96E010EEE
:10B62600F420DA6E070EDE6AE806FDE250501C0DC5
:10B636001B0EF324D96E010EF420DA6EDF6A505029
:10B646001C0D170EF324D96E010EF420DA6EDE6A95
:10B65600DE6ADE6ADD6A0B4A0C2A0CBEDBD70C50AA
:10B6660003E1040E0B5CD6E383904E6A1200070ECC
:10B67600106ED00E0F6E0FD0E6EC60F0116E112832
:10B686000DE1E40E00D000D0E82EFCD700D000D0AB
:10B696000F06D8A010060F501010EEE1FE0E11187E
:10B6A60001E0000CE6EC60F00BC0D9FF0CC0DAFF3D
:10B6B600DF6E0B4A0C2A0D06D8A00E060D500E1092
:10B6C600F1E1E6EC60F0E6EC60F0010C0BC011F085
:10B6D6000CC012F013D00F06D8A010060DC0D9FF6B
:10B6E6000EC0DAFF0D4A0E2A11C0E1FF12C0E2FFBA
:10B6F600114A122ADFCFE7FFE7500BE00F50101078
:10B7060008E0E9D711C0D9FF12C0DAFFDF6A114A93
:10B71600122A0F06D8A010060F28F4E11028F2E12D
:10B726001200A4EC5EF0000901E1000C0F50DDEC04
:10B7360060F0FD0E0F181EE0020E116E106A0DC0AD
:10B74600D9FF0EC0DAFFDF50DDEC60F00D4A0E2A9D
:10B756001006D8A0110610501110F1E1E6EC60F0C9
:10B76600E6EC60F0E6EC60F0126E12501F0B050A74
:10B7760001E0000C010C15D00CC0F6FF0DC0F7FF60
:10B78600000EF86E0E0EF76403D00800F55005D0D3
:10B79600F6CFE9FFF7CFEAFFEF50BFEC60F00C4AB7
:10B7A6000D2A0CC0F6FF0DC0F7FF000EF86E0E0E48
:10B7B600F76403D00800F55005D0F6CFE9FFF7CFC0
:10B7C600EAFFEF500009D8E112000EC012F00FC0D8
:10B7D60013F010C014F011C015F089EC5EF0CC0E19
:10B7E6008FEC60F0990E8FEC60F00C0E8FEC60F031
:10B7F600166A176A1650120FD96EDA6ADF508FEC86
:10B8060060F0164A172A17BEF5D7175002E089EFDF
:10B816005EF0040E165CEEE389EF5EF00C6E0B50E4
:10B8260001E1000C2F0E0C6409D03A0E0C6006D014
:10B836000B50D96EDA6A0C50D00F17D0400E0C643C
:10B8460009D0470E0C6006D00B50D96EDA6A0C5040
:10B85600C90F0BD0600E0C64000C670E0C60000C58
:10B866000B50D96EDA6A0C50A90FDF6E010C1F6EF1
:10B876003D0E206EF90E216E1E6A0AD020C0F6FF1C
:10B8860021C0F7FF204A212A0800F550F7E11E2AB9
:10B896001F501E1807E020C0F6FF21C0F7FF080062
:10B8A600F550ECE1550E00019C6FFE0E9D6F1FC01A
:10B8B6009EF09F6B20C0A0F021C0A1F0CAEF60F0FF
:10B8C6000D6E310EF66EF90EF76E0900F5500D5C31
:10B8D6001CE3320EF66EF90EF76E0D500900F55C9C
:10B8E60004E30C6A010E0B6E010C330EF66EF90EB4
:10B8F600F76E0900F5500D5C08E3340EF66EF90E8E
:10B90600F76E0D500900F55CECE20B6A0C6A12004A
:10B916000C6E87920A0EE82EFED700D00BB002D02E
:10B92600879401D08784000E0E6E010E0D6E0CAE4C
:10B9360002D0838A01D0839AD8900C36879000F083
:10B9460000F0878000F000F087900D4A0E2A0EBEA8
:10B95600EED70E5003E1090E0D5CE9E38782120073
:10B96600010E0B6E0C6A88868782878400F000F0D1
:10B97600879400F000F00D6A0E6A8DA602D00B5077
:10B986000C12D8900B36879000F000F0878000F0FC
:10B9960000F087900D4A0E2A0EBEEFD70E5003E137
:10B9A600030E0D5CEAE30C5012009F0E136E146832
:10B9B60011C015F012C016F0135015261450162299
:10B9C600165005E11A0E155C02E2010E01D0000EBA
:10B9D600176E186A1750181005E05F0E1114116ED5
:10B9E600126A120011C011F012C012F012000DC03E
:10B9F60013F00EC014F00BC011F00CC012F010D0F2
:10BA060013C0D9FF14C0DAFFDF50156E134A142A8B
:10BA160011C0D9FF12C0DAFF15C0DFFF114A122A82
:10BA26000F06D8A010060F28EBE11028E9E1120056
:10BA36000BC00DF00CC00EF002D00B4A0C2A0BC046
:10BA4600F6FF0CC0F7FF000EF86E0E0EF76403D07B
:10BA56000800F55005D0F6CFE9FFF7CFEAFFEF5023
:10BA66000009EBE10D500B5C0B6E0E500C580C6E82
:10BA760012000BC011F00CC012F00DC013F00EC076
:10BA860014F00F501010D8B4120013C0D9FF14C010
:10BA9600DAFF11C0E1FF12C0E2FFDFCFE7FF134A72
:10BAA600142A114A122A0F06D8A010060F50101099
:10BAB600ECE11200126A136A04D00F4A102A124AE5
:10BAC600132A0FC0D9FF10C0DAFFDF500EE011C0F5
:10BAD6000BF00FC0D9FF10C0DAFFDF500C6E0D6AF5
:10BAE60029EC60F00B500C10E8E112C00FF013C007
:10BAF60010F01200126A136A04D00F4A102A124A72
:10BB0600132A0FC0D9FF10C0DAFFDF500EE011C0B4
:10BB16000BF00FC0D9FF10C0DAFFDF500C6E0D6AB4
:10BB260029EC60F00B500C10E8E012C00FF013C0C7
:10BB360010F012001A0E11240B6E000E12200C6E5D
:10BB460013C00DF014C00EF002EC60F00FC0D9FF68
:10BB560010C0DAFF030EDE18D8A41200140E11244A
:10BB66000B6E000E12200C6E15C00DF016C00EF0F6
:10BB760002EF60F08F6B8380838E000E0B6E040ED7
:10BB86000C6E0E6AF60E0D6E010E106E0F6A7EECCE
:10BB960048F0470E00019C6FFE0E9D6FCAEC60F0E8
:10BBA6001C0E9C6FFF0E9D6FCAEC60F0839E839007
:10BBB60012000B6E0B500EE0FEEC60F0200EE82E2D
:10BBC600FED701EC61F0CC0E00D0E82EFDD700D0F8
:10BBD60000D01200FEEC60F0C00E00D0E82EFDD7BB
:10BBE60001EC61F0350EE82EFED700F0120048C0D9
:10BBF60046F049C047F0C7EC44F0736F735112E149
:10BC060048C00CF049C00DF0710E0E6E57EC53F0A3
:10BC16000001736F735106E148C0D9FF49C0DAFFCE
:10BC2600DE6ADD6A735112007D0E816F79C082F083
:10BC36007AC083F0846B856B866B876B820E736F1D
:10BC46007BC074F07CC075F0810E766F23EC05F036
:10BC5600000184517925D96E85517A21DA6EDF6A21
:10BC6600000C000EF2BE010E0E6E0C50030B7F6E22
:10BC76000BC07EFF0DC080FF3F0E81168184F29EB1
:10BC8600550E826EAA0E826E818281B2FED7819493
:10BC96000EB002D0F29E01D0F28E120002D00B4AF4
:10BCA6000C2A0BC0F6FF0CC0F7FF0800F55009E0A0
:10BCB6000BC0F6FF0CC0F7FF0800F5500D180E106C
:10BCC600EEE10BC0F6FF0CC0F7FF0800F5500B6E57
:10BCD6000C6A1200186E18AE0ED0189E0D6A0E6A07
:10BCE6000F6A106A370EF3EC58F0196E010E1964DC
:10BCF60002D01950120014C00DF015C00EF016C077
:10BD06000FF017C010F01850F3EF58F0FEEC60F08B
:10BD16000A0E0C6EF80EE82EFED70C2EFCD700D0BD
:10BD260001EC61F0E00E00D0E82EFDD7D4EC60F017
:10BD3600090E0C6E840EE82EFED70C2EFCD701EFF2
:10BD460061F0130E0C6E880E0B6E0ED0E6EC60F0F2
:10BD5600FF0A0DE0E40E00D000D0E82EFCD700D09C
:10BD660000D00B06D8A00C060B500C10EFE10B50C0
:10BD76000C10D8A4010C000C010E116E200E0B182D
:10BD86000C1011E0F70E0D6E0E680BC00FF00CC014
:10BD960010F00D500F260E501022105003E1050E24
:10BDA6000F5C01E3116A11C00BF00C6A120020EE61
:10BDB60001F00B50D9260C50DA22DF50106E116AB2
:10BDC6000BC0D9FF0CC0DAFFDF500D6E10500E6E9F
:10BDD6000D50106E0EC011F010C00BF011C00CF01B
:10BDE600120060900F0E0F01596F070E396F356FF5
:10BDF6004F0E936E8A6A8A888A828A82010E8F6EB5
:10BE0600130E0E01B76F0F0EFA6F100EFC6F140EA5
:10BE1600B86F140C9F0E0D6E0E68200E0B100F6E71
:10BE2600000E0C10106E0D500F260E5010221050E2
:10BE360005E11A0E0F5C02E2010E01D0000E0B6E38
:10BE46000C6A12001EBE04D01E500FE11D040DE246
:10BE56001DC01FF01EC020F01F1E201E1F4A202AD4
:10BE66001FC01DF020C01EF012001DC01DF01EC018
:10BE76001EF01200350E0B6E0B0E0C6E0E6A0D6A5E
:10BE8600010E106E0F6A7EEC48F02BEE35F08FC176
:10BE9600DFFF1F6A010E1E6E45EC38F001018F6B45
:10BEA6001200350E0B6E0B0E0C6E0E6A0D6A010E2D
:10BEB600106E0F6A7EEC48F0010EE8CF35FB0201EA
:10BEC600B9831F6A1E6E45EC38F00201B993120061
:10BED600186A196A09D017C00CF00D6A16C00EF060
:10BEE6003DEC57F0184A192A18501424D96E1950E7
:10BEF6001520DA6EDF50176E1750EDE112009F0E17
:10BF06000D6E0E680BC00FF00CC010F00D500F2612
:10BF16000E501022105005E11A0E0F5C02E2010EBF
:10BF260001D0000E0B6E0C6A1200BF0E0D6E0E686D
:10BF36000BC00FF00CC010F00D500F260E50102243
:10BF4600105005E11A0E0F5C02E2010E01D0000E40
:10BF56000B6E0C6A1200D00E0D6E0E680BC00FF041
:10BF66000CC010F00D500F260E501022105005E197
:10BF76000A0E0F5C02E2010E01D0000E0B6E0C6A77
:10BF860012009F869E84090E0E01FD6F9F98890EF2
:10BF96009B6E9C6A9E989D8E9D889D9AC599F28AF5
:10BFA600F28E9E909D9C9E9A9E8A1200106A110E99
:10BFB6000F6E09D00A0EE82EFED700D0010E0B6ECA
:10BFC600200E8BEC5CF00F06D8A010060F28F2E1CD
:10BFD6001028F0E112000B6E0B5009E0966A4F0E26
:10BFE600936E220E966E400E956E968A400C966A59
:10BFF600100E966E2A0E966E900E936EF4D70BC0A8
:10C00600D9FF0CC0DAFF0DC0DFFF0B4A0C2A0EC0A9
:10C016000DF00E6A0BC0D9FF0CC0DAFF0DC0DFFFB2
:10C026000B4A0C2A1200FEEC60F0200EE82EFED71A
:10C0360001EC61F0300EE82EFED7D4EC60F00C6E09
:10C04600B00E00D0E82EFDD70C5012000B50D96E62
:10C05600DA6A0C50DE1804E10BC00BF00C6A120011
:10C066000B2A0B04D96EDA6ADF50F0E10B6A0C6A10
:10C0760012000BC011F00CC012F011C0D9FF12C093
:10C08600DAFF0DC0DFFF114A122A0F06D8A01006EC
:10C096000F501010F2E11200070E8C6E9150070B34
:10C0A6000B6E888A8DAA02D0080E0B26020E01019D
:10C0B600971903E10B1C0F0B0B6E0B50120025EEAC
:10C0C60004F0010EDBBE05D0000EDE5C020EDE586B
:10C0D60001E2898204C50BF005C50CF012000D6A59
:10C0E6000E6AD8900D3216EC60F0000901E00D8E54
:10C0F6000E2A070E0E64F5D70D501200000EE8CF7B
:10C1060000F5E8CF01F5E8CF02F5E8CF03F5E8CF73
:10C1160004F5E8CF05F5000C0C6E0D6A0C50010B0A
:10C12600DCEC5DF0D8900C320D2A070E0D64F6D7C4
:10C13600070C06EC61F0E6EC60F0A4EC5EF000099A
:10C1460001E0010CF7EC60F0000C0C50030B7F6E65
:10C156000BC07EFF3F0E8116818000F000F08050FC
:10C1660012000B6E03D009EC61F004000E01CDA99C
:10C17600FAD70BC09AFF12000B6E03D009EC61F0E0
:10C1860004000E01CDA9FAD70BC09AFF12009E0E2D
:10C196001D6E9CC018F09DC019F01D0E1A6E20EF82
:10C1A60025F088888DA803D0010E0B6E01D00B6A8E
:10C1B6000B5012000B6E0BC092FF95B0FED795A0E8
:10C1C600FED792501200926895B0FED795A0FED782
:10C1D600925012000B6E0B5001E0010C54501200ED
:10C1E60083804E6A8390120004EC61F0E6EF60F003
:10C1F60083908F6B120083988898120083988888A2
:0FC20600120085801200859012001FE7120001C0
:10F9300000819FE0FC407E80FC000020004F4B00D7
:10F940004449534B5F455252004E4F545F5245411C
:10F950004459004E4F5F46494C45004E4F545F4F4F
:10F9600050454E4544004E4F545F454E41424C4534
:10F9700044004E4F5F46494C455F53595354454DE3
:10F9800000000D0A202532582025325820253273D8
:10F9900020253273202532732025327320253273BF
:10F9A00020253273202532732025327320253473AD
:10F9B0002025347320253473202534732025347397
:10F9C00020253473202534732025347320000D0A3C
:10F9D00048504469736B204D6B20494920283138C9
:10F9E0004634364B34302920257320257320257367
:10F9F000205374617274696E672E2E2E0D0A000DED
:10FA00000A4461746120706F7274206973202558F4
:10FA1000202D2053686F756C64206265203C3E2069
:10FA200030784646000D0A5365656B20657272207A
:10FA30002564203E2025642C202564203E2025645A
:10FA40002C202564203E202564000D0A5374617427
:10FA5000757320706F7274206973202558202D20D3
:10FA600053686F756C642062652030784646000DDF
:10FA70000A4461746120706F727420697320255884
:10FA8000202D2053686F756C6420626520307846A5
:10FA900046000D0A526420752025642072746E2081
:10FAA00025642C2025642062797465732072656159
:10FAB000640D0A000D0A4D617820566563746F72FB
:10FAC000206469736B20256420256C642028256CD4
:10FAD000582920000D0A253032582530325820533D
:10FAE0005338303A52707420515354415420256495
:10FAF00020000D0A44736B73656C206973202564C4
:10FB00002C206E756D62657220697320256420005B
:10FB1000466F756E6420616E205254432066696C96
:10FB2000652061742025580D0A004C6F6F6B696E5B
:10FB30006720666F7220616E205254432066696CA4
:10FB4000650D0A000D0A5573696E67206469736B51
:10FB50002067656F6D657472792025732000466992
:10FB60006E6446696C65206661696C6564207365C6
:10FB7000617263680D0A000D0A5374617475732015
:10FB8000706F7274206973202558202D204F4B0010
:10FB90000D0A5365656B20746F20256C64206661C7
:10FBA000696C6564202564000D0A454550524F4D2F
:10FBB000206469736B206E756D6265722025640028
:10FBC0000D0A4469736B2073656C656374206E75F0
:10FBD0006D626572202564005365656B696E6720F0
:10FBE000746F20736563746F722025580D0A004688
:10FBF000696E6446696C65206661696C6564207233
:10FC00006561640D0A000D0A5472616E7370617251
:10FC1000656E7420756E697420255820000D0A4F9A
:10FC200070656E696E67206578697374696E6720A8
:10FC3000257320000D0A4461746120706F72742076
:10FC40006973202558202D204F4B000D0A476F74F3
:10FC500020256C7520202D20726573657474696E83
:10FC60006700202558202558202558202558202574
:10FC70006C752020200A000D0A57726F746520648D
:10FC800069736B6E6F3A20256420000D0A57616915
:10FC900074696E6720666F72206361726420003C35
:10FCA0006964656E743E20255820255820256420FF
:10FCB0002564000D0A46696C652025732069732050
:10FCC0006F70656E20000D0A7274635F7265616407
:10FCD0002825642C255829000D0A4F70656E696E21
:10FCE00067206E657720257320000D0A2530325875
:10FCF00025303258204578697420004E6F74206199
:10FD0000204C4946206469736B0D0A000D0A526548
:10FD1000616420646573637269626520000D0A4640
:10FD2000696C6520255820697320257320000D0A11
:10FD30004469736B202558206973202573200020A7
:10FD400041544E20617373657274656420256400AC
:10FD50000D0A48737420627974657332202564003B
:10FD60000D0A5772697465206661696C202564000C
:10FD70000D0A52656164696E67205254430D0A0092
:10FD80000D0A416D69676F2039313231440D0A0027
:10FD90000D0A53532F38302039313232440D0A00C6
:10FDA0000D0A44736B73656C206973202564200011
:10FDB0000D0A5265616420256420627974657300C0
:10FDC000566563746F722069732025580D0A000D03
:10FDD0000A53533830657865632025642000222A51
:10FDE0002B2C3A3B3C3D3E3F5B5D7C7F000D0A4F38
:10FDF00070656E696E672025732020000D0A4465CA
:10FE000062756720697320256420000D0A436C6FBA
:10FE1000636B20697320256420000D0A50726F7493
:10FE20006F20697320256420000D0A5265616420EB
:10FE3000636F6E66696720000D0A46696C656E61C6
:10FE40006D6520257320000D0A466F726D61747414
:10FE5000696E67200072633D25752046525F2573E9
:10FE60000D0A002A2A204E4F204449534B202A2AAB
:10FE7000002A2A20566572696679202A2A000D0A0E
:10FE800073627974657331202564000D0A417373C0
:10FE900065727420454F49000D0A41737365727491
:10FEA0002041544E000D0A4E6F206361726420257C
:10FEB000640064657363726962652E636667002F10
:10FEC0006C6966646174612E62696E00EB769045C0
:10FED00058464154202020000D0A4D6F756E7469FC
:10FEE0006E6720004A756E20203720323032310094
:10FEF0000D0A4173736572742050500020255820FC
:10FF0000772041544E20004C6F6164696E672E2E3D
:10FF10002E002A2A20525141202A2A00466D7420A0
:10FF20006578697420000D0A53746174757300312B
:10FF3000303A34393A3035000D0A494431202558D9
:10FF4000000D0A494432202558005B2532582025EF
:10FF5000645D004572726F722025640048504469E8
:10FF6000736B20004E6F20636172640072633D25E5
:10FF700064200044534B53454C004E414D45255899
:10FF8000004449534B2558000D0A44534A0046414A
:10FF90005433320044454255470050524F544F00AD
:10FFA0005265616479007B4552527D00302E3139B3
:10FFB000004946432000454F49200052454E20004D
:10FFC000535251200044415620004E444143004EBC
:10FFD000524644004641540052544300434C4B00A7
:10FFE000253258004430004431004432004433008C
:0FFFF0004434004435004436004437002B0000F1
:020000040020DA
:10000000FF0FFF0FFF0FFF0FFF0FFF0FFF0FFF0F80
:020000040030CA
:0C0000008CFFFFFC8EFFFFFFFFFFFFFFE7
:00000001FF
